:10000000000001206D03010095030100970301002A
:10001000990301009B0301009D0301000000000003
:100020000000000000000000000000009F0301002D
:10003000A103010000000000A3030100A5030100CB
:10004000A7030100A703010025090100A703010080
:10005000E9AC0000A7030100A7030100A70301000A
:10006000A7030100A7030100A7030100A7030100E4
:10007000A7030100A7030100A7030100A7030100D4
:10008000A7030100E90C0100A7030100A703010079
:10009000A7030100A7030100A7030100A7030100B4
:1000A000A7030100A7030100A7030100A7030100A4
:1000B000A7030100A70301000000000000000000EA
:1000C000A7030100A7030100A7030100A703010084
:1000D000A7030100A7030100A7030100000000001F
:1000E0000000000000000000000000000000000010
:1000F0000000000000000000000000000000000000
:1001000000000000000000000000000000000000EF
:1001100000000000000000000000000000000000DF
:1001200000000000000000000000000000000000CF
:1001300000000000000000000000000000000000BF
:1001400000000000000000000000000000000000AF
:10015000000000000000000000000000000000009F
:10016000000000000000000000000000000000008F
:10017000000000000000000000000000000000007F
:10018000000000000000000000000000000000006F
:10019000000000000000000000000000000000005F
:1001A000000000000000000000000000000000004F
:1001B000000000000000000000000000000000003F
:1001C000000000000000000000000000000000002F
:1001D000000000000000000000000000000000001F
:1001E000000000000000000000000000000000000F
:1001F00000000000000000000000000000000000FF
:1002000010B5054C237833B9044B13B10448AFF350
:1002100000800123237010BDA00200200000000018
:10022000B8A1010008B5034B1BB103490348AFF364
:10023000008008BD00000000A4020020B8A1010059
:10024000154B002B08BF134B9D46A3F5803A0021A8
:100250008B460F461348144A121A13F076F80F4BC8
:10026000002B00D098470E4B002B00D09847002061
:10027000002104000D000D48002802D00C48AFF307
:10028000008012F0ABFF2000290010F06DFD12F08D
:10029000F3FD00BF00000800000001200000000086
:1002A00000000000A00200208809002000000000DB
:1002B000000000000020704700207047F0B50446A1
:1002C00085B00E46684611461F460AF08DF8236831
:1002D0006A465D6A31463B462046A84705B0F0BDF8
:1002E000F0B5044685B00E46684611461F4609F033
:1002F00086FF23686A465D6A31463B462046A8472A
:1003000005B0F0BD70B590B00C4615461E4605F020
:100310000DFE48B364B321464022684613F0E9FF5E
:100320002F21684613F07CFF28B923460322402181
:10033000684609F0D7FF3F223146684613F0B3FF05
:100340000C480EF0DDFE78B10B4B93F90030062B14
:100350000CD10A4B93F9003043B901232A46694670
:1003600004480FF02AF9012010B070BD0020FBE70F
:100370002046F9E7E8030020E0030020B80300204E
:1003800007B5002300931A46194603480FF026FECE
:1003900003B05DF804FB00BFBC02002007B50023DA
:1003A00000931A46194603480FF018FE03B05DF893
:1003B00004FB00BFC402002082B002AB012003E9AD
:1003C000060002B0704700207047406818B14068CE
:1003D00008B1007C0009704743682BB15B681BB112
:1003E0001A7C61F307121A747047406808B508B1A7
:1003F00001F08CFF012008BD13B500220446114610
:10040000684604F01BF9606801F080FF052807D8F2
:10041000DFE800F0110311060611012002B010BD43
:1004200061684FF40072684604F0FDFC00216846E4
:1004300004F0CCFBF2E70020F0E713B500220446FD
:100440001146684604F0FAF82046FF22694604F097
:1004500039FC204602B010BD07B5002300931A46B0
:10046000194603480FF0BAFD03B05DF804FB00BF66
:10047000CC020020704700002DE9FF4102AC84E867
:10048000060006463B493C489DF828809DF82C50C4
:100490001F460FF0EBFD204604F0B4FE204604F0AA
:1004A00052FA50BB204604F0B5FC052804D8DFE81A
:1004B00000F0152417030317054630492E480FF0A6
:1004C000D5FD0A2229462C480FF039FE2A480FF0A4
:1004D000DDFD204604F096FE00200BE04FF0010801
:1004E000CDE90085336894E80600DD6B30463B4675
:1004F000A847012004B0BDE8F081204604F0D2FBFB
:10050000012812D0022831D01D491B480FF0AEFD42
:10051000204604F0C7FB0A22014617480FF028FEC8
:1005200015480FF0B3FD0125C7E70021204604F070
:100530009FFA13280ED81E21204604F009FB71688B
:100540004FF40072204604F0C3FC4FF490517068E1
:1005500002F03CFD0195336801250095D3F83C80FD
:1005600094E806003B463046C047C2E700230393A9
:10057000F0E700BF847D0100700300209A7D010038
:100580008D7D010008B511B9B0F9080008BDB0F9BA
:100590000A208A4203DC0089084400B2F6E740687A
:1005A00001F04CFFF9E7000007B5002300931A465D
:1005B000194603480FF012FD03B05DF804FB00BFBD
:1005C000D40200200A460068022100F0A1BD00000C
:1005D00070B503680546F3B17221FFF7F3FF286891
:1005E0000E4E03680021DB69984700242868042C1C
:1005F00003680CD0DB689847A35D984205D0286853
:1006000003685B6A9847002070BD0134EEE75B6ABF
:1006100098470120F8E71846F6E700BFF47D01008F
:100620002DE9F041036804461BB900263046BDE8B9
:10063000F081FFF7CDFF07460028F6D0254672214E
:100640002046FFF7BFFF55F8100B03680421DB6954
:10065000984704F11608002620680368DB6898476D
:10066000C0B205F8010B0138C0B2FD2898BF3E4664
:10067000A845F1D1206803685B6A9847D6E7F8B5CA
:10068000036804460F4613B900252846F8BDFFF756
:100690009FFF05460028F7D072212046FFF792FF02
:1006A000206803682646DB690421984756F8100B3A
:1006B000036806225B68394698473B682361BB881C
:1006C000B380206803685B6A9847DEE770B503680B
:1006D00004460D46164613B90025284670BDFFF79F
:1006E00077FF0028F8D072212046FFF76BFF2068C3
:1006F00003684021DB699847731E2A460021206861
:100700000FF098FF06B2206803685B6A9847002ED6
:10071000E2D00023AB55E0E738B5036804460D4648
:100720000BB9002038BDFFF753FF0028F9D0284649
:1007300013F0B1FD0F28F4D872212046FFF742FFD5
:10074000206803684021DB699847294620680FF03C
:1007500096FC2068036800211B68984705462068BE
:1007600003685B6A9847281C18BF0120DAE738B590
:10077000036804460D460BB9002038BDFFF728FF7B
:100780000028F9D0284613F086FD0F28F4D87221EE
:100790002046FFF717FF206803685021DB69984760
:1007A000294620680FF06BFC2068036800211B6855
:1007B00098470546206803685B6A9847281C18BF5D
:1007C0000120DAE770B5036804460D46164613B9F2
:1007D0000025284670BDFFF7FBFE0028F8D07221E7
:1007E0002046FFF7EFFE206803682021DB69984769
:1007F000731E2A46002120680FF01CFF06B22068F5
:1008000003685B6A9847002EE2D00023AB55E0E70F
:1008100038B5036804460D460BB9002038BDFFF714
:10082000D7FE0028F9D0284613F035FD1F28F4D84C
:1008300072212046FFF7C6FE206803682021DB698D
:100840009847294620680FF01AFC206803680021A9
:100850001B6898470546206803685B6A9847281C10
:1008600018BF0120DAE773B5036805460E461BB9C9
:100870000024204602B070BDFFF7AAFE04460028FF
:10088000F6D072212846FFF79DFE286803681021E4
:10089000DB69984704220DEB020128680FF0B5FED2
:1008A000019930460FF0B7FB286803685B6A9847E8
:1008B0003379002BDCD0FF2BDBD17379FF2BD8D120
:1008C000B379FF2BD5D1F479FF3C18BF0124D0E7D1
:1008D00073B5036805460E461BB90024204602B0D6
:1008E00070BDFFF775FE04460028F6D07221284639
:1008F000FFF768FE286803681C21DB69984704221B
:100900000DEB020128680FF080FE019930460FF0D0
:1009100082FB286803685B6A98473379002BDCD038
:10092000FF2BDBD17379FF2BD8D1B379FF2BD5D136
:10093000F479FF3C18BF0124D0E773B5036805467E
:100940000E461BB90024204602B070BDFFF740FEE2
:1009500004460028F6D072212846FFF733FE2868A7
:1009600003681421DB69984704220DEB0201286813
:100970000FF04BFE019930460FF04DFB28680368DD
:100980005B6A98473379002BDCD0FF2BDBD173797E
:10099000FF2BD8D1B379FF2BD5D1F479FF3C18BF09
:1009A0000124D0E773B5036805460E461BB9002441
:1009B000204602B070BDFFF70BFE04460028F6D0BB
:1009C00072212846FFF7FEFD286803681821DB69BD
:1009D000984704220DEB020128680FF016FE0199DA
:1009E00030460FF018FB286803685B6A9847337934
:1009F000002BDCD0FF2BDBD17379FF2BD8D1B3795F
:100A0000FF2BD5D1F479FF3C18BF0124D0E737B5CF
:100A10004B6801930368044613B9002003B030BD4E
:100A2000FFF7D6FD0028F8D072212046FFF7CAFD57
:100A3000206803681021DB69984720680368042256
:100A40005B680DEB020198470546206803685B6A06
:100A50009847281C18BF0120E0E737B54B68019381
:100A60000368044613B9002003B030BDFFF7B0FDA2
:100A70000028F8D072212046FFF7A4FD2068036803
:100A80001C21DB6998472068036804225B680DEB32
:100A9000020198470546206803685B6A9847281C4E
:100AA00018BF0120E0E737B54B680193036804469F
:100AB00013B9002003B030BDFFF78AFD0028F8D03D
:100AC00072212046FFF77EFD206803681421DB6950
:100AD00098472068036804225B680DEB0201984781
:100AE0000546206803685B6A9847281C18BF0120E8
:100AF000E0E737B54B6801930368044613B900205B
:100B000003B030BDFFF764FD0028F8D07221204605
:100B1000FFF758FD206803681821DB6998472068B3
:100B2000036804225B680DEB0201984705462068C4
:100B300003685B6A9847281C18BF0120E0E713B5DB
:100B4000E723009303680446A3B1FFF741FD88B192
:100B500072212046FFF736FD206803680C21DB690F
:100B600098470422694620680FF04FFD206803680B
:100B70005B6A9847009B0020DAB262F30700C3F378
:100B8000072262F30F20C3F3074262F317401B0EE4
:100B900063F31F6002B010BD37B5019103680446CE
:100BA00013B9002003B030BDFFF712FD0028F8D0C4
:100BB00072212046FFF706FD206803680C21DB69DF
:100BC00098472068036804225B680DEB0201984790
:100BD0000546206803685B6A9847281C18BF0120F7
:100BE000E0E707B5FFF7ABFF80F48070C0F30020AB
:100BF00003B05DF804FB37B505460C46FFF79FFFD1
:100C000084F001040190C0F3072064F300008DF824
:100C100005000199284603B0BDE83040FFF7BCBF8E
:100C200007B5FFF78CFFC0F3402003B05DF804FB6D
:100C300037B50D460446FFF782FF0190C0F3072049
:100C400065F341008DF805000199204603B0BDE829
:100C50003040FFF7A1BF07B5FFF771FF80F010002C
:100C6000C0F3001003B05DF804FB37B505460C4631
:100C7000FFF765FF84F00104019064F304108DF820
:100C800004000199284603B0BDE83040FFF784BF57
:100C900037B50D460446FFF752FF019065F3030098
:100CA0008DF804000199204603B0BDE83040FFF7FD
:100CB00073BF37B50D460446FFF741FF019065F35A
:100CC00047108DF804000199204603B0BDE830407C
:100CD000FFF762BF07B5FFF732FF00F00F0003B068
:100CE0005DF804FB07B5FFF72AFFC0F3421003B01D
:100CF0005DF804FB70B51E4D0C468AB00646043400
:100D00001C4928460FF0B2F9214607A80FF0CFFE84
:100D100007A928460FF0AEF92846174D0FF0B6F98F
:100D200007A80FF034FE294601A80FF075FE01A9AF
:100D300004A80FF0BCFE214604A80FF0F8FE2946D7
:100D4000044607A80FF068FE07A920460FF0EFFE43
:100D5000014630460FF0ABFE07A80FF018FE04A8BE
:100D60000FF015FE01A80FF012FE30460AB070BD5C
:100D700070030020F97D0100047E01007FB50D465F
:100D80000446222128460FF027FF22210646284646
:100D90000FF03CFF002E034604F1040422DB002880
:100DA00020DD721C294601A80FF034FF01A920465E
:100DB0000FF087FE01A80FF0EAFD0D490D480FF076
:100DC00055F9214601A80FF072FE01A909480FF05C
:100DD00051F908480FF05AF901A80FF0D8FD012089
:100DE00004B070BD294620460FF052FEE5E700BF73
:100DF000067E0100700300207FB503680446002BC7
:100E000039D07721FFF7DEFB206803680021DB691A
:100E100098470025206802690368954204D21B6840
:100E2000002198470135F5E7DB69144E002198470A
:100E300000252068715D036801351B689847042D03
:100E4000F7D1206803685B6A98470D4901A80FF045
:100E5000E3FD01A92046FFF791FF01A80FF097FDE0
:100E600007212046FFF714FF07212046FFF721FF47
:100E7000012004B070BD1846FBE700BFF47D0100FF
:100E8000729C01007FB50368044613B9002004B0CA
:100E900070BDFFF79DFB0028F8D0E3681F2BF5D845
:100EA000264672212046FFF78DFB56F8040B036897
:100EB0006021DB699847314620680FF0DBF8206835
:100EC000036800211B6898470546206803685B6A31
:100ED00098478DB10A490B480FF0C8F8314601A870
:100EE0000FF0E5FD01A907480FF0C4F805480FF021
:100EF000CDF801A80FF04BFD281C18BF0120C6E754
:100F00001E7E01007003002030B5036885B00446E2
:100F100013B9002005B030BDFFF75AFB0028F8D008
:100F2000254672212046FFF74DFB55F8040B036858
:100F30006021DB6998470022216801A80FF094FB2B
:100F400001A928460FF0BDFD01A80FF020FD206883
:100F500003685B6A98470B490B480FF087F82946EE
:100F600001A80FF0A4FD01A907480FF083F8064877
:100F70000FF08CF801A80FF00AFDE068003018BFF0
:100F80000120C7E7117E01007003002007B5002390
:100F900000931A46194603480FF020F803B05DF895
:100FA00004FB00BFDC02002007B5002300931A46B3
:100FB000194603480FF012F803B05DF804FB00BFB8
:100FC000E402002001207047C08A704703699942FB
:100FD00028BF1946816108467047037D10B5044655
:100FE00033B9A069236998422CBF0020012010BDAD
:100FF00003681B699847FF28F3D10020F7E70368CF
:1010000010B504461B699847A3690133A36110BD5D
:101010007047000008B502698369934205D2C1692F
:10102000034819440EF029FE08BD4FF0FF30FBE7DE
:10103000EC02002010B5D0E906345A1C82610A4641
:101040000248E1180EF01BFE012010BDEC0200204A
:10105000037D10B504462BB10368FF211B68984738
:101060000023237510BD000008B590F82020772AD2
:101070000BD10368DB6A9847044905480EF0F6FF78
:101080000348BDE808400FF001B808BD437E0100E9
:1010900070030020F0B50D4685B004463F21284678
:1010A00017460FF099FD031E0BDB0022294601A80D
:1010B0000FF0B0FD01A928460FF003FD01A80FF0C5
:1010C00066FC114928460FF03EFD064660B100233C
:1010D000A3614FF4FA43236101208423E361207567
:1010E00084F8207005B0F0BD084928460FF02BFDAC
:1010F0000028F7D08423C4E906662361267584F8A6
:1011000020700120EEE700BF2A7E0100377E01003B
:1011100001294FF0000303D002290CD01846704774
:1011200083614FF4FA4303618423C361017580F83E
:101130002020012070478421C0E906330161037536
:10114000F5E7000007B5002300931A461946044846
:101150000EF044FF034803B05DF804EB0EF08ABDC7
:10116000ED020020EC02002038B50023836083806C
:101170008371036804460D46002B4CD0344A126834
:10118000002A48D0002908BF1D462B7C03F00F031E
:10119000062B15D12F4A304829460DF05FFC08B1C7
:1011A000436923712D4A2C4829460DF057FC00282D
:1011B00049D0037C03F00F03022B2DD0052B2ED03A
:1011C000274A216824480DF049FC054608BB2549FB
:1011D00025480EF04BFF0A22617923480EF0C8FF24
:1011E000224921480EF042FF0A2221791E480EF0C2
:1011F000BFFF1D480EF04AFF2B46194A21681648CA
:101200000DF074FC164A216813480DF027FC0546C2
:1012100008B11435A56038BD43696371D0E7C36870
:10122000002BCDD01A7C02F00F02022AC8D15A69D5
:101230006271DB68002BC3D01A7C02F00F02022A15
:10124000BED15B69E9E7286811F0F9FD6071B7E785
:1012500038040020B09B0100780700208C7E01003C
:10126000F27E0100F57E010070030020C18B0100B9
:1012700010B5044601601146FFF776FF204610BD09
:1012800070B5044686B028B3037C03F00F03062B29
:1012900020D106A8002140F8184DFFF765FF029BFA
:1012A0000D4A0E4800261E6021460DF0D7FB88B17E
:1012B000037C03F00F03052B0CD1C56855B1214603
:1012C00003A80395FFF750FF059B1E600FF020FD5C
:1012D0006D68F3E706B070BD807E010078070020DE
:1012E00038B583680446BBB1124B1B68A3B10068D4
:1012F000FFF7C6FFA36800251D602379032B0CD8D8
:10130000012B94BF0221294660790FF099FEA36852
:101310005A7865F303025A7038BD402B03D0422B34
:10132000FAD1294600E002216079BDE838400FF08B
:1013300087BE00BF3804002041790C4A002352F8D0
:101340002300884203D10A4A52F82300704752F81A
:10135000230028B942F82310054A42F823007047B9
:101360000133052BEBD10020704700BF04030020A0
:101370001803002010B50A4A4079002352F8234090
:10138000844203D1074A42F8231010BD52F823408B
:1013900014B952F82320F5E70133052BEED1F4E719
:1013A0000403002018030020F0B52DED028B9DB042
:1013B0000446FFF7C1FF05460FF054FC0023014629
:1013C00043F69822284609F025F8002800F0E98025
:1013D00006231622617907A80EF048FA372107A8DC
:1013E0000EF054FA0022114607A80EF069FB002106
:1013F00008EE900A07A80EF0FBFB6C4908EE100AF5
:101400006B480EF033FE0A22617969480EF0B0FE97
:10141000684967480EF02AFE18EE900A11F04EF95E
:10142000022502460B46009561480EF05DFF6249B9
:101430005F480EF01BFE18EE100A11F03FF9009500
:101440000B4602465A480EF04FFF5C4958480EF0D2
:101450000DFE57480EF01AFE594A216859480DF002
:10146000FDFA594A2168074656480DF0F7FAF4EE9E
:10147000688AF1EE10FA064610D60CAD18EE901AF6
:10148000284603F0E8F80023CDE90133009395E8FE
:101490000C004FF0FF31384608F0D6FFB4EE488A12
:1014A000F1EE10FA10D60CAD18EE101A284603F023
:1014B000D2F80023CDE90133009395E80C004FF0FA
:1014C000FF31304608F0C0FF404A21683D480DF02A
:1014D000C5FA054600285ED0037C03F00F03042BF9
:1014E00059D1F5EE408AF1EE10FA54D0B5EE408AAB
:1014F000F1EE10FA4FD0F4EE688AF1EE10FA4AD10C
:10150000B4EE488AF1EE10FA45D100213C220DA834
:101510000C9111F01AFF696940220CA812F0E9FE43
:101520002F210CA812F07CFE28B96B690322402100
:101530000CA808F0D7FE26490CA812F062FE04A8F9
:1015400018EE901A08F05BFE22480DF0D9FD40B16C
:10155000214B93F9003023B904AA0CA91D480EF0C1
:1015600017F80CA812F097FE1CAB1844482300F89B
:10157000413C18EE101A04A808F041FE15480DF081
:10158000BFFD40B1144B93F9003023B904AA0CA954
:1015900010480DF0FDFF0FF065FB01462046FFF7F8
:1015A000E9FE1DB0BDEC028BF0BD00BFEE7E010078
:1015B00070030020FA7E01000A7F0100117F010004
:1015C000137F010078070020187F01001C7F0100B5
:1015D000B09B0100E8030020B80300202DE9F04F84
:1015E000054600688BB00F46924640B1A86830B1FE
:1015F0000378FF2903F0100335D11BB901200BB08C
:10160000BDE8F08F032AF9D04778A149A1480EF030
:101610002DFD0A2269799F480EF0AAFD9E499D483A
:101620000EF024FDAB689B4859780A2201F00F01A7
:101630000EF09EFD3F09994996480EF017FD0A22CB
:10164000394694480EF094FD92480EF01FFDAB68A9
:101650005A7802F00F02BA4207D11A786FF30412D7
:101660001A700020CBE7002BFBD100220DF11808E7
:101670001146404602F0E2FFAB685B7803F00F03CF
:10168000BB4223D0BAF1030F20D0854981480EF028
:10169000EDFC0A2269797F480EF06AFD7E497D489B
:1016A0000EF0E4FCAB687B4859780A2201F00F0188
:1016B0000EF05EFD794977480EF0D8FC0A223946D3
:1016C00074480EF055FD73480EF0E0FC29680C2FAD
:1016D00000F2B780DFE807F0073A9CA9AB9C7B9C3F
:1016E000ADAF8CB1B300AB685B7803F00F03023B86
:1016F000082B24D8DFE803F0052323A5230F232399
:101700001900684A68480DF0A9F9AB681C780646CC
:1017100004F001042DE0654A63480DF09FF9AB68C1
:101720001C780646C4F3400423E0614A5E480DF08D
:1017300095F9AB681C780646C4F3800419E05D4A4D
:1017400059480DF08BF90646002412E05A4A5648D3
:101750000DF084F9AA681378D94303F0010461F30A
:1017600000031370064620B90122414608A803F081
:101770004AFB524A29684C480DF070F9504A2968D2
:10178000814649480DF06AF94E4A29688346464821
:101790000DF064F90590BBF1000F07D1B9F1000F0E
:1017A00004D14A46414608A803F02DFB002E4BD138
:1017B000404603F0C8F8002846D1AB685A7867F372
:1017C00003025A701A7866F304121A7016E73E4A3A
:1017D00035480DF043F9A9680B7883F00202C2F393
:1017E0004002C3F34004064662F341030B70C0E7B6
:1017F000364A2D480DF032F9A9680B7883F00402BF
:10180000C2F38002C3F38004064662F38203EDE76D
:10181000284A25480DF022F90646002894D10222D4
:10182000414608A803F0EFFA8EE7294A6AE7294AF9
:1018300068E7294A70E7294A6EE7294A76E7294A84
:1018400074E70024264694E7AB68BAF1030F5A7890
:1018500012D067F303025A701A786FF304121A70E9
:10186000059BCDF80090CDE901B3214698E80C0026
:10187000304608F0E9FDC1E602F00F01B9423FF43D
:10188000BDAE67F307125A701A7842F010029CE757
:10189000847E010070030020247F01008E7E010001
:1018A0008C7E0100927E010078070020917E01006D
:1018B000987E01009F7E0100A47E0100DA7E010077
:1018C0001C7F0100DF7E0100A97E0100AF7E0100C8
:1018D000B57E0100BA7E0100C07E0100C67E010017
:1018E000CD7E0100D37E01002DE9F043614A95B021
:1018F00006468846016860480DF0B0F85F4A3168D6
:1019000081465D480DF0AAF85D4A316807465A489D
:101910000DF0A4F8B9F1000F02D10FB900287CD066
:10192000584A316854480DF099F8574A31680546CD
:1019300051480DF093F85549044655480EF096FB72
:101940000A22717952480EF013FC524950480EF0A9
:101950008DFB0A2241464E480EF0F1FB4C480EF03A
:1019600095FB5FB33B7C03F00F03042B26D1402291
:10197000796904A812F0BDFC47480DF0C1FBE8B13D
:10198000464B93F90030CBB92F2104A812F048FC44
:1019900028B97B690322402104A808F0A3FCB8F110
:1019A000000F43D025B12B7C03F00F03042B37D05D
:1019B0003B4A012304A938480DF0FFFDB9F1000F9F
:1019C0002BD099F8103003F00F03042B25D1354BA1
:1019D000D9F814101A6804A800F0EEFE04A800F06C
:1019E00047FEB8B1B8F1000F35D025B12B7C03F01C
:1019F0000F03042B25D002AC01220021204602F067
:101A00001DFE01220023CDE9002304A894E806006E
:101A100001F03EFB04A800F06FFC15B0BDE8F083B8
:101A20006A691378002BC9D00123C3E724B1237C52
:101A300003F00F03042B02D001231B4ABAE76269AB
:101A4000EFE769690B78002BE4D000231A4604A85D
:101A500002F0DEF9DEE724B1237C03F00F03042B50
:101A600002D002AC0222C8E761690B78002BD1D00A
:101A70004346EBE7DA7E0100780700201C7F010077
:101A8000DF7E0100A47E01009F7E0100E77E010051
:101A9000700300200F7F0100E8030020B80300203E
:101AA00048950100DC0300205995010070B59AB0FB
:101AB000054604AC84E806003A483B490EF0D6FAE5
:101AC0000A22697937480EF053FB384935480EF041
:101AD000CDFA204603F096FB2968354A35480CF0CC
:101AE000BDFF0023CDE90133009394E80C004FF0D3
:101AF000FF3108F0A9FC29682F4A2E480CF0AEFFF0
:101B000029682E4A06462B480CF0A8FF054658B314
:101B1000037C03F00F03042B26D1416940220AA85D
:101B200012F0E7FB2F210AA812F07AFB28B96B69A3
:101B3000032240210AA808F0D5FB002300931022BD
:101B40004FF4007306A9204603F04AFA1C480DF032
:101B5000D7FA48B11B4B93F900302BB9012306AAE1
:101B60000AA917480DF029FDD6B1337C03F00F0305
:101B7000042B15D1144B71691A680AA800F01CFED9
:101B80000AA800F075FD40B101220023CDE9002331
:101B90000AA894E8060001F07BFA0AA800F0ACFB62
:101BA0001AB070BD70030020EE7E01000F7F0100AF
:101BB000807E010078070020DA7E01001C7F010092
:101BC000E8030020B8030020DC03002010B50378F0
:101BD0008B42044604D14378402B01D1408810BD8C
:101BE00040232170637008460FF034F980B26080A2
:101BF000F5E7000083682DE9F04104460D46002B0F
:101C000000F07B810379072B02D1042940F0758114
:101C1000A44F3B780133DBB22A46FF2120463B70BC
:101C2000FFF7DCFC637922790E3B072BC2F34008F7
:101C300001D9072A32D19C4A21689C480CF00EFF3A
:101C4000064658B3037C03F00F03052B26D12379F6
:101C5000A27961799648FFF7B9FF002280463146A4
:101C600092480CF0F1FE436998451FDA0026032DD7
:101C700060D0A3685A7802F00F02013A0B2A59D8B3
:101C8000DFE812F01F00ED0042006A00ED00720074
:101C9000ED009100A200AA00D300E50060790FF0EA
:101CA00009FAA8EB00035E425E41E0E731460122FB
:101CB0007E480CF0C9FE4669B045CCBF002601261F
:101CC000D5E7B3F802800EF0CDFF4FF6FF7381B277
:101CD0004FF47A72404608F09DFB58B3754A21686C
:101CE00072480CF0BBFE28B12A4603212046FFF7BC
:101CF00075FC1FE0704A21686C480CF0AFFE0028AC
:101D0000F2D12A460D21F1E7B3F802800EF0AAFFC6
:101D10004FF6FF734FF4967281B2404608F07AFB9B
:101D200040B12A4604212046FFF758FC0EF09AFFE6
:101D3000A3685880A2681378C3F3C001B14200F0D1
:101D4000438113F0E00F00F09C80C3F3421101398E
:101D500061F347131370CCE0B3F802800EF082FFFA
:101D60004FF6FF739622D7E7B3F802800EF07AFFA2
:101D70004FF6FF7381B24FF47A72404608F04AFB87
:101D80000028D7D04D4A216848480CF067FE10B1B2
:101D90002A460821AAE74A4A216844480CF05EFE18
:101DA0000028F5D1ADE7B3F802800EF05BFF4FF6E7
:101DB000FF734FF4967281B2404608F02BFB002867
:101DC000B8D02A460921AEE7B3F802800EF04AFFE8
:101DD0004FF6FF739622EEE7B3F802800EF042FF53
:101DE0004FF6FF7381B24FF47A72404608F012FB4F
:101DF00000289FD0334A21682C480CF02FFE10B1E8
:101E00002A460B2172E7304A216828480CF026FE4A
:101E10000028F5D12D4A216824480CF01FFE002827
:101E20007FF46FAF2A46062160E7B3F802800EF018
:101E300019FF4FF6FF734FF4967281B2404608F0D7
:101E4000E9FA00283FF476AF2A460C216BE7B3F895
:101E500002800EF007FF4FF6FF739622EDE7B3F80E
:101E600002800EF0FFFE4FF6FF7381B24FF4167240
:101E7000404608F0CFFA00283FF45CAF2A46002124
:101E800034E70EF0EFFEA36858805B7803F00F0391
:101E9000002E4FD0072B27D8DFE803F046261A265E
:101EA000261A264900030020E37E0100780700205F
:101EB0002C030020B57E0100BA7E0100C07E010027
:101EC000C67E0100CD7E0100D37E0100AF7E010001
:101ED0003E4A21683E480CF0C1FD80B12A460621E9
:101EE0002046FFF77BFB20B1A3681A7866F3C30294
:101EF0001A703B78013BDBB23B70BDE8F081354A9C
:101F0000216833480CF0AAFD0028E7D1324A216845
:101F10002F480CF0A3FD0028E0D1304A21682C485E
:101F20000CF09CFD0028D9D12A460121D8E72A4689
:101F30000A21D5E7013B0C2BD6D801A252F823F099
:101F4000751F0000E91E00007B1F00007B1F0000C2
:101F5000E91E0000811F0000E91E0000C31F0000F1
:101F6000C31F0000C31F0000C31F0000C31F0000E9
:101F70007B1F00002A460221B2E72A460521AFE76F
:101F8000124A216812480CF069FD10B12A46072157
:101F9000A6E7104A21680E480CF060FD0028F5D134
:101FA0000D4A21680A480CF059FD0028EED121683D
:101FB0000A4A07480CF052FD01460028E6D12A469D
:101FC0008EE72A4600218BE70221C1E6A97E0100A7
:101FD00078070020C07E0100C67E0100917E0100CE
:101FE0002DE9F047032986B007466DD00168624AA3
:101FF00062480CF033FD3B79BA797979064660483E
:10200000FFF7E4FD05B2002E6CD0337C03F00F0324
:10201000052B67D1314659480CF00CFD032856D9E1
:102020000022314655480CF00FFD01224469534807
:1020300031460CF009FD0222D0F814A04F48314679
:102040000CF002FD43694D484FF00A080322314667
:1020500008FB03F90CF0F8FC436908FB03F8214680
:10206000CDF800804B46524628460EF086FC0446CA
:10207000314642480CF0DEFC052830D104223146BE
:102080003E480CF0E1FCB0F914A03C484445C4BF04
:10209000444640F2FF3531464C45BCBF4C46002516
:1020A0000CF0C8FC022826D10022314633480CF03F
:1020B000CBFC4369AB424FDC012231462F480CF088
:1020C000C3FC4369AB4254DB06B0BDE8F08705EBC7
:1020D000850464004FF000094FF42058C8E74FF022
:1020E000010AD2E705EB850464004FF000094FF4C4
:1020F00020584FF0010ABB68B3F902002A1A002ADF
:10210000B8BF5242524507DC1A785109052907D851
:10211000013161F3471202E01A786FF347121A7027
:102120001B789F2B03D94C4501D04445CCD1A84204
:10213000CAD00022114604AE02A802F07FFA22465D
:1021400002A9304602F0EBFD96E806003846FFF79C
:10215000ADFCBB685D80B7E70024BB68B3F9023013
:10216000A342B1D021463846FFF7BEFBBB685C8076
:10217000AAE70124F1E700BFE37E01007807002011
:102180002C030020836810B5044643B34B1E032B79
:1021900015D8DFE803F01E0202160379402B0BD09E
:1021A00005D8032B0BD82046FFF724FD07E0422B70
:1021B00002D004D3803BF4E72046FFF711FF002054
:1021C0000FE00379072BFAD10421FFF709FF04215F
:1021D000E9E70379042BF2D1FFF7E6F8EFE74FF0D8
:1021E000FF3010BD002303807047000013B50024AA
:1021F000234600942246214603480DF0EFFE034B90
:102200001C805C8002B010BDF80200202C0300206E
:1022100010B5044670B3204912F00FF858B31F49A7
:10222000204612F00AF840B31D49204612F005F886
:1022300028B31C49204612F000F810B31A49204672
:1022400011F0FBFFF8B11949204611F0F6FFE0B19B
:102250001749204611F0F1FFC8B11649204611F088
:10226000ECFFB0B11449204611F0E7FF002814BF7D
:102270000020152010BD0120FCE70220FAE7052010
:10228000F8E70620F6E71320F4E71420F2E70E2023
:10229000F0E70F20EEE700BF347F01003D7F010033
:1022A000587F0100617F0100D67F0100DF7F0100C0
:1022B000A97F0100B27F0100E87F010070B50546EB
:1022C00080B1047864B1084E012404EB84013144E8
:1022D000284611F0B2FF18B101340E2CF5D10024BC
:1022E000204670BD0446FBE70C800100806910B1F8
:1022F00003681B691847704710B50446806910B120
:1023000003685B689847204610BD000008B50322AB
:10231000416804480CF098FB08B1007D08BDFF201F
:10232000FCE700BF7807002010B503220C46416887
:1023300009480CF089FB70B1037C13F00D0F0AD132
:10234000416921F07F41022221F0FF0162F3030382
:1023500021430374416110BD7807002010B50322AA
:102360000C46416808480CF06FFB60B1037C03F039
:102370000F03022B01BF24F07F41406921F0FF01D0
:10238000084018BF002010BD7807002010B50322B8
:102390000C46416809480CF057FB70B1037C13F000
:1023A0000D0F0AD1022262F30303037424F07F416C
:1023B000436921F0FF011943416110BD78070020F6
:1023C00010B50446806968B103685B69984718B125
:1023D000A06903681B699847A0690368DB68984790
:1023E00008B9012010BD2046FFF790FF20B14FF43F
:1023F00080712046FFF7CAFFE368002BF1D04FF44D
:1024000000712046FFF7C2FFEBE7000010B5032282
:102410000C46416808480CF017FB58B1037C13F0D8
:102420000D0F07D1E143436941F07F4141F0FF01C6
:102430001940416110BD00BF7807002038B50C4637
:102440008168054609B9002038BD0B7C03F00F03F5
:10245000022B03D1002CF6D14869F5E7052BF2D108
:1024600005480CF0E7FA8442EDDAE2B2A9680248C6
:102470000CF0EAFA4069E7E77807002038B50D4626
:102480008168044621B9DFED1A7A17EE900A38BD4B
:102490000B7C03F00F03052B15D116480CF0CAFA7C
:1024A000854210DAEAB2A16812480CF0CDFA002891
:1024B000E9D0037C03F00F03022B0FD1D0ED057A96
:1024C000F8EEE77AE1E7002DDDD1A268137C03F096
:1024D0000F03022B07D1D2ED057AF1E7032BD2D1FE
:1024E000D0ED057AD1E7032BCDD1D2ED057ACCE73B
:1024F000000000007807002008B5816869B10B7CF6
:1025000003F00F03022B06D0052B06D104480CF074
:1025100091FA00B208BD0120FCE70020FAE700BFF5
:102520007807002008B5C16809B9002008BD087CFB
:1025300000F00F039A1E012A00D90BB90009F5E734
:10254000052BF2D1002203480CF07EFA0028ECD0D3
:10255000007CF3E778070020C26810B5BAB1137C9D
:1025600003F00F039C1E012C00D983B95161C3688D
:102570001A7C022161F303021A74C268137C03F00F
:10258000F001602902BF0A2161F30713137410BD23
:10259000C26810B5BAB1137C03F00F039C1E012C66
:1025A00000D983B95161C3681A7C032161F3030226
:1025B0001A74C268137C03F0F001602902BF07217E
:1025C00061F30713137410BDC36853B11A7C02F092
:1025D0000F02901E012800D91AB91A7C61F3071264
:1025E0001A74704708B5016909B9002008BD0B7C51
:1025F00003F00F03022B01D14869F7E7052BF4D153
:10260000002203480CF020FA0028EED04069EDE7E4
:10261000780700202DE9F041036904460F46A3B96D
:1026200041681248114E0CF005FA0546042D0CDCE9
:102630003046D4F804800CF043FA4146024620614B
:1026400030460CF01AFA0135F0E7226962B1137CCA
:1026500013F00F0106D1022161F303031374236900
:102660005F6101E00229FAD0BDE8F081780700201F
:10267000406828B1007C00F00F00431F58425841C9
:1026800070470000F8B50446FFF7F2FF48B36168F1
:102690003248324F0CF0CEF90546032D666809DC4E
:1026A00038460CF00DFA3146024638460CF0E5F992
:1026B0000135F2E7F06808B14368A360A3680BB185
:1026C0005B68E360E3681BB15B680BB15B68236127
:1026D00002F052FCC0B20C2820752CD002D803287E
:1026E0000ED0F8BD102830D01228FAD10C200EF0F0
:1026F0004FFB1B4B44600360054606F027FD18E0C6
:1027000010200EF045FB174B036005464460002186
:102710002046FFF793FE03B2002BB6BF40422B8149
:1027200028816868FFF7E8FE0F4B2B600023688163
:10273000AB81A561D5E714200EF02AFB0B4B44605A
:102740000360054606F056F9F3E70EF021FB084B4F
:1027500044600360054606F03BFFEAE77807002087
:10276000DC950100B47D010038960100F894010069
:10277000D896010010B500230446C0E9002183610A
:102780000377C362FFF77EFF204610BD70B5066871
:1027900005462F21304611F0CDFD044630B100230F
:1027A00000F8013BBDE87040FFF788BD3046FFF7F9
:1027B00085FD00B12C6070BD2DE9F043054689B060
:1027C000002400F11C082A601646CDF804808461BC
:1027D0000477C4620F462346002939D0002A37D037
:1027E0002F21384611F01CFD814650B3234602AA22
:1027F000F85C19B238B12F2805D0142B02D0D05470
:102800000133F5E7194608AB1944002301F8183CD9
:10281000104831460CF022F90F22686009F10101DD
:10282000404611F066FD01A8FFF7B0FF019BE8628A
:1028300003B92B772846FFF725FF284609B0BDE8E6
:10284000F0833A46314603480CF008F96860F1E736
:102850006B60EFE77807002008B583693BB9007D1E
:10286000052809D014280CBF0020FF2008BD1A68D5
:102870001846926B9047F3E75020F7E708B505221A
:10288000416805480CF0E0F820B1037C13F0F0003B
:1028900018BF180908BD00BF780700202DE9F743CD
:1028A0006D4685E80600416881461F4619B900203B
:1028B00003B0BDE8F0833448DFF8CC800CF0BAF800
:1028C0000446052CD9F8046009DC40460CF0F8F801
:1028D0003146024640460CF0D0F80134F1E70522BB
:1028E000314629480CF0B0F804460028DFD02846CD
:1028F00002F0D8F90F28DAD8284602F06DF800283F
:1029000007DD237C13F00D0F10D003F00F03072B0E
:102910000CD0237C1D491E486FF3071323740DF060
:10292000A5FB1B480DF0B2FB0120C1E70EF09AF9A0
:102930000646284602F050F8002F237C0CBF0222E6
:10294000072262F30303304460612374284602F0D7
:10295000A9F9237C0F4960F3071323740C480DF089
:1029600085FB284602F038F80A22014608480DF097
:10297000C4FB094906480DF079FB0A226169044845
:102980000DF0BBFBCDE700BF780700207180010090
:10299000700300207B80010086800100F0B587B0C5
:1029A0006F4687E80600054697E8030002AC84E816
:1029B000050038461E4602F075F901380C2838D853
:1029C000DFE800F0424B959E8C0739373754627E22
:1029D00070004EBB0722214604A802F014FA4949B0
:1029E00049480DF043FB204602F05CF90A220146FB
:1029F00045480DF0BDFB454943480DF037FB2046E7
:102A000001F0EAFF0A2201463F480DF076FB3E48FE
:102A10000DF03CFB9DF8303094E806002846FFF7A7
:102A20003DFF012007B0F0BD2846FFF727FF002833
:102A3000D0D10020F6E70EB10622CCE72846FFF7FA
:102A40001DFF0028F8D1F4E70EB90222C3E728469B
:102A5000FFF714FF0028F8D1EBE70EB10122BAE727
:102A60002846FFF70BFF0028F8D1E2E74FF480314A
:102A70002846FFF773FC08B10B22ACE72846FFF7A6
:102A8000FDFE0028F8D1D4E74FF480312846FFF747
:102A900065FC08B90A229EE72846FFF7EFFE0028EA
:102AA000F8D1C6E74FF400312846FFF757FC08B9C4
:102AB0000C2290E72846FFF7E1FE0028F8D1B8E79E
:102AC0004FF400312846FFF749FC08B10D2282E798
:102AD0002846FFF7D3FE0028F8D1AAE70EB103225B
:102AE00079E72846FFF7CAFE0028F8D1A1E70EB91A
:102AF000052270E72846FFF7C1FE0028F8D198E7C5
:102B0000042268E7B980010070030020CD80010035
:102B100018B1034903480DF0A9BA0349FAE700BF09
:102B2000217F010070030020267F01002DE9F04382
:102B30009FB04FF0000802AC84E80600269FCDF855
:102B400024801022414606460AA81D4610F0FDFBCF
:102B5000A449A5488DF82080CDE906880DF08FFAAC
:102B60003946A1480DF08BFA204602F04BFBEA05EE
:102B70001AD5204602F096F8172800F2CE800123DD
:102B800003FA00F0994B18420AD1994B0340002BED
:102B900040F0C78010F0240F00F0BF80954900E09E
:102BA000954906A811F053FB94480CF0A9FA0028A7
:102BB00000F0AB80924B93F900209846002A40F039
:102BC000A480002F44D13B46032240210EA807F0E9
:102BD00089FB73683F2219680EA811F064FBAB05EE
:102BE00040F1AE80204602F05DF8022800F0A88097
:102BF000204602F057F8052800F0A280204602F097
:102C000053F8012840F090804FF001094FF4007311
:102C1000142209A9CDF80090204602F0E1F94B46B4
:102C200009AA0EA975480CF0C8FC76496E480DF04B
:102C30001DFA0EA96C480DF022FA73496A480DF08E
:102C400015FA09A968480DF01AFA67480DF01EFA3E
:102C5000204601F087FE05F4005908B1A90503D408
:102C6000B9F1000F00F09D800023032240210EA83F
:102C700007F038FB73683F2219680EA811F013FBA8
:102C800047B162490EA811F0BCFA3F2239460EA89E
:102C900011F009FB5D490EA811F0B3FA3F22B9F11A
:102CA000000F67D05A490EA811F0FDFA204601F036
:102CB000FBFF043801285FD81722214604A802F040
:102CC000A2F8002300934FF44073142209A9204670
:102CD00002F086F94B4944480DF0C8F90EA9424864
:102CE0000DF0CDF9484940480DF0C0F909A93E481A
:102CF0000DF0C5F93C480DF0C9F940480CF000FA58
:102D000018B198F90030002B40D030462946FFF723
:102D10003DFB00201FB0BDE8F0833E4932480DF076
:102D2000A5F925F480753FE7204601F0BDFF022894
:102D30003FF46AAF204601F0B7FF08283FF464AFC4
:102D4000E80585D59DF81830002B81D0012306AA0F
:102D50000EA92A480CF031FC2A4923480DF086F9C7
:102D60000EA921480DF08BF927491F480DF07EF977
:102D700006A967E7284996E70023B9F1000F0093F9
:102D80000CBF4FF400734FF440739EE70EA901236C
:102D900009AA1A480CF011FC4FF400713046FFF7F5
:102DA00035FBEA0540F18680204601F07BFF0138C3
:102DB000142837D8DFE810F0DB0036003600360084
:102DC0003600DB00360036003600360036003600AE
:102DD0003600DF00D9003600360036003200D5005C
:102DE000D70000BF8C8001007003002042C0380073
:102DF000010080003D7F0100347F0100E8030020D6
:102E0000B8030020B38001008E7E0100C18B010059
:102E10002080010099800100168001005C4906A80D
:102E200011F015FA0023032240210EA807F05AFAE8
:102E300073683F2219680EA811F035FA47B1554959
:102E40000EA811F0DEF93F2239460EA811F02BFA38
:102E500050490EA811F0D5F93F224F490EA811F0A4
:102E600022FA4E494E480DF001F90EA94C480DF0DA
:102E700006F94C494A480DF0F9F806A948480DF002
:102E8000FEF847480DF002F947480CF039F90028E0
:102E90003FF43BAF98F90030002B7FF436AF0EA91A
:102EA000012306AA40480CF088FB4FF4807130469D
:102EB000FFF7ACFA6B0552D54FF480313046FFF77F
:102EC0004DFA002859D0394906A811F0C0F900235D
:102ED000032240210EA807F005FA73683F22196803
:102EE0000EA811F0E0F947B12A490EA811F089F9AE
:102EF0003F2239460EA811F0D6F926490EA811F046
:102F000080F93F222A490EA811F0CDF9234924481F
:102F10000DF0ACF80EA922480DF0B1F82149204877
:102F20000DF0A4F806A91E480DF0A9F81C480DF0F4
:102F3000ADF81D480CF0E4F800283FF4E6AE98F92F
:102F40000030002B7FF4E1AE0EA9012306AA16483B
:102F50000CF033FB4FF480613046FFF757FA012045
:102F6000D8E614495BE7144959E7144957E7337D1C
:102F7000052B7FF457AF124951E74FF4003130462B
:102F8000FFF7ECF908B10F499EE70F499CE700BF36
:102F9000D67F0100C18B010011800100B3800100C8
:102FA000700300208E7E0100E80300208E7F010068
:102FB00039800100DF7F0100E87F0100B27F01005E
:102FC000A97F0100A07F0100857F0100F0B5CB073C
:102FD0000C4644BF21F4805424F0010414F48057BB
:102FE00085B005460CD004F4E0612846FFF7CEF921
:102FF000144915480DF03AF84FF0FF3005B0F0BD18
:1030000007F0F6F89528EED902F090FF0028EAD0F4
:1030100002AE3A463946304601F010FB4FF440729A
:103020002946304601F0FFFE4FF4E0612846FFF7E5
:1030300095F9009744EA000396E806002846FFF752
:1030400075FDDBE7528001007003002010B54FF4DE
:1030500040710446FFF782F9014670B1074B93F9BE
:103060000030062B09D12046FFF7B0FF20464FF471
:103070004071BDE81040FFF7C9B910BDE003002062
:1030800083691BB11A681846926B1047007D704720
:103090002DE9F04F93B00AAE09939DF87030039379
:1030A0009DF874300493054686E8060007F0A0F802
:1030B000B0F5966F04460EDAAF49B0480CF0D6FF73
:1030C0000A222146AD480DF03AF8AC480CF0DEFF7C
:1030D0004FF0FF39A9E30DF0C5FD0790304601F030
:1030E00099FE0290074602F021FF099B06901BB152
:1030F0001A78002A40F01B862B7F13B105F11C03C0
:103100000993002F40F02B86099B002B40F011867D
:10311000EB6A0293002B00F02286304601F07AFE23
:10312000002840F01C869DF80820314610A801F0C8
:1031300073FE00F014BE6B68002BC9D0029B042BF9
:1031400007D1049B96E806002846FFF7A7FB8146B7
:103150006BE396E803000CAB83E80300304601F014
:10316000A1FD092800F22282DFE810F00A00200207
:10317000200220026D01200220022002AF01AF01D7
:1031800000220DF138091146484601F057FA304641
:1031900001F0E8FB0746002800F04F81029B0C2B52
:1031A0001AD8DFE813F00D001900690019001900A2
:1031B0001900190019001900190017010301330142
:1031C000DDF82480B8F1000F0AD06D496D480CF08D
:1031D0004DFF6C480CF05AFF0024A2462746F6E04B
:1031E000284601F01DF80028D4BF002101210A2241
:1031F000044664480CF0A3FF634962480CF03FFFAB
:10320000304601F0E9FB0A2201465E480CF075FFEA
:103210005C480CF03BFF002C304640F37F8501F00A
:10322000DBFB70BB0222314610A801F0ECFD40F23E
:1032300001144FF0010806E00122314610A801F008
:10324000E2FD40F201144FF400722946484602F0B4
:103250003DFB484601F028FD042814D1304601F01A
:1032600023FD022814D1304601F01EFD0EA90246AE
:1032700010A801F01DFD0BE0002427464FF0FF3899
:10328000E1E74446D5E7484601F00EFD0528E5D0C4
:103290002B7D072B08D1304601F06AFB20B10222BA
:1032A0000EA910A801F004FD2846FFF7E9FE00B2C0
:1032B00000900DF1380A0DF1280910A899E80C00CA
:1032C000514602F01BF8504601F09CFF3FB14846C2
:1032D00001F0EAFC022859D1504602F023FB9AE89B
:1032E000030089E8030044F490544FF0000A4FF0C3
:1032F000FF392B7D072B40F05082039B73B3AB68E3
:103300001B7C03F00F03052B40F05981069B002B1B
:1033100000F05281284600F083FF049B00930028B0
:10332000099BA9680AAA2846D4BF4FF000094FF0AC
:10333000010900F0EFFE029B012B4FFA89F840F0E3
:103340003E810AA801F00EFB039038B1049B009364
:103350000CAA4B4606CA2846FFF720FB0AA801F034
:10336000A1FC0338042800F25081DFE810F02A01A4
:103370004E01ED0172015101D88001008C03002043
:103380001881010070030020247F0100484601F0ED
:103390008BFC0128A0D0484601F086FC0A289BD06F
:1033A000484601F081FC0B2899D195E729464FF456
:1033B0000072484602F08AFA304601F02BFAC1B298
:1033C000484601F0CCF998B9BA4600273C464FF080
:1033D000FF388CE729464FF40072484602F076FA2F
:1033E000304601F010FA0146484601F09DF9EAE73F
:1033F00099E80300022286E803000027314610A85E
:1034000001F00AFD4FF49054BA46E0E74FF4007221
:103410002946484602F05AFA304601F0D9F90146E9
:10342000484601F0AEF999E803004FF0000A86E83B
:1034300003004FF490545746C9E7824604464FF0C4
:10344000FF39C84655E7029B092B20D0284600F0DB
:10345000E7FE00280DDD0222314610A8012701F009
:10346000D2FC40F201144FF0FF394FF0000AB84689
:103470003FE70122314610A84FF0000A01F0C3FCDB
:1034800040F201144FF0FF390127D04631E74FF4E5
:1034900080312846FEF762FF07464FF48031284608
:1034A0005FB1FEF7B3FF40F201444FF001094FF066
:1034B000000A57464FF0FF381BE7FEF767FF40F260
:1034C00001444FF00109BA46F3E796E803000DF115
:1034D000380888E80300304601F044FAE0B90524D2
:1034E000304601F0DFFB4FF40072092829463046D0
:1034F00008BF644202F0EAF90022314610A801F048
:1035000082FC029B0B2B49D8DFE803F021480D48D1
:103510004848484848482343304601F033FA0446B7
:103520000028DCD0DCE700272846FFF795F9214684
:103530000246304601F070F9044690BB98E803005B
:1035400086E803004FF0010A4FF0FF39B2E7012788
:10355000EAE72146304601F0BCF950B1022231467B
:1035600010A84FF0000A01F057FC4FF49054574652
:10357000EAE798E8030086E80300AE49AE480CF09D
:1035800075FDAD480CF082FD00244FF0010A27467E
:10359000DAE72146304601F0C2F9DEE70024A24610
:1035A000F5E74FF490544FF0000ACDE700244FF0B8
:1035B000FF39A246274644E7069B0393CEE6002345
:1035C000FBE72846FEF7A2FE0528804602D04FF012
:1035D00003092AE199499A480CF048FD0A2241461C
:1035E00097480CF0ACFD96480CF050FD4FF400727B
:1035F00029460AA802F06AF901220AA910A801F0D6
:1036000002FC44F4807444F001044FF0000B47E0E6
:103610002846FEF77BFE062880460DD1894988485A
:103620000CF024FD0A22414685480CF088FD8448B0
:103630000CF02CFD0222E0E7834981480CF016FDD6
:103640000A2241467E480CF07AFD7D480CF01EFDB2
:10365000BDE74FF480312846FEF780FE002871D187
:10366000B8F1FF3F08D1284600F0DAFD0028D4BFAA
:103670004FF000084FF00108B8F1000F5DD14FF492
:10368000007229460AA802F021F901220AA910A80D
:1036900001F0B9FB44F4807444F001044FF0060BD0
:1036A0000AA801F055F900286BD10AA844F00104DA
:1036B00001F058F9002867D044F40074039B13B15B
:1036C00024F40074A4B2224629460AA801F000FCA2
:1036D0004FF00109BAF1000F40F07183A86900288A
:1036E00040F0E4814FF400312846FEF737FE002811
:1036F00000F0E581554950480CF0B8FC4E480CF0FC
:10370000C5FC630500F1FD8251494D480CF0AEFC4B
:103710000A2249464A480CF012FD4E4948480CF02E
:10372000A5FC0DF09FFA079B0A22C11A44480CF031
:1037300012FD43480CF0AAFC77E0474940480CF0E2
:1037400095FC44E74549F9E7B8F1FF3F08D1284621
:1037500000F066FD0028D4BF4FF000084FF00108CC
:10376000B8F1000F0BD002220AA910A844F480740B
:1037700001F049FB44F001044FF0050B90E7384994
:10378000DCE744F4807490E74FF4007229460AA8FD
:1037900001F049FB00288FD190E7B8F1FF3F08D135
:1037A000284600F03DFD0028D4BF4FF000084FF040
:1037B0000108B8F1000F2B49214818BF01270CF070
:1037C00055FC0A2241461E480CF0B9FC26491C480B
:1037D0000CF04CFC0A22394619480CF0B0FC184891
:1037E0000CF054FC0998002844D0FEF711FD089015
:1037F0002846FEF78BFD0FFA80FB089BBBF1000FFC
:1038000001D10FFA88FB002B5BD09B4530D01749C4
:103810000B480CF02BFC0A22594609480CF08FFC8F
:1038200007480CF033FC6FF00209484613B0BDE8BE
:10383000F08F00BF2D8101008C0300203981010031
:10384000700300204E810100658101001982010092
:103850008C82010097820100838101009D8101001B
:10386000B2810100CF810100DD810100E48101000E
:1038700000230993029B012B30D1039B1BB10AA8A3
:1038800001F070F803900AA801F00CFA152800F274
:10389000F880DFE810F0B700CA00A7002600B700E4
:1038A000970074005000B700B700F300F300040164
:1038B0000401E100E100F600F600F600E100E1009D
:1038C000E100A8690028D5D0049A0368CDE9007208
:1038D0000AAA9C6A099B06CAA04738E400230393FE
:1038E000D1E72846FEF712FD052807467FF46FAEA4
:1038F0008D498E480CF0BAFB0A2239468B480CF0F1
:103900001EFC8A480CF0C2FB4FF4007229460AA83C
:1039100001F0DCFF2B7D052B0CBF0E2201220AA932
:1039200010A801F070FA44F4807444F001044FF0E0
:10393000000B012768E02846FEF7E8FC062807464A
:1039400016D17B4979480CF091FB39460A22774819
:103950000CF0F5FB75480CF099FB0AA910A802229F
:1039600001F051FA4FF400212846FEF74FFDDAE747
:1039700070496E480CF07AFB0A22394662E64FF431
:1039800080312846FEF7EAFC00287FF4DBAEB8F170
:10399000000F7FF4D2AE4FF4007229460AA801F05E
:1039A00095FF01220AA910A801F02DFA44F48074B1
:1039B0004FF400212846FEF7E9FC44F001044FF0E3
:1039C000060BB6E7B8F1000F3FF4D9AE02220AA900
:1039D00010A844F4807401F016FA44F001044FF08A
:1039E000050BA6E70AA800F0B3FF074600285BD046
:1039F0002846FEF78BFC05283FF4E9AD44F48074BB
:103A000044F001044FF0000B039B002B3FF462AE27
:103A1000049B00930CAA08F0010306CA284624F46C
:103A20000074FEF7BBFFA4B254E60AA800F090FFB2
:103A300000283FF47CAFB8F1000F0DD03E493B4861
:103A40000CF014FB28460121FEF76EFC4FF4885160
:103A50002846FFF7BBFABAE50AA800F079FF074647
:103A600010B30AA800F07EFF28B94FF4007229466F
:103A70000AA801F02BFF44F44074C1E744F48064C9
:103A800055E70AA800F05FFF08B144F480740AA863
:103A900000F068FF074638B144F40074B2E74FF015
:103AA000000B4FF4806444E7BB4642E703680AAA70
:103AB0001B6B06CA984700287FF414AE1AE6D5F8A7
:103AC0001880B8F1000F39D00AAE24B12246294639
:103AD000304601F0FDF9049AA8690368CDE9007247
:103AE0009F6A099B96E80600B8478146A869036863
:103AF0009B6B9847052808BF44F0010414F4806FBD
:103B000018BF4FF00109BBF1000F03D059462846FA
:103B1000FEF70AFC069B002B3FF4F6AD2146284633
:103B2000FFF754FAF0E500BF39810100700300206F
:103B30004E81010065810100008201002B7D052B73
:103B400075D0062BDFD10AA800F0FDFE00286ED04C
:103B500041462846FEF772FC074606B20AA801F065
:103B6000A1F8049B8046002B47D024B12246294669
:103B70000AA801F0ADF9002EC5D0BCBF7E4236B216
:103B800006F1FF339BB2B4BF01270027192BBAD827
:103B9000012130460DF054FAB8F1150F09D8012370
:103BA00003FA08F8874B18EA030F35D118F0A40F71
:103BB0003AD1854985480CF059FA0A2231468348A2
:103BC0000CF0BDFA824981480CF050FA0A2205999E
:103BD0007E480CF0B4FA7D480CF058FA304606F0F6
:103BE0003DFE28B12846FEF749FE08B902F090FFD5
:103BF00044F4807444F001047DE0304606F02EFE6B
:103C00000028B2D0734974480CF030FA72480CF0B6
:103C10003DFA6FF0040908E687F0010305931946A1
:103C200030460DF035FAC4E705973946F8E724B178
:103C3000224629460AA801F04BF9029B022B5DD0CF
:103C4000032B09D0012B7FF45EAF44F4807444F061
:103C50000104DDF8089056E72846FEF7C3FC030C84
:103C6000074611D15D495E480CF000FA6B685C486C
:103C700019680CF004FA5A480CF008FA6B685949B4
:103C80001A6859480BF084FC304600F0C7FE0EF06D
:103C900015FD0022554B0EF069FD0FF017F80FFAD5
:103CA00080F8082006F0BEFD68F30F07064660F3B3
:103CB0001F474F4945480CF0D9F96B6843481968CC
:103CC0000CF0DDF94B4941480CF0D0F90A2241468D
:103CD0003E480CF034FA48493C480CF0C7F9B1B200
:103CE0000A223A480CF02BFA38480CF0CFF9394642
:103CF0002846FEF78FFC4FF0010904E744F40074F6
:103D000078E7069B002B3FF4FFAC29464FF4806216
:103D10000AA801F0DDF84FF4806100E700F05CFED6
:103D200000287FF489AA04468046FFF78CBA029ADD
:103D3000AAB91B78002B3FF4EBA909A8FEF726FDD2
:103D40000290304601F066F828B99DF80820314607
:103D500010A801F061F8029B002B3FF4D9A9274974
:103D60001A480CF083F90A22214618480CF0E7F9AA
:103D7000234916480CF07AF96B68144819680CF05E
:103D80007EF9204911480CF071F909990F480CF09F
:103D900076F91D490D480CF069F9304601F032FA08
:103DA000099B002B3FF4C7A91B78242B7FF4C3A9E0
:103DB000164906480CF05AF904480CF067F96FF000
:103DC000030932E542C03000588201007003002030
:103DD0000F7F01004B8201008C0300205D820100F7
:103DE000BC0300206D820100E80300200000594060
:103DF0007C8201008382010087820100EC80010047
:103E0000F7800100FE800100247F01000481010091
:103E10002DE9F04F91B08046CDE90421994609B9CA
:103E2000002013E006F0E4F9B0F5966F044610DACE
:103E3000B549B6480CF01AF90A222146B3480CF0ED
:103E40007EF9B2480CF022F94FF0FF3011B0BDE816
:103E5000F08F049B0BB11B782BB998F81C3013B171
:103E600008F11C030493049BE3B9D8F82C6016BB3B
:103E70004021059810F0D4F900283CD004460023D6
:103E800004F8013B0598214606F0E6FC05948246BD
:103E90000024059D2F5D87B3384611F01EFA285582
:103EA0000134F6E71B78002BDFD004A8FEF76EFC88
:103EB00006460028D9D00D2EDAD10AAC00221146D0
:103EC000204600F0BBFB059A21460CA800F08FFFAE
:103ED000324621460CA800F09FFFB9F1000F9FD198
:103EE000CDF8049001230093049B94E8060040461B
:103EF000FFF7CEF8AAE78246CAE7284600F050FB53
:103F000006ACC2B205463946204600F097FB052EA6
:103F100028D0062E08BF17255FFA86FB0CAF5A463D
:103F20002146384600F078FF092D1DDC082D80F26F
:103F3000DA80AA1C03DB6B1C7FF772AFF5B105A812
:103F400006F0ADF8024618B12146384600F0CFFE23
:103F5000B9F1000F7FF464AF01230093CDF804A002
:103F60004B46C2E71825D7E7172D00F08B80182D98
:103F7000E5D100222146384600F045FF08AD05A9ED
:103F8000284606F0ADF85A462946384600F044FF68
:103F9000284600F089FE10F1000B18BF4FF0010B0E
:103FA0000022059913B259B1032A08D005A803923B
:103FB00006F075F8039A47F822000132F1E713463C
:103FC0000B2E11D00C2E17D00A2E1DD1284600F032
:103FD00003FD81B2204600F0A7FBB9F1000F7FF48A
:103FE0001FAFCDF804A07DE7284600F0F5FCC1B274
:103FF000204600F0B4FBF0E7284600F0EDFC014657
:10400000204600F0BEFBE8E75B449BB2013B032B7C
:1040100030D8DFE803F00207122095E8030084E8B7
:104020000300DAE7284600F0D7FC9DF8303082B272
:1040300021460AA800F0A4FECFE7284600F0CCFCF9
:104040009DF8342000929DF8303082B221460AA8B3
:1040500000F07FFEC1E7284600F0BEFC9DF834204A
:104060000092214682B29DF830300AA800F071FE1D
:104070000E99C5E7264925480BF0F8FF23480CF0B8
:1040800005F8AAE700222146384600F0BCFE0025CC
:10409000059A2BB242B1042D0AD005A805F0FFFF06
:1040A00047F825000135F3E7032B10D0042B94D1FA
:1040B0009DF83C1001919DF8381000919DF8343026
:1040C0009DF8302021460AA800F07EFE85E79DF885
:1040D000381000919DF834309DF8302021460AA810
:1040E00000F062FE79E70AAC05A9204605F0F8FF6A
:1040F000EAB22146384600F086FE5A462146384646
:1041000000F08AFE69E700BF9E8201008C03002058
:10411000BC8201002DE9F04F91B0804616469946C9
:104120009DF868A0002973D00B7C03F00F03052BCA
:104130006ED1384DCC682B78DFF8E0B001332B70AE
:10414000002C62D0237C03F00F03042B04D001D396
:10415000062B4ED96468F3E76269D8F80010584618
:104160000AF07CFC07460028F4D0037C03F00F0320
:10417000052BEFD1284B01461A6804A8FEF7FAFA7E
:104180006EB104A8FEF774FA48B100230093CDF88D
:1041900004A04B463168726804A8FEF779FF9DF8C9
:1041A0002430072B18D10122394658460AF04CFC1E
:1041B000CDF800A001464B4632464046FFF7AAFF25
:1041C0009EB990B12B7804A8013B2B70FEF794F8B0
:1041D000012011B0BDE8F08F3EB904A8FEF748FAFF
:1041E00018B104A800F01CF8EBE704A8FEF784F867
:1041F000B0E70023CDE901330093326873684FF0D4
:10420000FF31204606F020F9A4E72B78013B2B7004
:104210000020DEE76D030020DC030020780700208B
:104220007FB500221146054602A800F007FA4A4968
:104230004A480BF01BFF6B68484819680BF01FFFDA
:10424000474946480BF012FF2846FEF711FA58B9C5
:10425000444942480BF00AFF40480BF017FF4FF06B
:10426000FF34204604B070BD2846FEF74FF80646DE
:10427000A86958B10368DB6A984704B2002C05DBD3
:1042800014BF01200020FEF743FCEAE72B7D072B3B
:1042900013D0701C152810D80126334C06FA00F0F4
:1042A000044004D110F0490F07D02046EBE72F4916
:1042B0002A480BF0DBFE3446D3E74FF40072294660
:1042C00002A800F0B0FD2B7D033B062B3DD8DFE8B4
:1042D00003F038233C3C04382300AB681B7C03F01C
:1042E0000F03052B4FF000041BD121491B480BF095
:1042F000BDFE234622460094A9682846FFF70AFF20
:104300001C49044615480BF0B1FE2046FEF700FCA0
:1043100012480BF0BBFEA4E7002102A800F056FCF7
:10432000044615490D480BF0A1FE21460A220B4810
:104330000BF005FF09480BF0A9FE003418BF01245B
:104340008FE702A800F048FBEAE70C4903480BF0AE
:104350008DFE002485E700BFF1820100700300207C
:10436000247F0100F982010084803000217F010058
:1043700005870100028301000F830100058301000E
:10438000F0B54FF4006185B00546FDF7E7FF002862
:1043900047D0002202AC1146204600F04FF94FF4FE
:1043A00040722946204600F03EFDAB69002B38D014
:1043B0004FF400612846FEF729F81B491B480BF013
:1043C00055FEA869002301260268CDE90063976ABB
:1043D00094E80600B847431C044622D06B68134893
:1043E00019687CB90BF04BFE114910480BF03EFEEA
:1043F00010490E480BF03AFE0C480BF047FE2046E1
:1044000005B0F0BD0BF03BFE094908480BF02EFE4D
:10441000094906480BF02AFE04480BF037FE3446E3
:10442000EDE70224EBE700BF63800100700300208A
:104430008A800100188D0100008601002DE9F04FEF
:10444000044689B08946FFF79BFF0522616847480B
:104450000AF0FAFA0646002872D0037C03934FEA6A
:10446000131A45690CF0FEFBBAF1000F68D0A5EBFA
:10447000000804AD52460B21284606AF00F0DEF8D6
:1044800042462946384600F032FCB9F1040F17D1F4
:104490000023009395E806004FF400532046FEF7F2
:1044A00045FB0A224FF47A71314898FBF1F10BF089
:1044B00024FE30492E480BF0D9FD2D480BF0E6FDC7
:1044C000B8F1000F3CDA2C4B984539DB05F090FE33
:1044D0004FF00008CDF8008083464FF4005395E874
:1044E00006002046FEF722FBBBF5966F10DA234943
:1044F00023480BF0BBFD0A22594621480BF01FFE52
:104500001F480BF0C3FD4FF0FF3009B0BDE8F08F3E
:10451000337C68F30713337452464146384600F043
:104520008DF8039B03F00F03DA1F534253410193AD
:104530000123009397E8060043462046FEF7A8FDB6
:10454000B9F1010F02D12046FEF780FDA06908B93C
:104550000020DAE703685B6998470028F8D0A06973
:1045600003680FFA89F19B689847CEE77807002027
:1045700070030020C982010002000080D88201007F
:104580008C03002007B5002300931A461946034800
:104590000BF024FD03B05DF804FB00BF30030020E6
:1045A000F8B50646F0B10378E3B12D2B1ED0A3F188
:1045B0003002092A1AD9252B1AD07B2B1AD0232B8B
:1045C0001BD00F4F012404EBC4053D4428460FF0D7
:1045D00062FE2946024630460FF079FE20B10134D2
:1045E000192CF0D14FF0FF342046F8BD0024FBE732
:1045F0000824F9E76FF00104F6E71724F4E700BF99
:1046000031830100F8B5064690B1037883B10A4FB3
:10461000002404EBC4053D4428460FF03CFE294627
:10462000024630460FF053FE20B10134172CF0D172
:104630004FF0FF342046F8BD1284010010B500236E
:104640008370C370037143718371C37161F303039A
:104650004370027010BD002202708270C270072287
:10466000427041607047000093B2112B70B516463E
:104670009CBF134AD25C4B7888BF002262F30303CD
:104680004B7005460C460F480F490BF0EFFC0A2211
:1046900031460C480BF053FD0C490A480BF0E6FC80
:1046A000617808480A2201F00F010BF061FD05480E
:1046B0000BF0ECFC23682B6063686B60284670BDD0
:1046C0001A830100700300205785010062850100F4
:1046D0004B7803F00F03013B082B1AD8DFE803F0F7
:1046E000160E0E19191919050C000D4B4B600B68AD
:1046F00003604B68436070470A4BF7E764238B7194
:10470000CB7923F00103CB7100234B71FF230B7195
:10471000EDE700230B714B718B71CB71E7E700BFA5
:104720000000A04100009642437813F00F0203D02E
:10473000022A05D000207047022262F3030343706F
:1047400040F26D139942A8BF1946C379817123F0D5
:104750000103C1F300211943C1710120704743785F
:1047600013F00F0203D0022A05D000207047022266
:1047700062F3030343706429A8BF642141710120DF
:10478000704713B50446084631B9E37960F347032F
:10479000E371012002B010BD642300934FF4FA725C
:1047A000002399210CF0E9F8637813F00F0208D088
:1047B000032A0BD820EAE0706428A8BF64200130E7
:1047C000E3E7022262F303036370F3E70020E1E70B
:1047D00007B5C27912F0FE0F12D0437803F00F0331
:1047E000013B022B0CD850084FF4FA73009364225B
:1047F0009923002101380CF0C0F803B05DF804FBE8
:104800004FF0FF30F9E7C379827903F0010342EA00
:104810000320704740797047437803F00F03013B52
:1048200010B50A2B53D8DFE803F00606525252485F
:104830002F2F2F1010000279642391FBF3F1114404
:1048400081F308010171012010BD632944684FF014
:1048500064030FDC03FB04112AB153439942A8BF40
:10486000194621EAE17143784160062262F30303AD
:104870004370E8E791FBF3F12144E2B19142A8BF14
:10488000114621EAE17116E0436807EE903AFDEE29
:10489000E77A642417EE903A91FBF4F1194422B1BF
:1048A0009142A8BF114621EAE17107EE901AF8EE95
:1048B000E77A17EE901A4160C5E743681944002A69
:1048C000F9D0642353439942A8BF1946D9E7002081
:1048D000BAE7437803F00F03022B1ED1C279837924
:1048E00002F0010243EA0223642291FBF2F119442F
:1048F000B1F5B77F0FDA40F26D1331EA210128BF1D
:104900001946C379817123F00103C1F300211943D2
:10491000C171012070470021F3E700207047437800
:1049200003F00F03022B0CD14379642291FBF2F1C7
:10493000194421EAE1719142A8BF11464171012059
:104940007047002070470078003018BF0120704782
:104950008378012B04D80078003018BF01207047FD
:1049600000207047407810F00F0018BF01207047FA
:10497000407800F00F00023803288CBF002001208F
:1049800070470000437803F00F03013B0A2B1ED849
:10499000DFE803F00A0A1D06061B0F0F0F060600CC
:1049A00043686420584370470079642310FB03F088
:1049B000704743689FED077A07EE903A67EE877A73
:1049C000FDEEE77A17EE900A7047406870470020C6
:1049D000704700BF0000C842437803F00F03013B5B
:1049E0000A2B18D8DFE803F00808170606120A0A8F
:1049F0000A0606004068704700797047406807EE75
:104A0000900AFDEEE77A17EE900A7047406864233B
:104A100090FBF3F07047002070470000437803F0EC
:104A20000F03013B0A2B1ED8DFE803F013131D060A
:104A3000060E191919060600436807EE903AF8EEBB
:104A4000E77A17EE900A70474368642293FBF2F30B
:104A5000F3E7037907EE903AF8EE677AF1E74368F7
:104A600007EE903AEDE7DFED017AEAE7000000009B
:104A7000437803F00F0307B50B2B60D8DFE803F092
:104A80006216165F5F5F44245F5F0606406849B1A7
:104A9000D0F1640056D46428A8BF642000B203B0EB
:104AA0005DF804FB0028F6DA0846F8E7007931B132
:104AB000002100916423FF220BF05FFFEEE76423E7
:104AC0000093FF220B46F7E7436807EE903A99B14F
:104AD0009FED1E7A77EE677AF5EEC07AF1EE10FA66
:104AE00030D4F4EEC77AF1EE10FA2DDCFDEEE77A61
:104AF00017EE903A18B2D2E7F5EEC07AF1EE10FA5E
:104B0000D2D49FED127AECE7436861B142F273723E
:104B1000934217DC13F1630F16DB6FF0630093FB16
:104B2000F0F06430BAE713F1630FBDDB42F2737249
:104B300093424FF06400B2DC93FBF0F0AEE74FF02D
:104B4000FF30ACE70020AAE76420A8E70000C842D5
:104B500013B504460846637803F00F03013B0A2BA4
:104B600032D8DFE803F00F0F313131281A31310626
:104B70000600FF2300930023642219460BF0FDFE7C
:104B8000606007E0FF2300930023642219460BF0C6
:104B9000F4FE2071012002B010BDFF23009300231A
:104BA000642219460BF0E9FE07EE900AF8EEE77A68
:104BB00017EE900AE4E746F29C3300930023642248
:104BC00019460BF0DAFE60600020E4E7437803F05A
:104BD0000F030B2B5FD8DFE803F06117175E5E5EF3
:104BE000461E5E5E0606406841B1002839DBFF289C
:104BF000A8BFFF20C0F1FF0001B20AE0002808DBD7
:104C0000FF28A8BFFF20F7E700790029F4D0C0F102
:104C1000FF01084670474368A9B107EE103AB5EEA8
:104C2000C07AF1EE10FA1CD4DFED1D7AB4EEE77A0B
:104C3000F1EE10FA32DC77EEC77AFDEEE77A17EE86
:104C4000903A19B2E5E707EE903AF5EEC07AF1EE48
:104C500010FADED49FED127AF4EEC77AF1EE10FA74
:104C6000EBDDFF21D5E7406859B110F1630FF8DBA8
:104C7000B0F5C84F12DA6FF0630190FBF1F0FF302E
:104C8000BAE710F1630FC4DBB0F5C84FE9DA64216D
:104C900090FBF1F0B0E74FF0FF31BAE70021B8E741
:104CA00000007F4300787047407800F00F007047A5
:104CB0004B7810B562F303034B700B6803604B68CD
:104CC000436010BD4B7810B503F00F04013C012C7C
:104CD00084BF012464F3030382F30802D2B288BFC5
:104CE0004B700B680A7103604B68436010BD4B78D2
:104CF0004A6030B50A2565F303034B700B68036007
:104D00004B68436030BD4B784A6030B5072565F38A
:104D100003034B700B6803604B68436030BD4B78F6
:104D200030B5062565F303034B700A235A434A60E6
:104D30000B6803604B68436030BD4B784A6030B508
:104D4000062565F303034B700B6803604B684360F3
:104D500030BD70B54C788A71022666F303044C703E
:104D6000C2F30024CA794B7122F001029DF8103081
:104D70000B7122430B68CA7103604B68436070BDBE
:104D800070B54C788A71032666F303044C70C2F345
:104D90000024CA794B7122F0010222430B68CA71C8
:104DA00003604B68436070BD70B54D784B7104264D
:104DB00066F303059DF810304D700B718A710B6816
:104DC00003604B68436070BD70B54D784B7105262C
:104DD0009DF810300B7166F303059DF814304D708B
:104DE000CB718A710B6803604B68436070BD4B7870
:104DF0004A6030B50C2565F303034B700B68036004
:104E00004B68436030BD10B50A700B6803604B6897
:104E1000436010BD8078704710B58A700B680360DE
:104E20004B68436010BD2DE9F041044616460D461F
:104E300019B900273846BDE8F0810846FDF718FC8F
:104E400007460028F5D02846FDF76CFBF3058046A1
:104E500003D52846FDF75AFA207006F40076B8F11B
:104E6000000F09D0637868F303036370002EE1D06C
:104E7000EB685B696360DDE7002EDAD0EA68137CDB
:104E800003F00F03022B03D0032B09D04746D1E7D1
:104E90006378526962600A2161F303036370C9E7B2
:104EA00053696278072161F303026270E2E710B58B
:104EB00000230446037043708370C3700371437111
:104EC0008371C3714FF40072FFF7ADFF204610BD30
:104ED000F8B5054617460C4611B900263046F8BD10
:104EE0000846FDF7C5FB06460028F6D079050CD527
:104EF0002B780A3B032B08D8DFE803F02002252B90
:104F00004FF480312046FDF741FAFA0507D529789C
:104F1000A1F10A03032B02D92046FDF705FABB05D0
:104F2000DCD56B78696803F00F03073B2046042B40
:104F300018D8DFE803F01111171414004FF4803172
:104F40002046FDF763FA4FF400312046FDF75EFA84
:104F5000DBE74FF40031D5E7FDF71AFBBEE7FDF7BD
:104F6000FBFABBE7FDF7F8FA6978204601F00F017C
:104F7000FDF72AFBB2E7000070B5174E174D044647
:104F800034B3237C03F00F03023B042B20D8DFE86B
:104F900003F0031F0F0608006569284670BDE4682A
:104FA000EEE721463246284609F058FD0446E7E779
:104FB00066693046FFF726FB051E09DB304609F01F
:104FC00043FE237C6561022262F303032374E4E75A
:104FD0004FF0FF35E1E700BF2C8301007807002088
:104FE0002DE9F0432DED028B85B004461546994618
:104FF0009DF838800F46002947D0002A00F0E6804F
:1050000000230B70017869B319F4807F2AD0704BAC
:1050100001EBC101194438460FF06BF963781907A9
:1050200007D019F4007F04D02A466A4938460FF0A9
:105030003AF938460FF02FF92D1A3E18013D6378E2
:105040001A0722D019F4007F1FD003F00F03013B91
:105050000B2B1AD8DFE803F0084071A6AC257B7B48
:105060007B221FB43E46EAE72079B8F1000F06D054
:10507000642300930023FF2219460BF07EFC564A5E
:105080000346294630460EF0FBFF384605B0BDEC1E
:10509000028BBDE8F0836368504AF2E76368504AC8
:1050A000EFE7616800294FF064020EDA91FBF2F03D
:1050B0004B4202FB1011494293FBF2F3494A009123
:1050C000294630460EF0DCFFDFE791FBF2F302FBEE
:1050D00013120092444AF3E72046FFF779FBE27986
:1050E000A37994F8059001B20029207902F0010219
:1050F00002DBB8F1000F14D043EA0224B8F1000F2C
:1051000006D0642300930023FF2219460BF035FCE0
:10511000CDE900902346354A294630460EF0B0FFCF
:10512000B3E7CDE90101CDF8009043EA0223304A0C
:10513000294630460EF0A4FFA7E7E379A27961790A
:10514000009103F0010342EA03232A4AB8E76368A7
:1051500008EE103AB5EEC08AF1EE10FA4CBFF1EE4F
:10516000487AF0EE487AFDEEE78AB8EEE87A77EE14
:10517000C77A9FED217A67EE877A17EE900A0CF0D6
:105180004DF807EE900AB5EEC08AFDEEE77AF1EE33
:1051900010FACDED007A18EE903A01D5174A8FE754
:1051A000174A8DE72279A379019262790092B2E7DA
:1051B000E279A37902922279019262790092B6E7AC
:1051C0002A46616830460FF094F85EE717465CE7C0
:1051D00031830100247F0100718501007485010085
:1051E000788501007C8501007D85010089850100AD
:1051F000868501008C85010000007A4492850100BB
:105200009385010030B58BB0134C0023202200930E
:1052100002A94FF440730546FFF7E2FE02A92046BB
:105220000AF02DFF0D4920460AF020FF69780A2276
:1052300001F00F0120460AF09BFF094920460AF0C1
:1052400015FF0A22A97820460AF092FF20460AF0AC
:105250001DFF0BB030BD00BF70030020658501004D
:105260006A85010070B54B7803F00F03934286B056
:1052700005460C46164606D123682B6063686B60B2
:10528000284606B070BD194919480AF0EFFE61784A
:1052900017480A2201F00F010AF06AFF1549144865
:1052A0000AF0E4FE0A22314611480AF061FF124971
:1052B0000F480AF0DBFE0023CDE9043366F3030355
:1052C00022788DF811304FF0FF338DF810200093C5
:1052D00002A86368226804A900F010F8029B23600A
:1052E000039B63602046FFF78DFFC5E79B850100A8
:1052F000700300208E7E0100247F01002DE9F04F15
:105300008DB004AD85E80C00BDF85830112B98BF66
:10531000BC4A804628460C4694BF12F803904FF0D2
:105320000009FFF755FA011E02DB2046FFF729FAB4
:105330009DF81230A3709DF810302370637803F04D
:105340000F030B2B3BD8DFE813F0A5000C000C007B
:10535000D4003F011901B000DA00DA00DA00B00031
:10536000B0009DF8113003F00F030C2B77D8DFE865
:1053700003F0265244180A073955767630306E000D
:105380009DF81720E2719DF81620A2719DF8152056
:1053900062719DF814202271627863F303026270D7
:1053A0000DE0BDF81630C3F30802E379A27123F0D3
:1053B000010343EA1223E3719DF815306371B9F1DB
:1053C000000F00F009814A46214606A8FFF74AFF70
:1053D00002E1059B002B36DBFF2BA8BFFF23DBB2CE
:1053E0002371ECE7059B13F1630F2CDBB3F5C84F7A
:1053F0002BDA642293FBF2F3F1E7BDF81630C3F326
:105400000802E379A27123F0010343EA1223E37156
:105410009DF8153063719DF81430E1E7DDED057AF4
:10542000F5EEC07AF1EE10FA0DD49FED777AF4EE36
:10543000C77AF1EE10FA08DCFCEEE77ACDED037ADC
:105440009DF80C30CCE70023CAE7FF23C8E7637858
:105450000C2262F303036370059B6360AFE76B4943
:105460006B480AF003FE9DF8111069480A2201F00A
:105470000F010AF07DFE674965480AF0F7FD617883
:1054800063480A2201F00F010AF072FE60480AF038
:10549000FDFD94E79DF81130C3F30303627805988E
:1054A000606063F30302627089E79DF8113003F0D6
:1054B0000F03032B04D00C2BC9D0059A62606BE755
:1054C00000212046FFF782FBBDF816302071C3F3A0
:1054D0000802E379A27123F0010343EA1223E37186
:1054E0009DF8153063716378022262F303036370E1
:1054F00065E700212846FFF769FB2071F3E79DF877
:10550000113003F00F030C2BA9D801A252F823F09D
:10551000BF5300004F5500009D540000C1540000CF
:105520009D5400009D540000455500007155000039
:1055300071550000715500005D5500006B5500006D
:105540004F540000059B636006226378CDE79DF809
:10555000143007EE903AF8EE677A03E0DDED057A55
:10556000F8EEE77A17EE903A77E7DDED057AF2E7A5
:10557000627863F303026270059B6EE701279DF872
:10558000113003F00F030C2B3FF669AF01A252F864
:1055900023F000BFBF530000ED550000415600004E
:1055A000ED550000CD550000CD550000ED55000033
:1055B000ED5500005F5400005F540000ED55000001
:1055C000ED5500004F5400000027D8E7059A6260AF
:1055D000627863F3030262702368C8F8003063687E
:1055E000C8F8043040460DB0BDE8F08F013B0A2BEF
:1055F00000F2CD80DFE803F0BACB10CBCBBFC4CB39
:10560000CBBDBD001A83010000007F43E18401008F
:10561000700300208E7E0100FF23BDF816208DF858
:105620001430642161F30802ADF8162000228DF8D1
:1056300015209DF81120022161F303028DF811203D
:105640000023FF259DF815000095642219460BF0F4
:1056500094F90028C0F29D8000239DF81500009564
:10566000642219460BF089F9A84208DC0023009552
:105670009DF81500642219460BF07FF905469DF848
:105680001400FAF7F7FE0646002F47D09DF8177072
:105690007F08013F3FB27B1C40F088807F2D4FF098
:1056A000FF0778DC0023C5F17F00194647F68162C9
:1056B000704300970BF061F94FF4FF7300930023E0
:1056C0001946E0717F2228460BF057F9002319464E
:1056D00000903A4630460BF050F900970646642396
:1056E00028467F2200210BF048F9BE420546A8BF9C
:1056F0003E466C496C480AF0B9FC0A2229466A48C1
:105700000AF01DFD694968480AF0B0FC0A223146DA
:1057100065480AF014FD64480AF0B8FC00231A46F4
:10572000194606A80AF01AFBBDF816004FF6FF73DB
:1057300000930023194640F26D12C0F308000BF0ED
:105740001CF9F2B2E9B280B20AF01EFB030CA3719D
:10575000030A63712071564953480AF087FC2046BA
:10576000FFF750FD06A80AF08EFA28E69DF81430DF
:1057700053E7059B51E7059B642293FBF2F34CE74B
:10578000DDED057AFDEEE77A17EE903A45E7002366
:1057900043E7002573E76423284600973A468021B3
:1057A0000BF0EBF800230546E371A2E74FF01E0B68
:1057B00064231A46CDF800B0002138460BF0DDF81E
:1057C0004FF0640A03905B463846CDF800A052467D
:1057D00000210BF0D2F87F2D83464FF0FF0754DCF9
:1057E000C5F17F00002370431946324A00970BFB36
:1057F00000F00BF0C2F84FF4FF73E07103980093D0
:1058000000231946E32228180BF0B7F800231946A5
:1058100000903A46824630460BF0AFF80023064629
:10582000009728467F2219460BF0A7F8BE4205468E
:10583000A8BF3E4620491C480AF018FC0A220399DA
:1058400019480AF05AFC1D4917480AF00FFC0A22B1
:10585000594615480AF051FC194913480AF006FC4C
:105860000A22294610480AF06AFC16490E480AF036
:10587000FDFB0A2231460C480AF061FC12490A4835
:105880000AF0F4FB0A22514642E7534628460097A5
:105890003A4680210BF071F84FF0000A054684F873
:1058A00007A0C7E7F3840100700300200085010012
:1058B00033850100646A31000E8501001485010002
:1058C0001A850100228501002A85010073B504466E
:1058D0000D46FFF7A8FA0646E8B9104910480AF045
:1058E000C5FB2846FDF7CCFB214602B26846FEF711
:1058F000BBFE21466846FEF7EBFE29464FF40072D8
:105900002046FFF7E5FA2046FFF77CFC4FF4905164
:105910002846FDF75BFB304602B070BD3A850100BA
:1059200070030020437803F00F03013B012B37B5D0
:10593000054620D80023FF240079009464221946EC
:105940000BF01BF8002814DB002328790094642254
:1059500019460BF012F8A04207DC002300942879C6
:10596000642219460BF009F8C4B22C71012003B06F
:1059700030BD0024F9E70020F9E7000007B5002357
:1059800000931A46194603480AF028FB03B05DF855
:1059900004FB00BF3803002002F02CBE02F0ECBD77
:1059A00007B5002300931A46194603480AF016FB70
:1059B00003B05DF804FB00BF40030020024B0F2240
:1059C0001A70C820704700BFE003002008B50449E2
:1059D00004480AF04BFB04F00DFD4FF4FA7008BDCB
:1059E000218B0100BC03002038B5094D01244FF480
:1059F0007A700BF06BF9214601340A222846E4B292
:105A00000AF0B6FB142CF2D14FF4FA7038BD00BF87
:105A1000BC03002008B504F0ABF8C82008BD10B5E1
:105A2000044604300AF0B3FF204610BD0128F8B543
:105A300007460C46174E184D13DD48680DF0FFF968
:105A4000C1B216483170FBF723F9022F07D0A068C6
:105A50000DF0F5F9C1B211482970FBF72AF9C824F5
:105A600001E04FF4C8740E490E480AF0FFFA0A220A
:105A700031780C480AF07CFB0B490A480AF0F6FA28
:105A80000A22297807480AF073FB06480AF0FEFA52
:105A90002046F8BD05000020060000204404002038
:105AA000C28C0100BC030020D68C010030B587B049
:105AB0000023044600931A460D4602A819460AF030
:105AC0008DFA04A80AF082FA042C12DD04A92869D0
:105AD00004F096FB68B104A92548FAF7BEFF04A9B3
:105AE000E86804F08DFB50B104A92148FBF701F8E8
:105AF0000BE002A91E48FAF7B0FF032CEFDC02A965
:105B00001B48FAF7F6FF022C1CDD04A9A86804F074
:105B100077FBB8B104A91648FAF7C5FF04A968686D
:105B200004F06EFBA0B104A91148FAF770FF114907
:105B300011480AF09BFA00210D48FBF779F8C820BC
:105B400007B030BD02A90A48FAF7ADFF012CE5DC29
:105B500002A90748FAF75BFF012CE8D102A9044823
:105B6000FAF755FF054904480AF080FADFE700BF5D
:105B7000440400206C870100BC0300205C87010006
:105B800008B548B149680548FAF7F1FD04490548E8
:105B90000AF06CFAC82008BD0146F4E7440400206E
:105BA0000B8B0100BC030020012838B50C4630DD0A
:105BB0004D68214928460EF006FB28B901211F48EF
:105BC000FBF753F8C82038BD1D4928460EF0FBFAF4
:105BD00001460028F3D01B491B480AF047FA174832
:105BE000FBF739F80A22014617480AF0A8FA1648C6
:105BF0000AF04CFA61681148FAF70AFE6168124827
:105C00000AF03DFA114910480AF030FA0E480AF03D
:105C10003DFA0F4B93F90020012A02DDF0221A70A1
:105C2000D0E70C490C480AF021FA0B480AF02EFA8A
:105C30004FF4FA70C7E700BFCA9201004404002085
:105C4000D39201009A870100BC030020BA870100AB
:105C5000E0030020C18701008C03002008B548B193
:105C600049680548FAF758FD044905480AF0FEF965
:105C7000C82008BD0146F4E744040020CE87010097
:105C8000BC03002030B5154D154C85B0772201219D
:105C90002846FBF73DFA00230193124B009312496B
:105CA00002954FF0FF33204603930AF0DFF90F49C6
:105CB0000F48096801236A4608F092FE2846FBF760
:105CC000D3F90C4920460AF0D1F920460AF0DEF952
:105CD0000948FBF7D7F805B030BD00BF5C040020D1
:105CE000BC030020509C01006A8A01003804002097
:105CF00078070020848A010044040020012810B5A0
:105D00000C4622DD124960680EF05DFA18B90121D7
:105D10001048FAF770FF104960680EF054FA014617
:105D200010B90C48FAF767FF0C490D480AF09EF9C4
:105D30000848FAF756FF0A22014609480AF0FFF917
:105D400007480AF0A3F9C82010BDFFF79BFFFAE748
:105D5000CA92010044040020D3920100948A0100F9
:105D6000BC03002008B50A48FBF746F818B10949FA
:105D700009480AF07BF9722201210848FBF7C8F9AB
:105D80000648FBF765F90548FBF76EF9C82008BD22
:105D9000440400202C8E0100BC0300205C04002081
:105DA0002DE9F041494F3B688CB0002B00F08B800F
:105DB000474B1B785BB283420ADD464946480AF0EE
:105DC00055F945480AF062F900200CB0BDE8F081B1
:105DD0004249434D4348444E0AF048F941480AF0CD
:105DE00055F92B7801335BB22B70336803B3DC6851
:105DF000DFF810811CB3237C03F00F03052B15D1B2
:105E00002146404608F016FE80B132682168684697
:105E1000FCF7D2FC6846FCF72BFC10B16846FCF797
:105E200065FA0AF075FF6846FCF766FA6468E1E710
:105E30002E492C480AF01AF92A480AF027F92C4B67
:105E40002C49284800241C600AF010F925480AF063
:105E50001DF964200AF03AFF274B28491C70284B93
:105E600020481C700AF002F904F0C2F90A22014627
:105E70001C480AF070F93968224808F0CAF9224B28
:105E800022491C60224B17481C60224B3C601C605E
:105E9000214B34601C60214B1C60214B1C70214B3A
:105EA0001C600AF0E3F804F0A3F90A2201460D4849
:105EB0000AF051F90B480AF0E9F81B4B1C702B78DB
:105EC000013B5BB22B7001207FE700BF380400204C
:105ED0006D030020369201008C0300204D920100DA
:105EE0008804002070030020DC030020639201007E
:105EF0003404002073920100800400207B92010092
:105F00006C03002078070020D803002015830100CF
:105F1000A004002068030020E40300208803002080
:105F2000640300202C0400206E030020034B93F92F
:105F30000000053818BF0120704700BFE0030020B3
:105F400030B593B000230A460546402101A804F06D
:105F5000C9F901A80EF09FF901A904460246284696
:105F60000EF0B5F900280CBF2046002013B030BD5C
:105F70002DE9F04304469DB00F4601B1AAB9784916
:105F800078480AF073F8784976480AF06FF82146A5
:105F900074480AF074F8754972480AF067F8714855
:105FA0000AF074F81DB0BDE8F08300258D5404F0AC
:105FB0001FF96F4906466B480AF058F80A22314625
:105FC00068480AF0BCF86B4966480AF04FF8214669
:105FD00064480AF054F8684962480AF047F8B6F590
:105FE0009D7F05DA654966480AF040F86448D7E7BE
:105FF0000421644803F0FAFE63495A480AF036F86F
:10600000394658480AF03BF85F4956480AF02EF8DE
:1060100054480AF03BF83C2229460DA80C950DF097
:1060200094F95A4B93F90020052A994627D1032168
:106030002046FFF785FF06B26EBB554DEB681B7817
:10604000DB07AFD501212046FFF77AFF00B2002819
:10605000A8D0242120460EF06DF90028A2D14D4988
:1060600040480AF003F821463E480AF008F83D4847
:106070000AF00CF82146284609F02BFA92E7012194
:106080002046FFF75DFF06B2002E4CD03F2221468E
:106090000CA80EF02EF9A846012526443E493046AC
:1060A0000EF0CBF8002849D0242120460EF042F90A
:1060B00000287FF477AF1DB9B8F1000F3FF472AF3D
:1060C000364B31461A686846FCF776FB6846FCF7A3
:1060D000CFFA044648B100231A4639466846FDF710
:1060E00097FE0028D4BF002401246846FCF704F979
:1060F000002C3FF457AF9DF83030002B3FF452AFE7
:1061000099F90030052B3FF44DAF2549154809F0AA
:10611000ADFF0CA9134809F0B2FF124809F0B6FF11
:106120000CA91B48A8E702212046FFF709FF06B289
:10613000002E3FF437AF4FF00108AEE738460EF0BF
:10614000AAF80128B0D92146114809F0C2F91DB9B1
:10615000B8F1000F3FF426AF384608F09DFD21E767
:10616000719C010070030020FE860100B0A10100B7
:10617000078701000D8701001087010013870100C8
:106180008C0300203C040020047E0100E00300207A
:10619000E803002020870100B8920100DC03002002
:1061A0003E8701002DE9F04116491748174E184F58
:1061B000154D09F05BFF0024A6F10F0816F8013F0A
:1061C0000F2B03D83946284609F059FF052C4FF00C
:1061D00010020DD03178284609F08FFF0D4928466E
:1061E00009F044FF0134E4B2062CE7D1BDE8F081A8
:1061F00098F81510284609F080FF284609F046FF58
:10620000F0E700BFA58A0100BC0300205304002072
:10621000349C01008A80010010B58AB00DF11F0383
:1062200004930DF12503039309AB0C4602930DF182
:10623000230301930DF12203009308AA0DF121031A
:106240000E4960680DF050FF05280BDC0C490D4825
:1062500009F00CFF61680B4809F011FF4FF4C8709A
:106260000AB010BD08A90848FAF709FAFFF79AFF23
:106270000649074809F0FAFEC820F1E7338B010010
:10628000478B01008C03002044040020598B01003F
:10629000BC03002008B508B9002008BD037C03F04A
:1062A0000F03052BF8D1CAB20146064808F0CCFB13
:1062B0000028F1D0037C03F00F03042BECD14069DC
:1062C000EBE700BF78070020F7B53D4C237803F0DB
:1062D000FF06002B6CD13B4B93F90030012B67DD9F
:1062E000394B1968002963D0384A394808F0B6FBA1
:1062F000054600285CD00146354808F09BFB07B2F4
:10630000002F55D031462846FFF7C4FF012F06461F
:1063100050D0294601222E4808F096FB4569684670
:1063200005F086FA10222B49684603F08FFF2A49B0
:106330002A4809F09BFE3146284809F0A0FE28496A
:10634000264809F09CFE0A222946244809F0F7FE57
:106350002349224809F093FE1E49204809F08FFE88
:106360001E4809F093FE40F202211E4805F0F8FC99
:10637000AAB231461C481D4D09F076FD15491A4850
:1063800009F076FD1A4B186818B10021FFF782FF5B
:106390002860296889B1144809F072FD002112486B
:1063A00009F076FD012313490C48237009F05EFEC5
:1063B00003B0F0BD40F20225B1E70F49EBE700BFA3
:1063C00080040020E003002038040020B98601008A
:1063D0007807002054030020C0860100BC03002081
:1063E0008A800100C8040020A40400208803002043
:1063F000E4030020CF8601005894010008B5094B42
:106400001B7873B1084B1B6813B1DA68074B1A602D
:106410000749084809F02AFE0648BDE8084009F087
:1064200035BE08BD6403002068030020E40300209B
:10643000E5870100BC03002008B50B4B1B788BB12E
:106440000A4A13685B6813601BB9BDE80840FFF790
:10645000D5BF0749074809F009FE0648BDE80840CE
:1064600009F014BE08BD00BF64030020E40300204F
:106470007F870100BC0300202DE9F04FA7B0002367
:1064800097488DF81330CDE90533CDE9073308F08F
:1064900037FE944F054610B105233B70F8E0924C4F
:1064A000216841B99149924809F0E0FD904809F00E
:1064B000EDFD0F23F1E78F4808F0BCFA0FFA80F8E2
:1064C000B8F1010FEEDD294620688B4EFFF7E2FEA2
:1064D000002800F0E08030608849894809F0C6FD56
:1064E0003168874809F0CBFD854809F0CFFD0121CF
:1064F0002068FFF7CFFEB8F1020F824600F0CE8091
:10650000022221687B4808F09FFAB8F1030FD0F807
:10651000149000F0C58003212068FFF7BBFE0546FC
:10652000102205A97748FAF7D1F8002840F0BB807F
:10653000B8F1040F40F3B78004212068FFF7AAFEEA
:10654000714904466E4809F091FD6D4809F09EFDC1
:106550001FFA89F25146624809F03EF90DF124080C
:106560006A495F4809F03BF90DF1340B1022684984
:1065700040460DF0BEFE002301222021584603F0C4
:10658000B1FE644958460DF03CFE63495C4809F091
:106590006DFD51465A4809F072FD6049584809F0AE
:1065A00065FD0A224946564809F0C9FD5C49544830
:1065B00009F05CFD2946524809F061FD59495048EF
:1065C00009F054FD2B780BB91C461D46CDF80C8004
:1065D0004FF002094FF001082A46CDE90198CDF8A5
:1065E00000B0234631683E484F4D08F09FFE00281A
:1065F0005BD04E4B4E49424800241C7009F036FDDA
:1066000031683F4809F03BFD3D4809F03FFD494BEB
:10661000032283F800804121234615A803F062FE7F
:10662000454915A80DF0EDFD15A92D4809F0A2F872
:1066300023464A46412115A803F054FE3F4915A8B8
:106640000DF0DFFD15A93E4809F030FD15A92448DD
:1066500009F090F842462346412115A803F042FE76
:10666000364915A80DF0CDFD15A9354809F01EFDD8
:1066700015A91B4809F07EF805233B700AF0F2FAD1
:10668000304928601E4809F0F1FC1D4809F0FEFC65
:1066900027B0BDE8F08F2C4B33601DE740F25B79EB
:1066A0000DF113053CE705AC52E72849104809F005
:1066B000DDFC0B4809F095F80A2201460C4809F068
:1066C0003EFD23490A4809F0D1FC094809F0DEFCE7
:1066D000FFF7B2FE0AF0C6FA0C232860DDE600BF21
:1066E000E8030020E0030020E40300200D900100F7
:1066F0008C030020780700208803002049900100C7
:10670000BC0300204404002056900100715F00008B
:10671000FE93010042940100769001008A800100FE
:10672000979001005E920100900400202804002050
:106730009E9001006E030020AC9001008C7E010051
:1067400070030020B290010058940100D590010020
:10675000E790010007B51049104809F087FC68462A
:1067600005F066F8684603F097FD0D4B00930D4B5E
:1067700068465B68019303F08FFD684605F09CF85E
:10678000684603F089FD684605F074F8684603F032
:1067900083FD03B05DF804FB448D0100BC030020C1
:1067A0001C9D01006406002010B5114C11492046C3
:1067B00009F05CFC1049204609F061FC4FF4FA70C6
:1067C0000AF084FA012115200AF03AFC0021152074
:1067D0000AF05EFC4FF4FA700AF078FA15200121F5
:1067E0000AF056FC4FF4FA70BDE810400AF06EBA99
:1067F000BC03002095920100B592010070B592B0E3
:1068000002A809F0E3FB04A809F0E0FB06A809F0E0
:10681000DDFB08A809F0DAFB71497248724E09F0F5
:1068200025FC704809F032FC02A97048FAF71BF801
:1068300000BB6F496B486F4C09F018FC4FF47A624B
:1068400042F6E0616C4804F093FE002840F092802C
:106850006A496B4809F00AFC6A49694809F006FC74
:1068600023780133DBB22370F6233370FFF79CFFEC
:1068700012B070BD5D48FAF7D3F918B15D4B1B78C3
:10688000022BD6D960495748604C10AD09F0EEFB99
:10689000039B10942846119303F0FEFC04A953486F
:1068A000FAF74BF800285DD059494E4809F0DEFB55
:1068B000059B10942846119303F0EEFC06A94B4863
:1068C000FAF770F8002841D05249464809F0CEFB4B
:1068D000079B10942846119303F0DEFC08A9434857
:1068E000F9F7F6FF10B34C493E4809F0BFFB099B8E
:1068F00011932846109403F0CFFC039B0095CDE93B
:106900000B34059B3C480A94CDE90D34079BCDE937
:106910000F34099B11930CAA0EAB0AA904F0B2FE26
:10692000304809F0B3FB02233370A1E7039B3248E0
:106930000C94CDE90D34059BCDE90F34079B1193E1
:106940000EAA2B460CA904F0CDFEE9E7039B2A48CA
:106950000E94CDE90F342A46059B11930EA904F03D
:10696000E9FEDDE7039B244810942946119304F0C7
:10697000FBFED5E729491B4809F078FB10A804F075
:1069800057FF119B039310A8204B109303F084FC36
:10699000144809F07BFB02A91448FAF738F8204B99
:1069A00012485B68119304A90593FAF77CF810A8C4
:1069B00004F082FF119B0D48079306A9FAF799F896
:1069C00010A804F057FF119B0848099308A9FAF78B
:1069D00044F801210548FAF72BF900232370A2E7B8
:1069E0006A8D0100BC030020E00300204404002065
:1069F000778D01004803002054040020AB8D010076
:106A00008C030020ED8D0100838D01001C9D010091
:106A1000998D01009F8D0100A48D01001C8E010045
:106A20006406002018B10349034809F01FBB03495D
:106A3000FAE700BF93920100BC030020B3A101005C
:106A400010B5264C2649204609F010FB2549204662
:106A500009F00CFB244B1868003018BF0120FFF729
:106A6000E1FF2249204609F001FB214B1868003064
:106A700018BF0120FFF7D6FF1E49204609F0F6FA9D
:106A80001D4B1868003018BF0120FFF7CBFF1B49D2
:106A9000204609F0EBFA1A4B1868003018BF0120A5
:106AA000FFF7C0FF1749204609F0E0FA164B1878A7
:106AB000FFF7B8FF204609F0E9FA1449204609F02B
:106AC000D5FA03F095FB0A220146204609F043FB64
:106AD0002046BDE8104009F0D9BA00BFBC03002031
:106AE0008B8C0100988C0100DC030020A08C01003D
:106AF000D8030020A98C0100E4030020B08C010021
:106B00002C040020B98C010080040020F2800100D8
:106B10000020704710B5484C4849204609F0A6FAB5
:106B20004749204609F0A2FA4649204609F09EFA54
:106B30004549204609F09AFA204609F0A7FA434948
:106B4000204609F093FA4249204609F08FFA41495C
:106B5000204609F08BFA4049204609F087FA3F4960
:106B6000204609F083FA3E49204609F07FFA3D4964
:106B7000204609F07BFA3C49204609F077FA3B4968
:106B8000204609F073FA3A49204609F06FFA39496C
:106B9000204609F06BFA3849204609F067FA374970
:106BA000204609F063FA3649204609F068FA35496B
:106BB000204609F05BFA3449204609F057FA334978
:106BC000204609F053FA3249204609F04FFA31497C
:106BD000204609F04BFA3049204609F047FA2F4980
:106BE000204609F043FA2E49204609F03FFA2D4984
:106BF000204609F03BFA2C49204609F037FA2B4988
:106C0000204609F033FA2A49204609F02FFA29498B
:106C1000204609F02BFA2849204609F027FA27498F
:106C2000204609F023FA2046254909F01FFA20469C
:106C3000BDE8104009F02ABABC0300203C8E0100D8
:106C40005E8E0100718E01007F8E0100878E010033
:106C5000978E0100A38E0100B08E0100C58E010049
:106C6000D48E0100DC8E0100E78E0100F48E01005D
:106C7000FE8E01000D8F0100158F0100218F010094
:106C8000B5920100378F0100568F01006B8F010014
:106C9000788F0100868F0100928F01009A8F01008A
:106CA000A58F0100B28F0100BA8F0100C58F0100CE
:106CB000D48F0100DD8F0100EB8F0100F98F0100FF
:106CC0000590010008B5FFF725FFFFF743FD0349D5
:106CD000034809F0CBF9C82008BD00BFFC870100BC
:106CE000BC03002070B594B003F082FA064609F0A8
:106CF000B9FF05462D4808F003FA002854D02C4B64
:106D00001C7864B2002C4FD123460122402104A8F4
:106D100003F0E8FA274904A80DF073FA264904A8FD
:106D20000DF06FFA254904A80DF06BFA314668465C
:106D300003F05AFB01236A4604A91C4808F03DFCF5
:106D400023460122402104A803F0CCFA194904A8E3
:106D50000DF057FA184904A80DF053FA184904A881
:106D60000DF04FFA68464FF47A71B5FBF1F103F07C
:106D70003BFB01236A4604A90C4808F01EFC23468D
:106D80000122402104A803F0ADFA0E4904A80DF039
:106D900038FA0F220C4968460DF0ABFA01236A4617
:106DA00004A9024808F009FC14B070BDE8030020F3
:106DB000B803002049940100C18B0100AC9301008D
:106DC00061940100429401003C94010010B50C4C08
:106DD0002046F9F725FC78B90A490B4809F046F92D
:106DE000DE232374AD236374BE23A374EF23E37403
:106DF000FE232375FF236375BDE81040FFF7D2B96A
:106E000044040020E48A0100BC03002008B50020EF
:106E100007F0FEFF1C491D4809F028F91C491D48D0
:106E200007F084FF1C491D4807F080FF1C491D48DE
:106E300007F07CFF1C491D4807F078FF1C491D48DE
:106E400007F074FF1C491D4807F070FF1C491D48DE
:106E500007F06CFF1C491D4807F068FF1C491D48DE
:106E600007F064FF1C491D4807F060FF1C491D48DE
:106E700007F05CFF1C491D4807F058FF1C491D48DE
:106E8000BDE8084007F052BFAA8A01007003002045
:106E9000C56C0000AE8A0100FD5C0000B38A0100F1
:106EA000BD590000B88A0100A95B0000C29401002E
:106EB00019620000BD8A0100AD5A0000C18A0100BC
:106EC000815B0000C48A0100E9590000CB8A0100FF
:106ED0005D5C0000C78A0100655D0000D08A01008A
:106EE000CD590000D68A01002D5A0000BC86010051
:106EF000155A0000DD8A01002DE9F04F424E33683B
:106F000087B08046002B7CD0404D2C7864B2002C9A
:106F100077D12B783E4FDFF8089101335BB22B70AD
:106F20003B7801335BB23B70D9F800A009F09AFEC0
:106F3000234601460B22504603F06CFA002858D035
:106F4000B8F1030F0BD0334BD3F800A009F08AFE41
:106F5000234601466422504603F05CFA0446336837
:106F6000DFF8C0B0DE68AEB3337C03F00F03062B4E
:106F70002ED1314600226846FAF77AF94146684632
:106F8000FBF700F91CB104216846FBF7FBF8224A25
:106F90003146584607F062FDD0B1037C03F00F0381
:106FA000052B15D1D0F80CA0BAF1000F10D0514626
:106FB000324603A8FAF75CF9414603A8FBF7E2F86A
:106FC0001CB1042103A8FBF7DDF8DAF804A0EBE715
:106FD0007668C8E7B8F1030F03D009F043FEC9F89B
:106FE00000001CB109F03EFE0A4B18600B48FBF78D
:106FF000F9F83B78013B5BB23B702B78013B5BB20D
:107000002B7007B0BDE8F08FD8030020D503002017
:107010006D030020EC040020807E01002C03002082
:107020008C040020780700200220FFF765BF0000D5
:1070300010B5094C237801335BB2237009F068FE68
:107040000320FFF759FF09F063FE07F0CFFE237816
:10705000013B5BB2237010BDB8030020F0B51E4E9B
:10706000336885B0002B34D01C4B1C7864B284BBD1
:107070001B4D2F6809F0F6FD2346014641F2883288
:10708000384603F0C7F920B3164A137801335BB2D0
:1070900013703368DC681646A4B1237C03F00F0339
:1070A000062B08D12146002201A8FAF7E1F80121B8
:1070B00001A8FBF767F809F02BFE0220FFF71CFF81
:1070C0006468E9E709F0CEFD28603378013B5BB2E4
:1070D000337005B0F0BD00BFD8030020D5030020F9
:1070E000980400206D03002030B51449144885B081
:1070F00008F0BCFF124808F0C9FF124B1968D9B15B
:10710000114CCD682278013252B2227085B12B7CAD
:1071100003F00F03062B07D10022294601A8FAF736
:10712000A7F801A8FAF7DCF809F0F2FD6D68EDE7C1
:107130002378013B5BB2237005B030BDC7850100E9
:10714000BC030020D80300206D0300202DE9F04F80
:10715000A74C20688FB0002800F04381A54F3B78F2
:10716000002B40F041813B78A349A448A44EA54D93
:1071700001335BB23B7008F079FFA04808F086FF4E
:10718000A14A2168A14807F069FCA14A3060216842
:107190009E4807F063FC9F4B9F4A186021689B48FC
:1071A00007F05CFC9D4B9E4A18602168974807F0E9
:1071B00055FCB14628609B4E002800F08180C368D2
:1071C000002B7DD01B7C03F00F03052B78D1964953
:1071D0008A4808F04BFF29688C4807F02BFC934B3A
:1071E000014618700A22854808F0C2FF834808F05B
:1071F0004DFF2B68DB683360FFF766F88C4A216827
:10720000824807F02BFC8B4B186070B18A4C2378B6
:107210005BB902F0AFFC003018BF0120207023786A
:107220001BB18649754808F021FF854A0023136089
:10723000D9F800309246002B00F0B380D3F80C80D0
:10724000DFF828B27F4DD9F80030002B00F0CE8057
:10725000B8F1000F00F0A28098F8102002F00F02A1
:10726000052AF2D14146694807F0E4FB0128EAD932
:10727000D9F80020414602A8FBF77CFA02A8FBF7E8
:10728000F7F9A8B102A8FBF79BF8064680B90146BA
:1072900002A8FBF7D3F8041E02A8BCBF6442012673
:1072A000FBF734F89DF81C20052A0BD0062A46D09F
:1072B00009F02EFD02A8D8F80480FBF71DF8C2E7FC
:1072C000306099E718B9022102A8FBF72DF84FF4B6
:1072D000807102A8FBF75AF8059B23B14FF40071A7
:1072E00002A8FBF753F820B203F0B8FA064660B1E3
:1072F0005549564808F0BAFE0A222146534808F07C
:107300001EFF524808F0C2FED2E70121204609F0D4
:1073100097FE3146204609F0BBFE5946284608F044
:10732000A5FE21460A22284608F009FF48492846BA
:1073300008F09CFE4749284608F098FEB8E70190FF
:107340000121204609F07CFE20B203F087FA019B60
:1073500020B10021204609F09BFEA9E7D6B113F128
:10736000FF3618BF01263146204609F091FE3A4902
:10737000284608F07BFE0A222146284608F0DFFE58
:107380003649284608F072FE0A223146284608F09F
:10739000D6FECFE7013B5E425E41E4E7DB68CAF818
:1073A000003028482E4C2F4D08F070FEFFF79CFE51
:1073B000FFF746FB01232C48237004F0DDFA20B1CF
:1073C000294804F09BFB04232B7095F90030072B10
:1073D00004BF04232B703B78013B5BB23B702078E9
:1073E000C0B20FB0BDE8F08F0020FAE7DB68FFDE27
:1073F000380400206D03002058860100BC030020E3
:10740000DC03002068030020688601007807002064
:10741000CE900100A0040020407E0100D80300208F
:107420006E860100E40300207386010064030020DF
:10743000878601002C040020300400208A86010089
:1074400034040020700300209A8601008C03002081
:10745000B2860100B7860100588201000F7F01004B
:107460006C030020E0030020A4030020AA86010092
:1074700070B5444C237888B0002B7FD123784249E3
:107480004248434E01335BB2237008F0EFFD3F48A2
:1074900008F0FCFD722201213D48F9F739FE3C4815
:1074A000F9F7B8FD7B2849D13A493B483B4D08F0F4
:1074B000DDFD394808F0EAFD2B6813B10120FEF725
:1074C0006FFC00230593364B049304A94FF0FF3360
:1074D00034480793069607F0D3F928602C48F9F74B
:1074E000C3FD2D68BDB93049304808F0BFFD2F48B5
:1074F00008F0CCFD2E4901A809F08EFA01A92D480B
:10750000F9F73CFC01A809F042FA2378013B5BB291
:107510002370002010E028491C4808F0A7FD1B48F4
:1075200008F0B4FD2378013B5BB22370FFF70EFE39
:107530002048F9F7E9FC012008B070BD3046F9F7A2
:107540004CFD80B13046F9F783FD194904A809F0D4
:1075500063FA04A91748F9F711FC04A809F017FA0F
:107560001448F9F78FFC0A48F9F77EFD13490748DC
:1075700008F07CFD054808F089FDC6E74FF0FF30B4
:10758000DAE700BF6D030020EB8C0100BC03002094
:107590005C040020068D01007003002038040020E8
:1075A000509C010078070020148D01008C030020FE
:1075B000729C010044040020208D0100338D0100E5
:1075C0002DE9F041C0B000211C2214A813910BF04A
:1075D000BCFE202213A9A248F9F7F4F878B92022BA
:1075E000A04913A80CF085FE9F49A04808F03EFD75
:1075F00013A99E4808F043FD9C4808F047FD984DAC
:107600006A7D2B7C04922A7D0392EA7C0292AA7CFA
:1076100001926A7C00924021954A1BA80CF030FD33
:107620009449924808F022FD13A9904808F027FDDC
:107630001BA98E4808F023FD8C4808F027FD4FF465
:107640007A730022CDE90F238B4A0E922BAC0822CD
:107650008DF84820ADF84A3013AA50230EA92046D1
:1076600006F05EFA4FF47A63844985483B9308F04C
:10767000FDFC02F0BDFD0A220146814808F06BFDC9
:107680007F4808F003FD204606F079FA1BA9204642
:1076900006F09CFB7B4906460AA809F0BDF929467D
:1076A00007A8F9F727FB079A0A99204606F06CFA13
:1076B00007A809F06CF90AA809F069F9204606F054
:1076C00082FB002E40F0C580204606F08DFBDFF8DF
:1076D000FC810646204606F0F9FC074600B3214629
:1076E00007A806F0F7FB41460AA809F095F90AA990
:1076F00007A809F03AFA07460AA809F048F907A8C6
:1077000009F045F9002FE5D021460AA806F0FCFB58
:107710000AA92846F9F732FB0AA809F038F9D9E78F
:107720005949524808F0A2FC0A2231464F4808F055
:1077300006FD4E4808F0AAFCC82E7ED1534B544992
:107740000A934F480B974FF0FF330D930C9408F0BA
:107750008DFC02F04DFD0A220146494808F0FBFC71
:10776000474808F093FC3846FEF71AFBA0B9494990
:10777000494808F07BFC484808F088FC204606F0A1
:10778000F3F94FF4FA76454B2B933DA809F0FFF837
:10779000304640B0BDE8F08141493948414D08F0DC
:1077A00065FC374808F072FC3949354808F05EFC42
:1077B00002F01EFD0A220146314808F0CCFC304898
:1077C00008F064FC0AA9384807F05AF828602046F7
:1077D00006F0CAF92C6884B934492F4808F046FCF1
:1077E000334907A809F018F907A91D48F9F7C6FA9F
:1077F00007A809F0CCF82646C5E72E49204808F02E
:1078000035FC02F0F5FC0A2201461D4808F0A3FCF5
:107810001B4808F03BFCFFF799FC2749134808F088
:1078200025FC264B1B78002BADD00D48F9F7D9F974
:107830000028A8D0FEF726FAA5E7B6F5987F0CBF7A
:107840001F492049144808F011FC204606F08CF925
:1078500099E71D49104808F009FC4FF0FF3692E700
:1078600044040020D1930100628B0100BC0300207E
:10787000808B0100AF8B0100B09A0100C38B010027
:1078800070030020D98B0100EC8B0100509C01009B
:10789000408C0100FF8B01008C030020BC9B010089
:1078A0000B8C01003804002078070020218C010097
:1078B000729C0100388C0100468C01006C03002092
:1078C0004D8C0100618C01007B8C0100E78B010075
:1078D0002DE9F0433C4C23688DB0002B70D03B4D1C
:1078E0002E6809F0BFF9002301464FF47A72304642
:1078F00002F090FD074610B109F0B4F92860344D4C
:10790000DFF8D8902B7801335BB22B702368DE68E8
:107910007BB2002B14BF4FF004084FF0020822681E
:10792000FAB1F6B1337C03F00F03052BF8D13146E1
:10793000484607F07FF80128F1D9226831466846A9
:10794000FAF718FF6846FAF793FE18B14146684601
:10795000FCF774FD09F0DCF968467668FAF7CCFCB0
:10796000DDE72B78013B5BB22B701A4B93F90030AB
:10797000052B25D027B3184F00263D463968F9B1AD
:10798000F6B90B7C03F00F03052B0DD12268684676
:10799000FAF7F0FE01216846FCF750FD061C684628
:1079A00018BF0126FAF7A8FC2B684BB109F0B0F913
:1079B0002B685B682B60002BE0D12368DB682B60B1
:1079C0000DB0BDE8F08300BFDC030020940400206C
:1079D0006D030020E003002034040020780700201D
:1079E000F8B580EAE074A4EBE074054620B20E46D8
:1079F00002F034FF074668B11549164808F036FB17
:107A00000A222146134808F09AFB1248BDE8F840C4
:107A100008F03CBB0121204609F012FB022E09D1DF
:107A20003946204609F034FB0B490C4808F01EFB90
:107A30000A48EBE736B9E943C90F204609F028FBAD
:107A40000749F2E7E90F204609F022FB0549ECE778
:107A5000E88601008C030020F686010070030020F8
:107A600047950100589501002DE9F04F2DED028B4F
:107A7000874C95B0256809F0F5F80023014647F2D8
:107A80003052284602F0C6FC002800F0FC8009F0C5
:107A9000E9F82060FFF726F97E497F487F4C804D4A
:107AA00008F0E4FA02F0A4FB0A2201467A4808F042
:107AB00052FB7C49784808F0D9FA217876480A22A6
:107AC00049B208F03CFB7849734808F0CFFA774B8D
:107AD000714819680A2208F03EFB6F4808F0D6FA90
:107AE0002A68002A00F0CF802378DFF8F89101336C
:107AF0005BB22370D468002C00F0C080237C03F0BC
:107B00000F03052B13D100222146484606F09CFFA7
:107B10004369052B0BD12A68214608A8FAF72AFEEB
:107B200008A8FAF7A5FD20B908A8FAF7E5FB6468EC
:107B3000E1E708A906A8FDF7BAF908A8FAF752FD87
:107B40000021074608A8FAF779FC064606A8FCF7C4
:107B500065FF08EE900A08A8FAF7D8FB3BB207EEDB
:107B6000903A9FED537AF8EEE77A834687EE878A5C
:107B700008A8FCF755FB4F498246474808F076FABB
:107B80004FF0020818EE900A0AF098FDCDF8008038
:107B900002460B46CDE904013F4808F0A5FB4649E3
:107BA0003D4808F063FA18EE100A0AF087FDCDF898
:107BB000008002460B46CDE90201374808F094FBED
:107BC0003E49354808F052FA59460A22324808F030
:107BD000B6FA5FEA174B4CD0082002F023FE4FF6AE
:107BE000FF7381B240F62712584602F013FCA8B189
:107BF0002168334808F043FA3249314808F036FA30
:107C000022683149314807F0C3FCB9B208A8FAF735
:107C100001FD41463046FFF7E3FE85E7DFED2C7AB4
:107C2000B4EEE78AF1EE10FA04DD2268294927480C
:107C300007F0AEFCBAF1000F01D10121EAE7002202
:107C4000254BDDE904010AF0D9FBDDE902230BF045
:107C50001DF808B10021DDE7F4EEC88AF1EE10FA54
:107C6000EBD91E490C4808F001FA0B4808F00EFA4F
:107C70005AE71B49084808F0F9F955E7074A13780D
:107C8000013B5BB2137015B0BDEC028BBDE8F08F09
:107C90009C040020F2800100700300206D0300208E
:107CA000DC030020048601000C860100840400200F
:107CB0000000C842148601001A8601007D8101007F
:107CC0008C0300202086010030860100E80300209C
:107CD000000018423C8601000000F03F4986010088
:107CE00026860100780700202DE9F3470024344D53
:107CF00000942246214623463248334FDFF808A13C
:107D000008F06CF928464FF47A76304B6C60AE6020
:107D100040F8143B4FF0080808F058F985F8208027
:107D200029462B4D0122384608F086F84FF001090C
:107D300000943B4629460722264802F0A1F83B461C
:107D40002946CDF800900322234802F099F80094C8
:107D50003B460622214F22482946224D02F090F848
:107D60004FF48053C5E901462B612C751E4BEC8204
:107D70001E492B60381DC5E9064485F8204008F0EF
:107D80004BFE3D601A4D1B495246384609F040FAF9
:107D9000C5E90146184C194B19482B60494685F82E
:107DA00010806E8202F020F82946204607F034FD4C
:107DB00014495246204602B0BDE8F04709F028BAFF
:107DC000C80400204C030020A40400200C9B0100E8
:107DD000E0070020700300208C03002044040020F2
:107DE000BC0300205C040020507E0100729C010056
:107DF000A40300201F5A0000E8030020B09A0100ED
:107E00003C0400206DEE0000000000202DE9F0474A
:107E10000024C8B03C22214609A808940BF095FA2A
:107E20007C22214629A828940BF08FFA23460122B0
:107E3000402108A802F056FAAF49B04EB04F08A84A
:107E40000CF0DFF97F22AF4928A80CF052FA012389
:107E500028AA08A9AC4807F0B0FB2346012240211C
:107E600008A802F03FFAA94908A80CF0CAF97F2235
:107E7000A74928A80CF03DFAA64928A80CF0C1F99A
:107E8000012328AA08A9A04807F097FB234601224E
:107E9000402108A802F026FA9F4908A80CF0B1F981
:107EA0007F229E4928A80CF024FA012328AA08A9B9
:107EB000954807F082FB23460122402108A802F0E2
:107EC00011FA974908A80CF09CF97F22954928A837
:107ED0000CF00FFA012328AA08A98B4807F06DFBC4
:107EE00033783D6801335BB23370002D00F03B8185
:107EF0008D4BDFF86092B3F80080ADF800801E2251
:107F000021460DF102000BF020FA3E2221460DF130
:107F10006200ADF86080DFF840A2DFF840820BF02D
:107F200014FAED683B68002B00F0AE80002D00F0E5
:107F3000AB802B7C03F00F03052B40F08E8029468D
:107F4000404606F077FD002800F0878028680CF096
:107F5000A2F90134044400222946404606F074FD8B
:107F60004369112B12D8DFE803F07C87877C7C09FA
:107F70007C7C7C7C11111111111111871F226B491E
:107F800068460CF0B6F900238DF86030002301221A
:107F9000402108A802F0A6F93F22296808A80CF0A1
:107FA00082F9494608A80CF02CF9514608A80CF0B3
:107FB00028F901235E4A544808A907F063FB00230F
:107FC0000122402108A802F08DF93F22296808A863
:107FD0000CF069F9494608A80CF013F9554908A8AE
:107FE0000CF00FF90123544A474808A907F04AFB4F
:107FF00000230122402108A802F074F93F222968D9
:1080000008A80CF050F94D4908A80CF0FAF85146B0
:1080100008A80CF0F6F801236A4608A93A4807F0C8
:10802000CCFA9DF86030C3B100230122402108A89A
:1080300002F058F93F22296808A80CF034F93F49AA
:1080400008A80CF0DEF83B4908A80CF0DAF8012388
:1080500018AA08A92C4807F0B0FA08F059FE6D6874
:1080600060E71F22364968460CF043F935493F2244
:1080700018A80CF03EF989E71F22334968460CF036
:1080800038F93F223149F3E700230122402108A8B3
:1080900002F028F92E49DFF8C4901B4D08A80CF017
:1080A000B0F80123621E08A9174807F000FB3B68DF
:1080B000DC683B68002B53D0002C51D0237C03F0AC
:1080C0000F03052B14D12146484606F0B3FC78B1C6
:1080D000D4F8008040460CF0DEF8414602462846BF
:1080E00006F0B5FE63681BB12C21284606F0A2FEFF
:1080F00008F00EFE6468DCE7429401006D03002086
:10810000DC0300203C940100E80300201C940100E3
:108110007B9401006894010049940100BB93010025
:108120002E940100B5930100A78501002894010059
:108130001794010050940100DD930100798701003C
:108140000F940100CB930100229401000B940100D5
:108150003594010073870100A29301007807002085
:10816000044806F05CFF3378013B5BB2337048B0E3
:10817000BDE8F087E803002030B59F4C94F900304B
:10818000113393B0242B35D8DFE813F0A301940109
:1081900034003400340034000301F30034003400B0
:1081A000340034003400340034003400340025003E
:1081B000510054006400A100BE00E300340034000C
:1081C000340034003400130120016F012F0134000A
:1081D000340034006001894B89481B78002B14BFA0
:1081E0000921012101F001FE03F0D4FA022801D097
:1081F000FEF704FB94F90030012B40F38481814B9E
:108200001B78002B40F0748103F0CEFA054603F092
:10821000C1FA022800F06E81013D042D00F2738145
:10822000DFE815F0750177018501870168010223F8
:108230002370DFE7744D2B7853B9FEF745F8734987
:10824000734807F013FF724807F020FF01232B70DB
:108250000323EDE7694D6A482B78002B14BF0B21EF
:10826000032101F0C2FD6B4B1B78002B40F06381B2
:108270006948F8F7F0FCE0B1684B1B78BBB9FFF731
:108280009FF9C82808D02B7843B16549654807F0A5
:10829000EDFE644807F0FAFE0423C9E701A803F0E5
:1082A000C7FA029B002B00F0DE800F23C0E75E4977
:1082B000ECE72B784BB104235C495A48237007F054
:1082C000D5FE584807F0E2FE94E70F23F4E74B4B46
:1082D0004B481B78002B14BF0B21032101F085FDB7
:1082E000534B196841B953494E4807F0BFFE4D48FA
:1082F00007F0CCFE07239BE74F4806F09BFB0128C5
:10830000F1D9FEF7B9F875E74C4B1D6808F0AAFCE7
:10831000002301464FF4FA52284602F07BF8002869
:108320003FF468AF00230322412101A801F0DAFFE6
:10833000434901A80BF065FF01A9424807F01DFA67
:10834000FFF764FD062340493648237007F08EFE90
:1083500050E72A4B2A481B78002B14BF0A21022120
:1083600001F043FD374806F0CBFE00287FF442AF12
:1083700092E708F077FC314B1860F52323701F4B10
:108380001F481B78002B14BF0921012101F02DFD8E
:1083900030E72A4B1D6808F065FC0023014641F2D6
:1083A0008832284602F036F800283FF423AF002335
:1083B0003EE7244806F0A4FE10B1224806F06DFE08
:1083C00008F050FC1D4B18600D2331E71B4B1D6856
:1083D00008F048FC0023014642F21072284602F0E1
:1083E00019F800287FF458AF04E708F03BFC134B62
:1083F00018600E231CE700BFE00300206C03002080
:108400003C04002048030020D4030020FF9001001A
:10841000700300206D030020440400206E03002040
:1084200009910100BC03002030910100409101003E
:10843000E40300207A9101007807002090040020D6
:10844000AC900100E80300208D9101003C4B1D68B9
:1084500008F008FC002301463A4A284601F0DAFFFA
:1084600000283FF4C7AEF623E2E6FFF701F8D0B1EB
:1084700001283FF411AF01307FF4BCAE304B1D68D2
:1084800008F0F0FB0023014647F23052284601F085
:10849000C1FF00283FF4AEAE2B492C4807F0E6FDA3
:1084A00001F0A8FFA6E61323237008F0DBFB244BA2
:1084B00018609FE6264806F023FE10B1244806F017
:1084C000ECFDFDF79BFF08F0CDFB1D4B1860EF2383
:1084D000AEE6204D20482B78002B14BF0B21032142
:1084E00001F083FC1D4B1B783BBB12232370C6E6B7
:1084F00000258CE61A49154807F0B8FD134807F027
:10850000C5FDF623237094F9000013B030BD154962
:10851000F1E71549154807F0A9FD01A803F088F90E
:1085200001A801F0B9FE114807F0B0FDEBE71049D2
:10853000E1E71049EEE70320E7E76FF01000E4E71A
:1085400090040020C0D40100AA9101008C030020F7
:10855000E80300206C0300203C0400206D03002091
:10856000CD910100D6910100EA910100BC030020E9
:10857000079201001A92010008B5184801F037FC73
:1085800008F0C6FB06F032FCFFF7F6FD022802DD1C
:10859000134806F0DDFE08F0BBFB124B1B7823B13D
:1085A000114B1B680BB101F0FBFB104B1B6843B177
:1085B0000F4B93F90030052B01D0FFF789F908F034
:1085C000A7FBFFF751FA08F0A3FB0220FEF794FC8B
:1085D00008F09EFBBDE80840FEF740BD3C040020CB
:1085E000E8030020300400202C040020DC030020DD
:1085F000E003002010B54FF4E1311B4808F04EF8BD
:108600001A48F7F7E5FF044630BB1949164807F04A
:1086100043FD21462046FDF7A5FB1448F8F75AFB19
:10862000144B18701148F8F75DFB134B1870FEF7E8
:10863000EDFBFEF76FFAFEF7C9FB142008F046FBCE
:108640000E490F4807F0CBF84FF4FA7008F03EFBE4
:10865000BDE81040FEF70CBF0A490B4807F006FDC5
:10866000094807F013FDD8E7E00700204404002084
:10867000DB8501000500002006000020715F00007E
:10868000E8030020F08501007003002007B50023F7
:1086900000931A461946034807F0A0FC03B05DF8A2
:1086A00004FB00BFF0040020032070477047000067
:1086B00073B56E460546304686E80600FCF7AAFB11
:1086C00004463046FCF73FF910B1002C08BF0124E6
:1086D0004FF480416868F9F759FE012C1BD0022C39
:1086E00004D0FCB91C491D4807F0C0FC3046FCF71B
:1086F00039F970B36868F9F775FF18B90124204695
:1087000002B070BD00206C6802F08CF80146204673
:10871000F9F780FFF2E73046FCF7C4FA01280AD0E7
:10872000022808D00E490D4807F0A0FC0B4807F0BE
:10873000ADFC0024E3E76868F9F754FF0028DDD0BA
:1087400000206D6802F06EF801462846F9F762FFD6
:10875000D5E70446D3E700BF8594010070030020ED
:108760009D94010010B5044608F014FB204610BD8E
:1087700010B504461649174807F098FC00216068B8
:10878000F9F748FF236820469B690021984794F930
:10879000080002F063F840B10F49104807F066FC8A
:1087A0000E4807F073FC002010BD94F9090002F098
:1087B00055F80028F0D1A17C94F9080008F068FC75
:1087C00094F90900A17C08F063FC0120ECE700BFEC
:1087D000C694010070030020D59401008C03002092
:1087E00001292DE9FF41044600F089804FF48041C2
:1087F0004068F9F7B3FD002800F081804FF4004194
:108800006068F9F7ABFD60B9764D95F90030002B43
:1088100075D04FF400416068F9F7B8FD2B78013B43
:108820002B7094F9080002F019F8002867D194F928
:10883000090002F013F80546002860D16068F9F7D6
:10884000D1FE2A462946074602A8FBF7F7FE4FF459
:108850000072616802A8FCF7E6FA294602A8FCF754
:10886000B5F906466068F9F751FD022801D00528E0
:1088700000D1002694F90A00A0F10E03DBB2072B09
:1088800000F29C804FF0FF0808F0E4FAE289218AA8
:10889000CDF80080002308F070F8051EC0F28A8031
:1088A000454500F38980002F40F08B80751B15F142
:1088B0000A0F55DA94F90900A17C08F0E9FB606819
:1088C000F9F790FE30B9666801F0ACFF014630461A
:1088D000F9F7A0FEA37C6842002B3CD00021009158
:1088E000FF23192208F049F8FF280146A8BFFF21FD
:1088F000462994F90800B8BF462108F04FFB002034
:1089000004B0BDE8F0813849384807F0AFFB37487C
:1089100007F0BCFB3649354807F0C8FBA17C94F949
:10892000080008F0B5FBA17C94F9090008F0B0FB41
:1089300000216068F9F76EFE4FF480416068F9F736
:1089400065FD4FF400416068F9F760FD254A137832
:1089500001331370D3E7FF22009219461922C1E7B1
:108960000A2DD7DD94F90800A17C08F091FB60681E
:10897000F9F738FE30B9666801F054FF0146304619
:10898000F9F748FEA37C83B100210091FF23332235
:10899000284607F0F2FFFF280146A8BFFF2146291D
:1089A000B8BF462194F90900A7E7FF2200921946B3
:1089B0003322EDE7002576E7454674E77FB14FF0B7
:1089C000FF3508F04FF900230146B4F90C20384672
:1089D00001F020FD002896D16B1C7FF467AFA6F153
:1089E0007F0564E704000020A994010070030020C3
:1089F000B8940100002110B5044681744068F9F76D
:108A00001DFD43B2002BBBBF4042207223720123E5
:108A1000B8BFA374237A6068013B182B84BF20235E
:108A200023720121F9F70AFD43B2002BBBBF40427C
:108A3000607263720123B8BFA374637A6068013BFC
:108A4000182B84BF212363720221F9F7F7FCC3B20C
:108A5000192B8ABF0023A072A37203216068F9F763
:108A6000EDFC80B2431EB3F5806F26BF0023E38187
:108A7000E08104216068F9F7E1FC80B2B0F5806F15
:108A80008ABF4FF480632082238205216068F9F752
:108A9000D5FC00B20028D6BF42F21073A081A3819A
:108AA00010BD000038B50446F7F79FFC2046FFF7DD
:108AB000A1FF2549254807F0F9FA94F9080001F0CB
:108AC000CDFE40B12249234807F0D0FA214807F0F3
:108AD000DDFA002038BD94F9090001F0BFFE05461B
:108AE0000028EFD1012194F9080008F0A9FA01212A
:108AF00094F9090008F0A4FAA17C94F9080008F0A0
:108B0000C7FAA17C94F9090008F0C2FA294694F941
:108B10000A0008F095FA29466068F9F77BFD4FF4E2
:108B200080416068F9F772FC4FF400416068F9F722
:108B30006DFC236820469B6902219847064B022260
:108B40001A700120C6E700BFE29401007003002004
:108B5000D59401008C0300200400002007B50023F9
:108B600000931A461946034807F038FA03B05DF837
:108B700004FB00BFF804002000207047032070476A
:108B8000704700002DE9F0410646F7F72EFCB46867
:108B9000002C41D0E468254F254DDFF8A88064B350
:108BA000236843B31B7833B33A462146284605F081
:108BB00055FF30B94FF0FF333A462146284605F0BD
:108BC00095FF42462146284605F048FF30B94FF050
:108BD000FF3342462146284605F088FF154A2146C4
:108BE000284605F03BFF30B94FF0FF33114A2146CC
:108BF000284605F07BFF6468D1E70F490F4807F06E
:108C000035FA0E4807F042FA336830469B69022174
:108C100098470120BDE8F0810949084807F026FA85
:108C2000064807F033FA2046F4E700BFEC9801004D
:108C300078070020B4940100B4950100700300206F
:108C4000BF950100A594010038B5084D08490446B8
:108C5000284607F00BFA284607F018FA2368204642
:108C60009B6900219847012038BD00BF7003002098
:108C7000A69501002DE9F04F93B00AAC804620463E
:108C800084E806000893FCF70DF80B2800F04482F6
:108C90002046FCF707F80A2800F03E822046FCF741
:108CA000B9F882462046FBF74EFE20B1BAF1000F1C
:108CB00008BF4FF0010A2046FBF745FE90B1204661
:108CC000FCF7A8F807280DD12046FBF7EBFF112889
:108CD00068D0122868D0102804D1FF22214610A89D
:108CE000FBF7F0FFD8F80830002B00F015820027C2
:108CF000CDE90477DC68B946BB46002C00F0DE8085
:108D0000AF4AB048214605F0A9FEAF4A21460546C4
:108D1000AC4805F0A3FEAD4A06462146A94805F039
:108D20009DFE0790002D00F08B80002E00F08880C3
:108D30002B7C03F00F03022B40F08280337C03F086
:108D40000F03022B7CD1A24A9E48214605F086FEE5
:108D500043690693089B002B5FD0194620680BF0EF
:108D60006CFA002859D10AA8FBF7EDFD08BBBAF14F
:108D7000070F6FD00AAA10460992FBF7F3FD099A74
:108D800000283DD0104600210992FBF71FFF6861C3
:108D9000FDF7CCF8099A002832D0236800934FF4ED
:108DA000007328E0802299E70A212046FBF7D0FED5
:108DB00098E70AA8FBF776FF70610AA8FBF772FF35
:108DC00001283FD0022843D0FDF7B0F858B17369AD
:108DD000012B08D16B69132B05DC1E226A610AA9DD
:108DE00010A8FBF76FFFFDF7A1F848B123680093C7
:108DF0000AAA4FF4407306CAD8F80400F9F796FEA1
:108E0000079B53B10023CDE9013300930AAB0CCB90
:108E10004FF0FF31079801F017FB7369022B0DD05B
:108E200001330BD06B69069ABB4202FB03F2C2BF4F
:108E30001F46069B04929344C8BF0593069B994422
:108E400064685AE76A690AA910A8FBF73BFFBBE709
:108E50000022F8E70AA8FBF785FD00288AD00AA8B7
:108E6000FBF7BAFD7369A8B1022B01D001330CD115
:108E70005849594807F003F9574807F007F9012204
:108E800072610AA910A8FBF7BEFF0AA8FBF7A4FDB0
:108E90006861A8E7022B0ED001330CD04F494E4831
:108EA00007F0EDF84C4807F0F1F8022272610AA9C8
:108EB00010A8FBF7A8FF00236B6194E7B9F1000F3E
:108EC00000F02A81464944489BFBF9F507F0CEF8AB
:108ED0000A224946404807F032F942493E4807F025
:108EE000C5F8FF260A229BFBF6F13B4807F027F95D
:108EF0003D49394807F0BAF80A222946364807F0B2
:108F00001EF93A49344807F0B1F8049B324893FB04
:108F1000F6F10A2207F013F935492F4807F0A6F8B1
:108F20000A2205992C4807F00AF932492A4807F025
:108F30009DF8294807F0AAF810AE0EAF2E4AD8F8CF
:108F4000081020481DB305F089FD224681462146C0
:108F50003846FBF773FB2A46394630460CADFBF723
:108F6000B1FE012231462846FBF74DFFCDE9014411
:108F7000009495E80C004FF0FF31484601F064FA88
:108F8000D8F80830D3BB012013B0BDE8F08F05F04E
:108F900065FD2246054621463046FBF74FFB22463B
:108FA00031463846FBF78EFECDE90144009497E840
:108FB0000C004FF0FF31284601F046FAE3E700BF0E
:108FC000EC98010078070020A59401003495010079
:108FD000389501003A950100700300204B9501007F
:108FE0005D9501006C950100779501007E9501006B
:108FF000889501008F950100729C0100DD68DFF803
:109000003881DFF838B1002DBDD0444A29464046AA
:1090100005F024FD5A4644692946404605F01EFDE8
:109020003F4A81462946404605F018FD3D4A8246A2
:109030002946404605F012FDB9F1000F66D0BAF19D
:10904000000F63D0002861D099F8102002F00F02C1
:10905000022A5BD19AF8102002F00F02022A55D1A1
:10906000027C02F00F02022A50D1002C4ED042693D
:10907000022A4DD001324BD0049B002B4AD0DAF8A3
:1090800014302949294803FB04FA059BCAEB0A223C
:1090900092FBF4F45C43049B94FBF3F406F0E6FFCC
:1090A0002968224806F0EBFF2149204806F0DEFF40
:1090B0000A22FF211D489AFBF1F107F040F81D49F3
:1090C0001A4806F0D3FF0A222146184807F015F87F
:1090D000164806F0DBFFD9F81430A34216D0002260
:1090E00011463846FBF7AAFA224639463046FBF7C6
:1090F000E9FD0023CDE90133009396E80C004FF021
:10910000FF31284601F0A0F9C9F814406D687AE7EC
:109110000024E0E7049CDEE7002035E738950100F5
:10912000EC980100A59401009395010070030020C4
:109130009A950100A095010078070020B4940100E1
:1091400010B5044607F026FE204610BD00238360BC
:1091500043683BB19B682BB11A7C02F00F02062AD0
:1091600008BF83607047000007B5002300931A46CC
:109170001946034806F032FF03B05DF804FB00BF58
:109180000005002043687BB1B0F90A20042A05D00D
:10919000052A05D0032A05D1022070470120704717
:1091A00011207047187D70471846704770470000BF
:1091B00038B50446F7F719F92849294806F056FF4B
:1091C0000A22B4F90810264806F0B9FF25492448B8
:1091D00006F04CFF636822485B68196806F04FFF91
:1091E00021491F4806F042FF1D4806F04FFF606806
:1091F00088B3B4F908307BBB236820469B6B984743
:109200000128054605D002280AD00121B4F908003A
:1092100019E003212046F7F7B5F9294607F010FFBA
:1092200000212046F7F7AEF9012107F009FF0121DF
:109230002046F7F7A7F9012107F002FF0221204697
:10924000F7F7A0F9012107F0FBFE236820469B6990
:1092500002219847012038BD0020FCE71896010044
:1092600070030020247F0100B995010010B5044669
:109270002449254806F0FAFE0A22B4F908102248CB
:1092800006F05DFF2149204806F0F0FE63681E48A5
:109290005B68196806F0F3FE1D491B4806F0E6FE00
:1092A000194806F0F3FE236820469B6B9847012877
:1092B00005D002280AD00021B4F9080019E00321E2
:1092C0002046F7F75FF9002107F0BAFE002120469B
:1092D000F7F758F9002107F0B3FE01212046F7F710
:1092E00051F9002107F0ACFE02212046F7F74AF9B8
:1092F000002107F0A5FE236820469B6900219847BE
:10930000012010BD1896010070030020247F010089
:109310006D9201002DE9F041044688B040689DF847
:1093200038309DF83C5002AF87E80600002800F076
:10933000A780B4F90820002A00F0A180002B00F0DB
:10934000A2800021F9F77AF8236880469B6B2046BB
:10935000984706B2022E19D0032E19D0012E0CBF49
:1093600005210121002204A8FBF768F94FF0FF3323
:10937000009397E80C0004A906A8FBF7BFFF012E95
:1093800041D0022E27D1002D52D14CE00421E9E733
:109390001DB34FEAD8713846B4F90860FBF716FCE4
:1093A00001460546304607F0F9FD3849384806F0D1
:1093B0005DFE0A22B4F90810354806F0C0FE3549B2
:1093C000334806F053FE0A222946314806F0B7FE1C
:1093D0002F4806F05BFE012052E0B4F9080001F0CE
:1093E0003DFA0028D5D029492B4806F03FFE0A2235
:1093F000B4F90810284806F0A2FE2849264806F0CD
:1094000035FE2548E5E703212046F7F7BBF8064679
:109410002DB19DF81710304607F0C0FDB3E701F0FD
:109420001DFA0028F5D0B4F9080001F017FA28B9A0
:109430009DF81610B4F9080007F0B0FD0121204690
:10944000F7F7A0F8064685B19DF81510304607F0ED
:10945000A5FD20460221F7F795F8044655B19DF881
:109460001410204607F09AFDB5E701F0F7F900283F
:10947000EAD0EEE701F0F2F90028F0D0ABE71046B1
:1094800008B0BDE8F0811846FAE700BF5882010035
:10949000700300200F7F01008C0300202296010042
:1094A00010B5044607F076FC204610BD07B5002332
:1094B00000931A461946034806F090FD03B05DF884
:1094C00004FB00BF08050020032070477047000020
:1094D00038B50446F6F789FF2249234806F0C6FD51
:1094E0000A22B4F90810204806F029FE1F491E4838
:1094F00006F0BCFD1C4806F0C9FDB4F9080001F0F7
:10950000ADF9054640B11A491A4806F0AFFD1948B1
:1095100006F0BCFD002038BD0121B4F9080007F0B9
:109520008FFDB4F90800A17A07F0B2FD606810B1B0
:109530002946F9F76FF8236820469B69022198476E
:10954000606808B90120E6E7FAF76AFE0028F9DD4D
:109550000020646801F066F901462046F9F75AF8E0
:10956000F0E700BFAE96010070030020B99501003E
:10957000D59401008C03002038B50F4D0F490446E7
:10958000284606F073FD0A22B4F90810284606F0B2
:10959000D6FD0B49284606F069FD284606F076FD03
:1095A000B4F90800002107F04BFD236820469B69B1
:1095B00000219847012038BD70030020AE960100BD
:1095C0006D92010010B5044607F0E4FB204610BD83
:1095D000002110B5044681724068F0B1F8F72EFF03
:1095E00003B2002BBBBF4042208123810123B8BFBF
:1095F000A37223896068013B182B84BF2023238139
:109600000121F8F73BFF09F059F80022054B09F05A
:10961000ADF809F083FB08B1E06010BD41F288337A
:10962000E360FAE700408F4030B5044687B000237E
:109630002F22CDE90023ADF80830B0F90800A37A55
:109640000D4671B383F0010107F022FDE368B3F525
:109650007A7F57D33149324806F008FD0A22B4F91F
:1096600008102F4806F06BFD2E492D4806F0FEFC31
:109670000A2229462A4806F062FD294806F006FD1E
:10968000294968460AF0BDFD6068F8F73FFE002DE5
:109690003ED0142807D0152836D00F2836D12349BC
:1096A00002E01946D0E7224903A80AF0D0FD21497B
:1096B0001B4806F0DBFC63685968236809685D6A2B
:1096C00003AA6B462046A8470A220146144806F022
:1096D00036FD1949124806F0C9FC636810485B68FA
:1096E000196806F0CCFC69460D4806F0C8FC134921
:1096F0000B4806F0BBFC03A9094806F0C0FC08486B
:1097000006F0C4FC07B030BD0D49CDE70D49CBE7ED
:1097100002280CBF0C490D49C6E700BFBA960100EC
:1097200070030020158301008596010078960100E2
:1097300093960100BF9601008A800100CB9601003C
:109740008C9601009B9601007C960100809601009A
:109750000129F7B5044644D04368002B41D00022CC
:1097600011466846FAF76AFF4FF40072616868466E
:10977000FBF759FB00216846FBF728FA05466846C7
:10978000FBF790FA6068F8F72DFF064607F06AFAD3
:10979000E268FF216A430023B2FBF1F20146304642
:1097A00000F038FE0746E6B107F05CFA00230146F8
:1097B000E268304600F02EFE064620B300206668C0
:1097C00001F030F801463046F8F724FF4DB1207A19
:1097D00001F032F8A37A834203D101212046FFF73A
:1097E00023FF002003B0F0BD9FB131462046FFF7B4
:1097F0001BFF6068FAF714FD01460028F1D160688C
:10980000F8F708FFEDE7207A01F016F8A37A834213
:10981000EAD1002DE5D0207A01F00EF8A37A834238
:10982000DFD1002FDDD1D8E7F7B56E4686E8060018
:109830000446454945489DF820501F4606F016FC51
:109840003046FBF7DFFC37B1414938460AF0F5FCFA
:1098500008B9002051E06368002BFAD0B4F9080081
:1098600000F0FCFF0028F4D13046FBF76CF800282C
:1098700045D13046FBF7CEFA012840D010D302285C
:109880000DD004463349314806F0F0FB0A22214648
:109890002E4806F054FC2D4806F0F8FBD9E7D5B168
:1098A00000213046FBF792F9054658B16068F8F799
:1098B00099FE08BB646800F0B5FF01462046F8F742
:1098C000A9FE19E001466068F8F7A4FE2946204683
:1098D000FFF7AAFE10E06068F8F718FD15280BD80E
:1098E000012303FA00F01C4B184205D029463046EC
:1098F000FBF76CF90028D9D1012003B0F0BD304648
:10990000FBF7D0F915280DD80125144F05FA00F002
:109910000740CBD1430705D539466068F8F77AFE92
:109920003946D4E70E49094806F0A0FB3046FBF75C
:10993000B9F90A220146054806F01AFC034806F068
:10994000A5FB01249EE700BFA39601007003002041
:10995000859601009A7D01000240380002C038005F
:109960008D7D010007B5002300931A461946034870
:1099700006F034FB03B05DF804FB00BF10050020C7
:1099800090B1C3687BB11A7C02F00F02042A01D1A6
:10999000586948B9D86838B1037C03F00F03042B29
:1099A00001D14069704700207047000030B52DEDAF
:1099B000028B054689B008EE101A002852D0324BAF
:1099C0001B68002B4ED0FFF7DBFF304904463048C0
:1099D00006F04CFB18EE100A08F070FE0223024657
:1099E00000932B480B4606F07FFC2A49284806F0D6
:1099F0003DFB2968264806F042FB2749244806F02B
:109A000035FBDFED267AB4EE678AF1EE10FA2DD041
:109A1000DFED237AB4EE678AF1EE10FA26D0B5EEC8
:109A2000408AF1EE10FA21D01CB12146184806F008
:109A300026FB174806F02AFB06AC18EE101A04A8FD
:109A4000FAF709FE032204A92046FBF7E5F90023F3
:109A5000CDE90133009394E80C004FF0FF31284624
:109A600000F0F2FC09B0BDEC028B30BD002CF9D047
:109A70000C49074806F0FAFA2146054806F0FFFAB5
:109A8000034806F003FBEDE72C04002014970100C7
:109A900070030020B3980100A19801000000FEC2ED
:109AA0000000AA42199701002DE9F043284F3868B9
:109AB00089B0002846D0274E3368002B45D001F0EE
:109AC00077F925492548DFF8A080DFF8A090234CDE
:109AD00006F0CCFA214806F0D9FA01A9386801F05D
:109AE000F9FA00282DDD03AA082101A800F078FA70
:109AF000002303AA31688DF81C30404604F0AEFF05
:109B000049460546204606F0B1FA03A9204606F06C
:109B1000B6FA8DB12846FFF733FF05460028DCD0A2
:109B20000F49204606F0A2FA2946204606F0A7FA79
:109B3000204606F0ABFAD0E70A49204606F096FA2E
:109B4000F6E7012009B0BDE8F0831846FAE700BF48
:109B5000240500202C04002035980100BC030020BF
:109B60001583010048980100780700201497010030
:109B7000FFF79ABF2DE9F3413E4C2368002B77D1C4
:109B80003D493E4806F072FA3C4806F07FFA142040
:109B900007F0FEF8054601F0C5F83948256000F0E9
:109BA0001BFF206801F0D8F800284AD03549364814
:109BB00006F072FA206801F015FA206801F0D8F872
:109BC000206801F053FA002839D030492B4806F0BC
:109BD00063FA2F4E3068002847D02E4D2F687FB98A
:109BE0001C2007F0D5F82168804601F0F7FA4046BE
:109BF000C5F8008001F0D2FB3946286801F00CFC62
:109C00003368DFF8A480DC681C4F336883B37CB30F
:109C10006946206800F01CFA50B34146384606F009
:109C200025FA2168384606F02AFA384606F02EFA58
:109C30000C226946286801F06EFB6468E5E7164966
:109C4000C4E700F00DFE206801F086F8054638B143
:109C500012490D4806F00AFA0B4806F017FAB8E761
:109C60000F49104806F018FA284602B0BDE8F08106
:109C70000120FAE7240500207797010070030020F7
:109C80009C0500209D970100BC030020BC970100AB
:109C90002C0400202C050020D0970100E59701003E
:109CA000029801008C0300201E980100034B01461E
:109CB000186808B101F046B8704700BF24050020BD
:109CC00037B52D4C206801F03FF8022805D0042854
:109CD00011D0012818D129490EE02949294806F058
:109CE000C5F9284806F0D2F9206801F0BFF941F221
:109CF000883003B030BD2449224806F0B7F9214826
:109D000006F0C4F900F0ACFD204D2B6813B1204BD8
:109D10001B683BB91F491B4806F0A8F9194806F013
:109D2000B5F9E4E71C4C22683AB91A7C02F00F023C
:109D3000062A02D1DB6803B123601848FFF7B6FF9B
:109D40002368A3B16946186800F082F978B19DF8DC
:109D50000030282B0BD16946286801F0EDFB014645
:109D60002068FFF723FE6946286801F08BFB236813
:109D70005B682360BBE700BF240500205797010004
:109D80002A9701008C0300203E9701002C0500203B
:109D90002C04002069970100200500202970000094
:109DA00038B5094C256806F05DFF0023014641F2F5
:109DB0008832284600F02EFB20B1FFF781FF06F025
:109DC00051FF206038BD00BF2805002007B50023E3
:109DD00000931A461946034806F000F903B05DF8EF
:109DE00004FB00BF1805002070477047704770479C
:109DF00007B5002300931A461946034806F0EEF80B
:109E000003B05DF804FB00BF30050020174B1B7842
:109E100070B504460D469BB1154B027A1B789A42E9
:109E20000ED8144A0A291368164616D1124A002180
:109E3000D154406910B1217A06F096F800233360BE
:109E4000E06840B10D4B227A1B789A4203D8036830
:109E500029461B689847012070BD4E2BF0DC0D2968
:109E60001FBF591C1160044AD554E9E78004002043
:109E7000060000209005002040050020050000207D
:109E800030B5002545604361034D9DF80C300560F9
:109E9000C1600272037430BD5898010007B50023F9
:109EA00000931A461946034806F098F803B05DF887
:109EB00004FB00BF38050020D0E90423D05C7047C4
:109EC0000368DB681847704700207047184B70B56F
:109ED0000E461968044679B10B7C03F00F03062B7C
:109EE0000AD13246134804F0B9FD037C03F00F0396
:109EF000042B01D1406970BDB4F924506B1E9BB294
:109F00000C2B13D80C4930460AF097F970B90B495D
:109F10002F2305EB850584F826300622294404F119
:109F200027000AF0E6F904F12600E4E70020E2E762
:109F3000A0040020780700207C9901002F990100DF
:109F40002DE9F041056A044625B100230362284645
:109F5000BDE8F081D0E90432995C242934D1991804
:109F600049787B2930D1023213442E461A4613F821
:109F7000017B4FB37D2F0FD00136F7E7A261226935
:109F80003AB16369D25C12B10133636125E02261A9
:109F9000DDE74FF0FF35DAE7B6B14FF0000882F8A1
:109FA000008061692269236802319B69114420465F
:109FB0009847D4E9043233441344C4E906089F7037
:109FC000636903331E446661A269002AD7D0E3693E
:109FD000D25C002AD2D00133E3611546B7E7000016
:109FE00070B5D0B1CAB14D1E0C4E441E1346284464
:109FF000844203F102030CD014F8015F2D11755D4A
:10A0000003F8025C257805F00F05755D03F8015C27
:10A01000EEE709B2002302F8113070BD1599010076
:10A02000A0F16103052B02D85738C0B27047A0F1E8
:10A030004103052B01D83738F7E73038C0B209287B
:10A0400005D919B101230B700020704708467047ED
:10A0500037B500238DF80730F9B1E0B1851C4C1EEF
:10A0600000F1120215F8020C0DF10701FFF7D8FFFD
:10A07000000104F8010F0DF1070115F8010CFFF7BD
:10A08000CFFF23780235184395422070EAD19DF81E
:10A09000070080F0010003B030BD0846FBE738B58B
:10A0A0000546D8B10468ACB124789CB1286803781F
:10A0B0003BB12D2B05D0303B092B02D90130286054
:10A0C000F4E708F0C0FE2C21044628680AF0A8F83E
:10A0D00010B92860204638BD0130FAE70446F9E798
:10A0E0002DE9F7430E46002206210746FAF7A6FAA5
:10A0F000002E55D03368002B52D01B78002B4FD048
:10A10000D6F8008098F800404CB32D2C6CD0303C31
:10A11000092C03D908F101033360F1E7414600241B
:10A1200000220FFA82F9013211F80930303B092B75
:10A13000F7D92E2140460AF073F818B3002211B265
:10A14000431801325B78303B092BF8D94378A3F1EF
:10A150003002092A01D82F2B03D8002204E0A1469F
:10A16000E7E7392B88BF09220A2555438278A2F1F7
:10A170003003092B05D82F2A16D9392A88BF09237D
:10A180001D4499B9404608F05EFE394602466846CD
:10A19000FAF7ADFD2C2130680AF042F810BB3060B0
:10A1A000384603B0BDE8F0830023E9E702294046C2
:10A1B0000EDCB9F1070F0BDC08F045FE64224243C8
:10A1C00004B16D422A4439466846FAF7B6FDE1E724
:10A1D00008F032FE08F0C2FD394602466846FAF73A
:10A1E00092FDD7E70130DAE708F10101012497E792
:10A1F00008B500200BF05CF8ADEB000008BD70471F
:10A2000030B5441E224612F8013F002BFBD11A46FE
:10A210000A2514F8010F70B1032A14DC2E2806D188
:10A22000FF2B10DC8818013203710023F1E730386E
:10A2300005FB0303EDE7FF2B04DC032A02DC1144DA
:10A2400001200B7130BD0020FCE700002DE9F34137
:10A250000024DFF840800C700D461746061D0A22C8
:10A2600001A916F8010B09F007F83A4601A928469A
:10A270000AF019F8032C04D03A46414628460AF061
:10A2800012F80134A3B2042B1CB2E8D1284602B064
:10A29000BDE8F081619201002DE9F0410E4D0F4FB4
:10A2A000DFF83C8006460024032C0ED033190A2226
:10A2B0001979284605F021FF41462846013405F06A
:10A2C000D5FE042CF0D1BDE8F081F1790A222846B0
:10A2D00005F013FF3946F0E7BC030020247F01009E
:10A2E000619201002DE9F047DFF8F8A0DAF800509C
:10A2F00004460E4617469946002D3ED02B7C03F0AF
:10A300000F03062B38D12E4A2E48294604F0A6FB0F
:10A31000022F80462CD0032F2CD12B4ADAF80010C4
:10A32000284804F09BFB0546B8F1000F25D098F8AB
:10A33000103003F00F03042B1FD1D8F8141032464D
:10A34000204609F0D6FF32462049204609F0ABFFEF
:10A35000B5B12B7C03F00F03042B11D13246696990
:10A36000204609F0A0FF042F16D12046BDE8F08753
:10A37000174AD3E70025D7E7002532461549DFE71E
:10A38000022F1AD0032F15D0012FECD1124B1968D0
:10A390003246204609F087FF32460C49204609F034
:10A3A00082FFB9F1000FE0D032464946204609F05D
:10A3B0007AFFDAE732460949EBE732460849E8E72F
:10A3C0000B99010078070020B4940100C18B0100B3
:10A3D0001099010075990100880300202999010056
:10A3E00026990100A00400200B460A2201461846C7
:10A3F00006F08FBC10B5054C0549204605F03FFE20
:10A400002046BDE8104005F041BE00BF70030020AB
:10A41000D698010010B54AB102441BB1B2FBF3F467
:10A4200003FB14228A4208D288420AD9012010BDB7
:10A43000884294BF00200120F9E78242F8D800202A
:10A44000F5E78242F5E700002DE9F04FA7B004AE32
:10A450000D4686E80C00DDE930BA0446002800F01D
:10A46000F180037C03F00F03062B1ED8DFE813F006
:10A47000E3001D001D001D00DF0007001F00934FBB
:10A48000C4683B7801333B7064B1329BCDF800B0B7
:10A49000CDE901A3204696E80C002946FFF7D4FF3A
:10A4A0006468F1E73B78013B3B7000200FE0014618
:10A4B000874A884804F0D2FA814658B10023CDE992
:10A4C0000133009396E80C002946FFF7BDFF27B043
:10A4D000BDE8F08F804A7F48214604F0BFFA7F4AEA
:10A4E000214680467B4804F0B9FA7D4A074621465A
:10A4F000784804F0B3FA1DB1012D7BD04D460EE033
:10A50000784A7448214604F0A9FA8146764A71488F
:10A51000214604F0A3FA0546B9F1000F00D1A14687
:10A52000002D08BF2546B8F1000F00F08780002FEE
:10A5300008BF5746B9F1000F00F0828099F810204B
:10A5400002F00F02042A7BD1D9F81440002D7BD0F1
:10A550002B7C03F00F03042B76D1D5F814904FF029
:10A56000000AB8F1000F00F0D380002C00F08E80BC
:10A570005E495F4805F07AFDD8F814105C4805F094
:10A580007EFD5C495A4805F071FD2146584805F0AA
:10A5900076FD574805F07AFD3046FAF733FE002F76
:10A5A00040F0288198F8103003F00F03042B40F09E
:10A5B0001F81514BD8F814101A6816A8F8F7FCF848
:10A5C00016A8F8F755F888B1FFF712FEB0F5966FA8
:10A5D000054669DA49494A4805F048FD0A222946F4
:10A5E000474805F0ACFD464805F050FD16A8F7F7C2
:10A5F00083FEFDE0434A3748214604F02FFA424AE1
:10A6000081462146334804F029FA0546B9F1000F86
:10A6100040F0F480334A2F48214604F01FFA814667
:10A62000002D3FF473AF002808BFA1467BE700254B
:10A630002F46A84673E70025A9462F46D84676E759
:10A64000002483E75746D8460023009310224FF496
:10A65000407306A93046FAF7C3FC81463046FAF744
:10A66000D9FB0FFA80FABAF1000F7FF47AAF3046C7
:10A67000FAF769F938B93046FAF774F9002818BFC3
:10A680004FF0020A6DE74FF0010A6AE71F491848C8
:10A6900005F0ECFCD8F81410154805F0F0FC15494D
:10A6A000134805F0E3FC77E734B100231A4621464E
:10A6B00016A8F9F7ADFB99E701230093019423460F
:10A6C00096E8060016A8F8F7E3FC8FE76D03002074
:10A6D000807E010078070020DA7E01001C7F0100E7
:10A6E000DF7E01008498010089980100989801009C
:10A6F000700300209F980100DC030020BD9801003A
:10A700008C0300208E98010093980100A49801000A
:10A71000002F6DD0B9F1000F6AD03B7C03F00F031E
:10A72000042B61D17B69ADF84CA000254FF47A72FF
:10A73000CDE90B52334A0A92CDE90E3516AA4023D1
:10A7400029460AA8CDE9105512958DF84E5005F00E
:10A7500071FF26AB18442C4900F8405C2B4805F0EB
:10A7600085FC7969294805F08AFC2949274805F0C4
:10A7700086FC16A9254805F082FC2649234805F0E9
:10A7800075FC4946214805F07AFC204805F07EFC1E
:10A79000214804F0B5FC38B3204B93F900301BBBC3
:10A7A0002F2116A809F03CFD28B97B69032240211E
:10A7B00016A8FFF797FD1A49144805F057FC16A98B
:10A7C000124805F05CFC1349104805F04FFC49465F
:10A7D0000E4805F054FC0D4805F058FC01234A468C
:10A7E00016A90D4804F0E9FEB8F1000F7FF4DAAEC7
:10A7F00001206CE6B9F1000F8FD1D3E600287FF479
:10A8000092AE83E668980100AE98010070030020C4
:10A81000A19801009F980100E8030020B8030020E0
:10A82000B698010010B5044606F01CFAE040431E3D
:10A83000033388BF012010BD054B1A68054B53F840
:10A84000201001238B40134214BF012000207047C9
:10A8500008050050AC9C01000120704700207047A3
:10A8600038B52149214805F017FC0121204800F0A6
:10A870007CF91F4800F006F90121172006F0E0FBE3
:10A880000021162006F0DCFB1424002529461720A1
:10A8900006F0FEFB0A2006F019FA013C85F00105DE
:10A8A000F4D11420134C06F011FA114800F094F87A
:10A8B0002068A0B100F050FA88B1206800F092FB47
:10A8C0000D490A4805F0E8FB206800F051FA2068BD
:10A8D00000F0CCFB28B10949044805F0DDFB01205C
:10A8E00038BD0749F8E700BFE69801007003002073
:10A8F0009C05002024050020F0980100BC97010071
:10A90000D097010007B5002300931A461946034863
:10A9100005F064FB03B05DF804FB00BF9405002064
:10A920002DE9F84380460D46174601EB02090C4617
:10A930004C45A4EB05060BD0D8F8003014F8011BE9
:10A940001B68404698470028F2D13046BDE8F8839E
:10A950003E46FAE77047203005F0F1BC203005F0A4
:10A96000E0BC203005F0F1BC38B5437F0D460BB993
:10A97000002038BD00F16804204605F0EEFC0028F8
:10A98000F6D12046294605F0BDFC0120F1E7000084
:10A990002DE9F0411E4600254FF47A73C0E90153BA
:10A9A0000C4B044640F8203B8846174605F0A1FCB6
:10A9B00004F1680005F09DFC9DF8183063769DF861
:10A9C0001C302676C4E90487A37665772046BDE867
:10A9D000F08100BF88990100817E284A0123C37657
:10A9E00070B552F82140417E52F821104FF0A04539
:10A9F00004F5E07401F5E07140F20C6645F824605E
:10AA000045F8216001694FF0CC74C1F82445016913
:10AA10000624C1F80045847E016952F82440C1F83B
:10AA20000845447E016952F82420C1F80C2590F9AC
:10AA30001820510902F01F0293406031104A42F879
:10AA4000213090F91830002BBDBF03F00F0302F640
:10AA5000FC32D2189B18B5BF40234022137683F8EE
:10AA6000002390F918300122590903F01F0302FA5C
:10AA700003F3034A42F8213070BD00BFAC9C0100D3
:10AA800000E100E0C37E23B103690022C3F8002582
:10AA900070474269C2F8003570472DE9F04104461D
:10AAA00088461F461546002A50D000F12006304641
:10AAB00005F033FC2369C3F88885236901221A62F3
:10AAC0002369C3F834652369C3F8385523691A60CC
:10AAD0002269D2F84C311BB9D2F82431002BF8D0BE
:10AAE0000023C2F84C312269D2F85C311BB9D2F88C
:10AAF0002431002BF8D00023C2F85C3122696FB9F1
:10AB0000D2F8243153B90123D3612369D3F8482102
:10AB1000002AFBD00022C3F8482109E00123536139
:10AB20002369D3F80421002AFBD00022C3F80421B2
:10AB30002369D3F8242112B10022C3F82421236908
:10AB4000D3F83C052066C0B2BDE8F0811046FBE7B3
:10AB50000123FFF7A2BF10B5044680F8B01068309B
:10AB600005F0DBFB0123637710BDF8B500234377C5
:10AB7000036990F8B020C3F88825036901261E6296
:10AB8000036900F168050446C3F8445528460F469A
:10AB900005F0D5FB2369C3F8480523699E60236946
:10ABA000D3F850211AB9D3F82421002AF8D0002272
:10ABB000C3F85021284605F0C2FB236930B1D3F811
:10ABC00060211AB9D3F82421002AF8D00022C3F852
:10ABD000602123696FB9D3F8242152B90122DA61C7
:10ABE0002369D3F84821002AFBD00022C3F848216A
:10ABF00009E001225A612369D3F80421002AFBD01D
:10AC00000022C3F804212369D3F8240168B100228B
:10AC1000C3F824212369D3F8C404C3F8C404022868
:10AC200003D004280CBF03200420F8BD0121FFF746
:10AC30009CBF70B54369D3F86421044692B10022E9
:10AC4000012500F12006C3F864210577304605F0A0
:10AC500064FB6369C3F8346563694022C3F838252F
:10AC600063691D636369D3F86821DAB10025C3F80D
:10AC7000685104F16806012363772577304605F0B3
:10AC80004CFBD4F8B43003B198476369657730461C
:10AC9000C3F8446505F053FB6369C3F8480563696D
:10ACA00001225A636369D3F8042162B10022C3F818
:10ACB0000421237F3BB16369D3F83C05D4F8B83055
:10ACC000206603B198476369D3F8242152B100226A
:10ACD000C3F824216369D3F8D024C3F8D02463696E
:10ACE00001225A6170BD00000148FFF7A2BF00BFFA
:10ACF0009C05002007B516231722CDE900324FF03E
:10AD00004022042311460348FFF742FE03B05DF8DA
:10AD100004FB00BF9C0500200148FFF787BF00BF70
:10AD20009C05002010B54FF4C05303800023044657
:10AD3000837003610248FFF74FFE204610BD00BF3D
:10AD40009C05002001617047807870474178014878
:10AD5000FFF701BF9C05002008B5FFF7F7FF034888
:10AD6000FFF764FFB0FA80F0400908BD9C050020A1
:10AD7000012303707047FF23C37200230373C37062
:10AD8000037143718371C37103724372837270479D
:10AD900010B5064A01440023884204D010F8014B44
:10ADA0006340D35CF8E7184610BD00BFA0990100CE
:10ADB000FFF7E1BF38B5084C0D46FFF7C7FFE121AB
:10ADC0002046FFF7D1FD29462046FFF7CDFDBDE81F
:10ADD0003840FFF7A1BF00BF9C05002010B5054C0F
:10ADE000417801222046FFF7B3FE2046FFF7B6FD6B
:10ADF000C0B210BD9C05002010B5F0210446FFF73D
:10AE0000D9FF2046BDE81040FFF7E8BF70B5044603
:10AE100005F028FF0025064605F024FF801BB0F54D
:10AE20007A7F4DD2236903B198472046FFF7E4FFAC
:10AE300010F00103054605D1A278012A00D1A370C4
:10AE4000284670BD1420013800BF00BF00BF00BFFE
:10AE500000BF00BF00BF00BF00BF00BF00BF00BFFA
:10AE600000BF00BF00BF00BF00BF00BF00BF00BFEA
:10AE700000BF00BF00BF00BF00BF00BF00BF00BFDA
:10AE800000BF00BF00BF00BF00BF00BF00BF00BFCA
:10AE900000BF00BF00BF00BF00BF00BF00BF00BFBA
:10AEA00000BF00BF00BF00BF00BF00BF00BF00BFAA
:10AEB00000BF00BF00BF00BF00BF00BFC3D1ABE7F2
:10AEC0000123BCE710B5E1210446FFF773FF2046DC
:10AED000BDE81040FFF782BF10B50446FFF796FFAC
:10AEE0002046FFF733FF96210648FFF73DFDFFF7A9
:10AEF00013FF2046FFF78AFF2046BDE81040FFF70A
:10AF0000E1BF00BF9C050020FFF7E6BF10B5C321DD
:10AF10000446FFF74FFF2046BDE81040FFF75EBF35
:10AF200038B504460D46FFF771FF2046FFF70EFFC8
:10AF3000D2210C48FFF718FDE94345EA0111C9B2D7
:10AF40000848FFF711FDFFF7E7FE2046FFF746FF31
:10AF5000A84202D00423A37038BDA378042BFBD1F0
:10AF60000023F8E79C05002010B50446FFF7CEFF4C
:10AF700040F00401C9B22046BDE81040FFF7D0BF41
:10AF800070B5164604460D46FFF740FF16B1204641
:10AF9000FFF7EAFF2046FFF7D9FEA5210548FFF796
:10AFA000E3FC29460348FFF7DFFCBDE87040FFF7EC
:10AFB000B3BE00BF9C05002070B500220C46552191
:10AFC0000646FFF7DDFF651E073415F8011F002256
:10AFD0003046FFF7D5FFA542F7D170BDFFF7ECBFB4
:10AFE000FFF7CEBF10B50446FFF7B0FE20460022A3
:10AFF000F021FFF7C5FFBDE81040FFF78DBE000050
:10B0000070B5164605460C46FFF700FF16B12846F8
:10B01000FFF7AAFF2846FFF799FE87210648FFF7AA
:10B02000A3FC002C0CBF214680210348FFF79CFCA9
:10B03000BDE87040FFF770BE9C05002010B50022EF
:10B0400004460121FFF7DCFF2046FFF7DFFEC0F3D7
:10B05000401010BDFFF7F2BF10B50446FFF756FFD2
:10B0600020460021BDE81040FFF75ABF38B504461E
:10B07000FFF7CCFEC30729D42046FFF7EDFF20469B
:10B08000FFF7C4FE2046FFF761FEB4211048FFF72A
:10B090006BFCFFF741FE2046FFF7B8FE10F00403FB
:10B0A000054602D00223A37002E0A278022AFAD059
:10B0B000237843B12046FFF729FF40F00101C9B2D0
:10B0C0002046FFF72DFFC5F3400038BD0020FCE708
:10B0D0009C0500202DE9F74F057B04460F46002D07
:10B0E0006BD1FFF7C3FF002869D02046FFF78EFE23
:10B0F0002A46F0212046FFF743FFDFF8C8804FF0D3
:10B10000FF394FF0010A94F90B30EEB24FEAD60B3B
:10B110009D4206F007060AFA06F623DA04EB0B0353
:10B12000DB78334020460193FFF770FE2046FFF79F
:10B130000DFE78214046FFF717FC019B002B0CBF4A
:10B14000194680214046FFF70FFCFFF7E5FD20463A
:10B15000FFF75CFE820600F0400307D55BB16FF09D
:10B16000010027E00CBF01230023DBE71BB9030626
:10B1700058BF4FFA85F904EB0B03010693F903203E
:10B1800076B205F101054CBF3243B243402DDA706F
:10B19000B9D1B9F1FF3F04BF0123237384F80B90A9
:10B1A000E31C013F0B3413F8012B07F8012FA342D6
:10B1B000F9D1012003B0BDE8F08F0020FAE74FF08D
:10B1C000FF30F7E79C05002008B5FFF783FF20EA72
:10B1D000E070C0B208BDFFF749BF7047054A826101
:10B1E0000022027102700922427001228160827085
:10B1F000C2707047DBB1000010B50C462046072135
:10B20000FFF7C6FDE3791B1A5842584110BD70B5CF
:10B21000044680680E461546FFF7DDFFB8B131469B
:10B22000A068FFF7DBFE0022BE21A068FFF7D8FE72
:10B230006E1E0835A068FFF767FE06F8010FAE42E4
:10B24000F8D1A068FFF7C7FF431E5842584170BDB0
:10B2500010B51446FFF7DBFF38B108212046FFF791
:10B2600097FD237A1B1A5842584110BD70B5044609
:10B270000D4680681646FFF7AEFF2946A068FFF727
:10B28000ADFE00224E21A068FFF7AAFE0022B17891
:10B29000A068FFF7A5FE0022F178A068FFF7A0FEE6
:10B2A0002B78102B04D000223179A068FFF798FE8C
:10B2B000A068FFF790FF2946A068FFF78FFE22786D
:10B2C000A0684821FFF78CFE142005F0FFFC2378CE
:10B2D00013B10A2005F0FAFCA068BDE87040FFF742
:10B2E0007ABF38B504460D468068FFF774FF2946DB
:10B2F000A068FFF773FE0022B421A068FFF770FE7C
:10B30000A068FFF7A7FE0546A068FFF764FFB5FA3F
:10B3100085F0400938BDF0B585B0144601AA07464E
:10B320000E46FFF795FF054690B13378102B0FD0EE
:10B330000B2C10D00C2C03D00A2C0ED13F2300E094
:10B340007F2301AA314638468DF80830FFF78EFF7B
:10B35000284605B0F0BD5F23F3E71F23F1E71FB5D3
:10B360000B78102B10D001AAFFF772FF78B19DF86F
:10B3700008303F2B0ED003D81F2B0DD0002006E045
:10B380005F2B03D07F2BF9D10C2000E00B2005B000
:10B390005DF804FB0A20FAE70920F8E7F0B587B06A
:10B3A000044605F05FFC00F51C55A068FFF700FDA2
:10B3B000002310352371012601A9A068FFF704FFBF
:10B3C00040B305F04FFCA84224D201A92046FFF764
:10B3D00013FF0028F0D023782BB901A92046FFF7EE
:10B3E00080FF00B1267003AA01A92046FFF70FFFD6
:10B3F00001A920466778FFF7B2FF874205D9607838
:10B400002379607001332371D6E701A92046FFF745
:10B41000A6FFF5E707B0F0BD817070471FB501AA20
:10B42000FFF7F5FE9DF80400003018BF012005B0BD
:10B430005DF804FB0939C9B20229F8B598BF104B71
:10B440000546164694BF33F9114040F2EE248AB106
:10B45000C3787BB103786BB905F004FC074631462D
:10B460002846FFF7DBFF20B905F0FCFB001BB842C4
:10B47000F5D3F8BD2046BDE8F84005F027BC00BF75
:10B48000A09A0100F8B504460F46FFF768FF06468C
:10B4900010B900252846F8BDA068FFF79CFE0028DB
:10B4A000F7D03946A068FFF799FD2278A0684421BB
:10B4B000FFF796FDA5782DB13A4631462046FFF7B5
:10B4C000B9FFE7E70125E5E710785378C00040EAC7
:10B4D000C3200B78102B00B20BD1D1799379C00027
:10B4E000CB1ADB0120F07F0093FBF1F3103B1844F3
:10B4F00000B2704730B585B001AA04460D46FFF78B
:10B50000A7FE30B101AA29462046FFF7DDFF05B0AE
:10B5100030BD0148FBE700BF80E4FFFF10F5DC5FB2
:10B52000CABF07EE900ADFED037AFAEEEC7A17EE67
:10B53000900A70470000FEC208B5FFF7DBFFBDE8C8
:10B540000840FFF7EBBF01460422012001F0AABA30
:10B5500001460422052001F0A5BA01460622092071
:10B5600001F0A0BA014604220F2001F09BBA0000AE
:10B570002DE9F04F3D4E3E4C336813F0010387B088
:10B5800082468B4615460ED1E3644FF47A732365E9
:10B59000384BA36404F15C0004F018FD082384F820
:10B5A000683001233360344E346001F04DFC0027D5
:10B5B000002859D04FF000494FF00208CDF80C9008
:10B5C00005978DF8108003AC94E80E002B4805F029
:10B5D000E9FD5046FFF7C1FF3B463A463946009722
:10B5E000204604F0FBFC04A8FFF7BCFF234805F04D
:10B5F000E5FD2B465A465146306801F08FFF012881
:10B6000005462DD1CDF80C9005978DF8108094E863
:10B610000E001A4805F0C6FD3168204601F0E5FC31
:10B6200004A8FFF79FFF3168204601F0ECFC04A856
:10B63000FFF789FF3168204601F0DEFC04A8FFF720
:10B6400087FF0E4805F0BAFD3168204601F0E2FCA4
:10B650000B4B049A5A6005F01FFB80B200F08EFD80
:10B66000284607B0BDE8F08F0546F9E758060020E8
:10B67000700600200C9B01006C060020580800207A
:10B6800064060020F0B585B007460E4614461D46F8
:10B6900001F0DAFB00B34FF0004301930023039362
:10B6A00002238DF8083004AB13E90E000B4805F0B7
:10B6B00079FD3846FFF751FF301DFFF753FF281D76
:10B6C000FFF741FF0A980430FFF742FF034805F0F7
:10B6D00075FD034B62685A6005B0F0BD5808002044
:10B6E00064060020F0B58DB01D4600230F46009380
:10B6F000FF230446164619461A4602A804F06EFCBB
:10B700000B4B7A680493CDE905237268CDE90723D2
:10B710006A68CDE90923039B0B930AAB009306AA41
:10B7200008AB04A92046FFF7ADFF0DB0F0BD00BF88
:10B730001C9D010000B50B4B4968526889B0CDE9EA
:10B740000231CDE905230493012301918DF80730DF
:10B75000019B079304AA06AB02A9FFF7C3FF09B038
:10B760005DF804FB1C9D01007FB5094B4A680493FA
:10B77000CDE90232012301928DF80730019B059338
:10B7800004AA02A9FFF7D6FF07B05DF804FB00BFCB
:10B790001C9D010008B501F0BDFB012803D0022863
:10B7A0000CBF0220002008BD7FB51E4E3068002867
:10B7B00036D001F0CBFE0228044601D004282CD15B
:10B7C0004FF00043019300230393022301AD8DF852
:10B7D000083095E80E00144805F0E4FC316828466E
:10B7E00001F003FC02A8FFF7BDFE3168284601F016
:10B7F0000AFC02A8FFF7A7FE3168284601F0FCFB0F
:10B8000002A8FFF7A5FE084805F0D8FC31682846D5
:10B8100001F000FC054B029A5A60204604B070BD4E
:10B820000446FAE76C060020580800206406002051
:10B8300030B585B0044604F0C9FB4FF000430193D6
:10B84000002303930A4D02238DF8083004AB13E95B
:10B850000E00284605F0A6FC0422A1180F2001F0D6
:10B86000D9F9284605F0AAFC204605B030BD00BF36
:10B870005808002030B585B0044604F0A7FB4FF00F
:10B8800000430193002303930A4D02238DF80830EF
:10B8900004AB13E90E00284605F084FC0422A1182D
:10B8A000052001F0B7F9284605F088FC204605B0D0
:10B8B00030BD00BF5808002030B585B0044604F004
:10B8C00085FB4FF000430193002303930A4D0223AD
:10B8D0008DF8083004AB13E90E00284605F062FC31
:10B8E0000422A118012001F095F9284605F066FC14
:10B8F000204605B030BD00BF5808002007B5002322
:10B9000000931A461946044804F068FB034803B044
:10B910005DF804EB04F05ABB5C06002064060020CE
:10B92000007C07288CBF00200120704781F00100B7
:10B9300070470846704708B50368DB6B984780F08E
:10B940000100C0B208BD4182704713B502AB026866
:10B9500003F8011D546819460122A04702B010BD2A
:10B96000037C087C984204D107288CBF002001206A
:10B97000704700207047000010B50446007C07287F
:10B9800016D800F0A1FD182806D80A4B23FA00F0BB
:10B99000C04300F0010010BD1C2807D123682046D9
:10B9A0009B689847003018BF0120F4E70120F2E7B8
:10B9B0000020F0E701001001F0B591B0044604A8A2
:10B9C0000F46164604F002FB00224FF47A73CDE9CD
:10B9D00008230CA8184B079304F0F8FA08236846CC
:10B9E0008DF83C3004F0F2FA207C072807D800F0EC
:10B9F0006BFD10B1207C00F0CBFD082323740F4BAE
:10BA00000F4D5B68039302A904A8029501F0DDFDC8
:10BA100041F288336A46394604A801F05FFF40B11D
:10BA20002368019A9B6903920295324602A9204637
:10BA3000984711B0F0BD00BF0C9B010064060020C8
:10BA40001C9D010008B5007C072802D800F02EFFDD
:10BA500008BD0020FCE710B50446207C07280BD861
:10BA600000F032FD172801D01C2805D1207C00F001
:10BA70001DFFB0F5006FF0D310BD38B50546007C52
:10BA80000728144605D892B200F092FE10B901239F
:10BA90006B600024204638BD08B5007C072802D81A
:10BAA00000F02EFE08BD0020FCE7007C072802D82D
:10BAB00012B200F08BBD0020704707B501220DF1D6
:10BAC0000701007C00F082FD0028CCBF9DF8070034
:10BAD0004FF0FF3003B05DF804FB10B5037C072B7B
:10BAE000044602D94FF0FF3010BD03689B689847A9
:10BAF0000028F7D0207C00F02FFEF5E738B504468B
:10BB0000007C07280AD800F043FD05F0ABF8054695
:10BB1000207C00F0D9FC10B90823237438BDFBF752
:10BB200087FA012005F0D2F805F09CF8638A401BE3
:10BB30009842EDD3207C00F0E5FCEDE77FB50446AC
:10BB4000007C07280D46164607D800F0BDFC10B152
:10BB5000207C00F01DFD082323740021684604F0BA
:10BB600049FA6A68019B9A4202D1002004B070BD74
:10BB70004FF0FF3102A804F03DFA6A68039B9A4235
:10BB8000F3D00021212000F003FB07282074ECD81B
:10BB9000291D324600F0D4FC05F064F80546207CEF
:10BBA00000F092FC172815D01C2813D00028DCD0F8
:10BBB00005F058F8638A401B984205D8FBF738FA1D
:10BBC000012005F083F8EAE7207C00F09BFC0823C5
:10BBD0002374CAE70120C9E710B41446064A127854
:10BBE00001EB022101EB00201A46214680B25DF8EC
:10BBF000044B01F00FB800BF3C0700207FB5037C69
:10BC0000072B05464FF000041BD84FF000430226D7
:10BC10000394019301AC8DF8086094E80E000A4883
:10BC200005F0C0FA334622460421287CFFF7D4FFF2
:10BC30009DF804309DF80540034844EA032405F0CC
:10BC4000BDFA204604B070BD580800207FB50B7CBB
:10BC5000072B05460E4605D9002104F0CBF92846EE
:10BC600004B070BD4FF000430193002303930223FF
:10BC700001AC8DF8083094E80E00084805F092FAFF
:10BC8000042322460C21307CFFF7A6FF034805F071
:10BC900095FA2146284604F0B3F9E0E75808002059
:10BCA0007FB5037C072B05464FF000041BD84FF0EF
:10BCB000004302260394019301AC8DF8086094E8D8
:10BCC0000E000A4805F06EFA334622461021287C01
:10BCD000FFF782FF9DF804309DF80540034844EAD1
:10BCE000032405F06BFA204604B070BD580800200C
:10BCF00007B5002300931A461946034804F06EF96D
:10BD000003B05DF804FB00BFDC06002003681B6B7A
:10BD100018470000024A02608A694260704700BF0B
:10BD20001C9D0100808B7047008A7047408C7047D3
:10BD300013B502AB026803F8011D546819460122CD
:10BD4000A04702B010BD704710B5044690F820001F
:10BD5000072804D800F0D6FB082384F8203010BD53
:10BD600038B5044690F8200007280D4601D800F0A9
:10BD7000C9FB2946022000F00BFA072884F82000AE
:10BD80004FF000009EBF60842582012038BD000076
:10BD9000F0B591B0044604A80F46164604F016F913
:10BDA00000224FF47A73CDE908230CA8134B0793B4
:10BDB00004F00CF9082368468DF83C3004F006F9CD
:10BDC0000F4B104D5B68039302A904A8029501F084
:10BDD000FCFB41F288336A46394604A801F07EFD37
:10BDE000012808D12368019A1B6A03920295324602
:10BDF00002A92046984711B0F0BD00BF0C9B01007E
:10BE0000640600201C9D010008B50023C383043193
:10BE100090F8200000F09CFD08BD08B590F82000C7
:10BE200000F0C4FD08BD10B593B204460A46C18BAC
:10BE300090F8200000F060FDE38B0344E38310BD25
:10BE400013B5438C04461BB94FF0FF3002B010BD50
:10BE500001220DF1070190F8200000F0B7FB002847
:10BE6000F2DD638C9DF80700013B6384EEE710B5BB
:10BE7000438C044613B94FF0FF3010BD934294BF7A
:10BE80001AB212B290F8200000F0A0FB0028F2DDF8
:10BE9000638C1B1A6384F0E708B590F82030072BF9
:10BEA00005D8428C1AB1184600F056FC08BD4FF078
:10BEB000FF30FBE773B5044690F8200007280E46D4
:10BEC000154601D800F01EFB094B00932A46736803
:10BED00001936946822000F017FA072884F82000B1
:10BEE0004FF000009EBF60840120258202B070BD2B
:10BEF0001C9D010013B50446628C2AB12368002101
:10BF00001B6B20469847F7E794F8200000F0F8FBF9
:10BF1000D8B10822694694F8200000F057FB0028A9
:10BF200013DD694604F1140004F072F89DF8042052
:10BF30009DF805309DF8070003EB0223A3839DF8CD
:10BF4000063000EB032080B2608402B010BD000018
:10BF500007B5002300931A461946034804F03EF83B
:10BF600003B05DF804FB00BFE406002007B5084BF2
:10BF70001B7801EB032101EB002001220DF10701E9
:10BF800080B200F047FE9DF8070003B05DF804FBA7
:10BF90003C07002007B5084B1B7801EB032101EBA0
:10BFA000002002A980B201F8012D012200F07AFDE3
:10BFB000C0B203B05DF804FB3C07002010B4144687
:10BFC000064A127801EB022101EB00201A462146B5
:10BFD00080B25DF8044B00F065BD00BF3C07002057
:10BFE0002DE9F7430C4617461E4601AA02232421D9
:10BFF0000546FFF7F1FD9DF804209DF8053043EA62
:10C000000223224A1C441378332B0CBF05F108008D
:10C0100005F11000A4B2C002C4F30A0980B248447A
:10C02000372B904680B22DD009EB0603B3F5006F95
:10C0300028DDC9F500691FFA89F94A46394600F03A
:10C0400031FD98F80030332B0CBF05F1080005F1E5
:10C050001000C002A6EB090280B292B207EB090100
:10C060003444A4B200F01EFD23128DF8043001AA5E
:10C070000223242128468DF80540FFF79FFF03B0D7
:10C08000BDE8F08332463946EAE700BF3D070020AD
:10C0900008B50321FFF76AFF08BD07B50B128DF83D
:10C0A00004308DF80510022301AA0421FFF786FF52
:10C0B00003B05DF804FB08B50A4604230C21FFF722
:10C0C0007DFF08BD07B50B128DF804308DF8051003
:10C0D000022301AA1021FFF771FF03B05DF804FBF2
:10C0E00007B5022301AA2021FFF776FD9DF8040081
:10C0F0009DF8053043EA002003B05DF804FB000022
:10C1000038B50546FFF7ECFF04462846FFF7E8FF81
:10C110008442034604D1034B03EBC5039C8038BD26
:10C120001C46F2E7F406002007B5022301AA2621E7
:10C13000FFF752FD9DF804009DF8053043EA00200A
:10C1400003B05DF804FB07B5022301AA2821FFF71D
:10C1500043FD9DF804009DF8053043EA002003B03C
:10C160005DF804FB044B1B78332B0CBF0C301830EC
:10C17000C00280B2704700BF3D070020034B1A8801
:10C18000C0F30D0050401880704700BF0800002029
:10C190002DE9F043574B1B7885B081460F468BB392
:10C1A000332B4FF0004301934FF000054FF0020393
:10C1B00003958DF8083001AE96E80E004E4814BF86
:10C1C0004FF008084FF0040804F0ECFFECB22046F2
:10C1D000FFF75EFF7055D8B10135EBB29845F5D841
:10C1E00000234FF03451F25C1D2ADCB203D821FA4F
:10C1F00002F2D20708D40133DAB24245F3D33E4803
:10C2000004F0DCFF082465E01021204600F0C6FEA3
:10C210003A4B002123F81410FA20013800BF00BF68
:10C2200000BF00BF00BF00BF00BF00BF00BF00BF16
:10C2300000BF00BF00BF00BF00BF00BF00BF00BF06
:10C2400000BF00BF00BF00BF00BF00BF00BF00BFF6
:10C2500000BF00BF00BF00BF00BF00BF00BF00BFE6
:10C2600000BF00BF00BF00BF00BF00BF00BF00BFD6
:10C2700000BF00BF00BF00BF00BF00BF00BF00BFC6
:10C2800000BF00BF00BF00BF00BF00BF00BF00BFB6
:10C29000C3D14A462046FFF77DFEFF2202212046F9
:10C2A000FFF778FED7B139462046154DFFF7F5FE6A
:10C2B00000260121204600F071FE25F8346020465A
:10C2C000FFF741FF05EBC40358809E719E800A482A
:10C2D00004F074FF204605B0BDE8F083094B1A88CE
:10C2E000013292B2B2F5404F38BF4FF440421A804B
:10C2F0001988D9E73D07002058080020580700207A
:10C30000F4060020080000202DE9F047694B1B7857
:10C3100086B082460E461746A3B3332B4FF0004338
:10C3200003934FF000054FF0020305958DF8103090
:10C330000DF10C0898E80E005F4814BF4FF0080993
:10C340004FF0040904F02EFFECB22046FFF7A0FEE8
:10C3500008F80500E0B10135EBB29945F4D80023A7
:10C360004FF0345118F803201D2ADCB203D821FA0B
:10C3700002F2D20708D40133DAB24A45F2D34E486A
:10C3800004F01CFF082485E01021204600F006FE82
:10C390004A4B002123F81410FA20013800BF00BFD7
:10C3A00000BF00BF00BF00BF00BF00BF00BF00BF95
:10C3B00000BF00BF00BF00BF00BF00BF00BF00BF85
:10C3C00000BF00BF00BF00BF00BF00BF00BF00BF75
:10C3D00000BF00BF00BF00BF00BF00BF00BF00BF65
:10C3E00000BF00BF00BF00BF00BF00BF00BF00BF55
:10C3F00000BF00BF00BF00BF00BF00BF00BF00BF45
:10C4000000BF00BF00BF00BF00BF00BF00BF00BF34
:10C41000C3D152462046FFF7BDFDFF220221204630
:10C42000FFF7B8FD002F39D039462046FFF735FE1B
:10C430005E238DF80630737903F07F038DF80730A3
:10C44000B3798DF808300125F3798DF80930311D65
:10C450002046ADF80450FFF72EFE39462046FFF780
:10C4600031FE0623194601AA2046FFF7A7FD2946FB
:10C47000134D0026204600F091FD25F8346020463B
:10C48000FFF761FE05EBC40358809E719E800A4849
:10C4900004F094FE204606B0BDE8F087094B1A88E8
:10C4A000013292B2B2F5404F38BF4FF440421A8089
:10C4B0001988BAE73D0700205808002058070020D7
:10C4C000F40600200800002030B585B04FF000438E
:10C4D0000193002303930A4C02238DF8083004AB28
:10C4E00013E90E000546204604F05CFE2846FFF7DF
:10C4F000CFFD0546204604F061FE284605B030BD5C
:10C500005808002030B585B04FF000430193002358
:10C5100003930A4C02238DF8083004AB13E90E0094
:10C520000546204604F03EFE2846102100F036FD68
:10C53000204605B0BDE8304004F040BE5808002059
:10C54000F0B585B04FF000430193002303930F4DE6
:10C5500002238DF8083004AB04460F4616462846E1
:10C5600013E90E0004F01EFE39462046FFF7A3FD36
:10C5700031462046FFF7A6FD2046042100F00EFDBF
:10C58000284605B0BDE8F04004F018BE5808002069
:10C5900030B585B04FF000430193002303930A4C5C
:10C5A00002238DF8083004AB13E90E00054620463F
:10C5B00004F0F8FD2846082100F0F0FC204605B004
:10C5C000BDE8304004F0FABD580800202DE9F04FD6
:10C5D00085B04FF000430193464E0023039302239E
:10C5E00036F830408DF8083001AB174605468946CD
:10C5F00041480ECB04F0D6FDA7420EDD2846FFF7DA
:10C6000093FD04462846FFF78FFDA042F9D106EBC3
:10C61000C5039B79E41A26F835408CB92846FFF704
:10C6200037FD142805D020B1B0F11C0418BF4FF01D
:10C63000FF34314804F0C2FD204605B0BDE8F08F5C
:10C640004FEAC50BBC4206EB0B03A8BF3C46B3F850
:10C650000280A7B2B9F1000F21D02846FFF782FD72
:10C66000264A1278C8F30A0A5044372A80B23DD0CD
:10C670001AFA84F2B2F5006F38DDCAF500631FFACA
:10C6800083FA5246494600F0C5FA2846FFF76AFD8C
:10C69000A7EB0A02D14492B2494600F0BBFA06EB7E
:10C6A0000B0236F835309179B844DB1B0F44BFB22A
:10C6B0001FFA88F89BB2F92FA2F8028026F83530CD
:10C6C00000D8ABB95E440023B3714FEA28238DF83C
:10C6D000043001AA0223282128468DF80580FFF79F
:10C6E0006DFC4021284600F059FCA2E73A46D3E70A
:10C6F00097719EE7F4060020580800203D070020AF
:10C700007FB5134D064635F83000F8B94FF00043B9
:10C710000193022303908DF8083004AB0D4813E910
:10C720000E0004F03FFD3046FFF7FEFC04463046A5
:10C73000FFF7FAFCA042F9D1064804F03FFD05EBF3
:10C74000C6039879201A80B225F8360004B070BD6F
:10C75000F4060020580800207FB54FF000430193F5
:10C7600000230393104D02238DF8083001AC94E8A8
:10C770000E000646284604F015FD3046FFF7F2FC91
:10C780000A4B03EBC60301225B88C3F30A03184478
:10C79000214680B200F03EFA284604F00FFD9DF8D5
:10C7A000040004B070BD00BF58080020F40600204B
:10C7B0002DE9F04FB2F5006F87B028BF4FF400624B
:10C7C000DFF8E49005468A46164603AC02234FF094
:10C7D00000474FF000080397CDF814808DF8103013
:10C7E00094E80E00484604F0DDFC2846FFF788FC7C
:10C7F00083462846FFF74CFC0190484604F0DEFCD7
:10C80000019B172B01D01C2B32D104F081FAB345C8
:10C81000DCD303974FF000080227CDF814808DF881
:10C82000107094E80E00204804F0BCFC41463346EA
:10C8300052462846FFF7D4FB2021284600F0AEFBE5
:10C84000DFF864804FF0004B02212846FFF78EFB93
:10C8500010F0100A1FD12846FFF71AFC814648B98C
:10C86000114804F0ABFC4E46304607B0BDE8F08FEF
:10C870004646CEE7404604F0A1FC04F049FACDF864
:10C880000CB0CDF814A08DF8107094E80E0040465E
:10C8900004F088FCD8E7102202212846FFF77AFB33
:10C8A000014804F08BFCDFE75808002030B585B064
:10C8B0004FF0004301930023039302238DF80830C7
:10C8C00004AB054613E90E000A4804F06BFC284649
:10C8D000FFF716FC04462846FFF7DAFB0546054835
:10C8E00004F06CFC172D02D01C2D18BF002420462C
:10C8F00005B030BD580800202DE9FF411C464FF01F
:10C900000043019300230393104D02238DF8083058
:10C9100004AB06460F469046284613E90E0004F085
:10C9200041FC3046FFF7ECFB844228BF0446A4B22A
:10C930002346424639463046FFF752FB284604F06C
:10C940003DFC204604B0BDE8F08100BF580800203F
:10C950007FB50B7806460D4614462BB94B781BB9AC
:10C960008B780BB9C878D0B1DCB14FF0004301939C
:10C970000023039302238DF8083004AB13E90E0063
:10C98000094804F00FFC29463046FFF794FB214686
:10C990003046FFF797FB044804F010FC012004B078
:10C9A00070BD2046FBE700BF580800202DE9FF4777
:10C9B00000234FF000480227CDF8048003938DF840
:10C9C000087001AC94E80E0005461F48DFF8789027
:10C9D00004F0E8FB2021284600F0E0FA0221284676
:10C9E000FFF7C4FA10F0100623D102212846FFF702
:10C9F000BDFA10F0080A0BD0182202212846FFF7D2
:10CA0000C9FA114804F0DAFB304604B0BDE8F087FB
:10CA1000484604F0D3FB04F07BF9CDF80480CDF850
:10CA20000CA08DF8087094E80E00484604F0BAFB9C
:10CA3000D4E7102202212846FFF7ACFA024804F09E
:10CA4000BDFB0120E1E700BF5808002007B5002327
:10CA500000931A461946034803F0C0FA03B05DF884
:10CA600004FB00BFEC06002070B505460C468E188E
:10CA7000B44206D02178284604F0A1FB04F8010B4B
:10CA8000F6E770BD024B0021187804F001BB00BF2F
:10CA90000A000020024B0121187804F0F9BA00BF07
:10CAA0000A0000202DE9F3414F4B1B78332B04463D
:10CAB0000D4616461FD100EB02084C4F4D1E1FFAC3
:10CAC00088F8A0457AD0FFF7DDFFF021384604F062
:10CAD00076FB210A384604F072FBE1B2384604F0D6
:10CAE0006EFB013415F8011F3846A4B204F067FB51
:10CAF000FFF7D0FFE5E7342BC7B21DD1FFF7C2FF28
:10CB0000330A241263F07F030422694637488DF804
:10CB100000408DF801708DF802308DF80360FFF74A
:10CB2000A3FF013D314CAF19AF4245D015F8011FAD
:10CB3000204604F044FBF7E7FFF7A4FFFF2C08D8DA
:10CB400000238DF800308DF8017004238DF8023039
:10CB50000DE0230419D4E41024F01F04002344F052
:10CB60000C048DF800308DF801708DF80240052E10
:10CB700028D82A46531BDBB2B34218DA02A8034472
:10CB800012F8011B03F8051CF4E744F3871323F0A4
:10CB90001F03B4F5404F4FEA14228DF800208DF8A2
:10CBA000017034BF43F0140343F01C03CEE7F21CC2
:10CBB00069460E48FFF758FFFFF76CFF304602B09A
:10CBC000BDE8F081032269460848084FFFF74CFF93
:10CBD000731E6C1E15FA83F514F8011F384604F015
:10CBE000EEFAA542F8D1E7E73D07002058080020FB
:10CBF00007B502AB012203F8011D1946FFF752FFEA
:10CC0000C0B203B05DF804FB08B501460020FFF791
:10CC1000EFFF08BD2DE9F3413E4B1B78332B044653
:10CC20000E46154620D100EB02083B4F4E1E1FFA60
:10CC300088F8A0453AD0FFF725FF0F21384604F0C9
:10CC4000BEFA210A384604F0BAFAE1B2384604F0D6
:10CC5000B6FA0021384604F0B2FA013406F8010FA2
:10CC6000A4B2FFF717FFE4E7342BC7B222D1FFF7D6
:10CC700009FF2412C5F3062304228DF804408DF821
:10CC800005708DF806308DF807500DEB0201224833
:10CC9000FFF7EAFE2A460021304606F056FB2A46F8
:10CCA00031461D48FFF7E0FEFFF7F4FE284602B0CC
:10CCB000BDE8F081FFF7E6FEFF2C07D800238DF8D2
:10CCC00004308DF805708DF806300DE023040ED485
:10CCD000E41024F01F04002344F008048DF804300D
:10CCE0008DF805708DF80640032201A9CFE744F3C3
:10CCF000871323F01F03B4F5404F4FEA14228DF839
:10CD000004208DF8057034BF43F0100343F018037E
:10CD1000D9E700BF3D0700205808002007B50122D1
:10CD20000DF10701FFF776FF9DF8070003B05DF8EE
:10CD300004FB08B50020FFF7F1FF08BD10B5802007
:10CD4000FFF762FF1424FFF7F4FF40B1013C01201C
:10CD5000A4B203F0BBFF002CF5D1204610BD01208A
:10CD6000FCE7000008B50F4B33221A70FFF7E6FF0F
:10CD700008B9002008BD1020FFF746FFFFF7D9FFD4
:10CD80001028F6D11220FFF73FFFFFF7D2FF12283D
:10CD9000EFD10020FFF738FFFFF7CBFFB0FA80F0AC
:10CDA0004009E7E73D07002008B5124B34221A700E
:10CDB000FFF7C4FF08B9002008BD0820FFF724FFD3
:10CDC000FFF7B7FF0828F6D11020FFF71DFFFFF788
:10CDD000B0FF1028EFD10020FFF716FFFFF7A9FFE3
:10CDE0000028E8D11F20FFF799FFC31E5842584181
:10CDF000E2E700BF3D07002008B5124B37221A704A
:10CE0000FFF79CFF08B9002008BD0820FFF7FCFED3
:10CE1000FFF78FFF0828F6D11020FFF7F5FEFFF788
:10CE200088FF1028EFD10020FFF7EEFEFFF781FF0B
:10CE30000028E8D13920FFF771FF031F58425841FD
:10CE4000E2E700BF3D0700207FB52D4E3478002C6F
:10CE500053D14FF40C7003F039FF2A4804F08CF9D9
:10CE6000294B0121187804F0EBF8FFF713FE4FF07F
:10CE70000043019302238DF80830039404AB13E9B7
:10CE80000E00204804F08EF9FFF78EFFB0B11F4B63
:10CE900040221A70E5B202221E212846FFF77AF8D6
:10CEA000013402221F212846FFF774F8082CF1D123
:10CEB0001448012404F082F934701BE0FFF79CFF52
:10CEC00018B1124B10221A70F2E7FFF74BFF04461D
:10CED00058B10E4B042255211B201A70FFF788FE13
:10CEE00055211A20FFF784FEE2E7094B1870054828
:10CEF00004F064F9204604B070BD0124FAE700BFD5
:10CF00003E070020580800200A0000203C070020AF
:10CF10003D0700201FB5FFF797FF38B11D4B1B7869
:10CF2000342B4FF0000003D0372B1BD004B010BDC2
:10CF30004FF000430193022303908DF8083004ABB7
:10CF400013E90E00144804F02DF93520FFF7E6FE32
:10CF50000446114804F032F914F0200F14BF0120E8
:10CF60000220E3E74FF000430193022303908DF882
:10CF7000083004AB13E90E00074804F013F92E2023
:10CF8000FFF7CCFE0446044804F018F914F0010F32
:10CF9000E4E700BF3D0700205808002038B50A46E6
:10CFA00001210446FEF7F6FF054D2402287804EB24
:10CFB0000020013080B2FFF7B1FE0028F6D138BD65
:10CFC0003C07002007B5002300931A461946034882
:10CFD00003F004F803B05DF804FB00BF3407002041
:10CFE00014220021103006F0B0B910B510310446FB
:10CFF00003F006F8204610BD10B51431044602F0C7
:10D00000FFFF204610BD10B51831044602F0F8FFAE
:10D01000204610BD10B52031044602F0F1FF204635
:10D0200010BD30204B1C0870110902F00F02092AB4
:10D0300094BF3032373203F801290A460029F3D170
:10D040007047000007B5002300931A4619460348AD
:10D0500002F0C4FF03B05DF804FB00BF40070020EE
:10D060002DE9F0418EB00446884616460021202264
:10D0700006A806F06AF9FF231A461946009302A88B
:10D0800002F0ACFF04F14805554B04934322039B87
:10D09000059304A92846FEF7B7FE013000F09D80F5
:10D0A000504B069363688DF821601BBA0793330ACF
:10D0B0008DF820301C22802306A926462846ADF88C
:10D0C0002230FEF7B0FE1A2200210DF11E0006F0FC
:10D0D0003CF956F8080F0690B388ADF81C301022C2
:10D0E00006A92846FEF79FFE2022002106A806F08A
:10D0F0002CF90627202206A92846FEF794FE013FB8
:10D10000F8D1394B069340F23513ADF81C303D236E
:10D110008DF81F3007238DF8203001238DF8213042
:10D120003368CDF82230B388ADF826302F498DF81A
:10D130001E8040F60C430DF12A00ADF8283007F0B0
:10D1400086F8E27A0CA92046FFF76BFF227B0DF1EF
:10D1500032012046FFF765FF627B0DA92046FFF7ED
:10D1600060FF1E2206A92846FEF75DFEB8F1030FF8
:10D1700024D140F23243ADF81830237C8DF81A30B8
:10D18000637C8DF81B30A37C8DF81C30E37C8DF81C
:10D190001D3040F23643ADF81E30237F8DF820302D
:10D1A000637F8DF82130A37F8DF822300C22E37F3E
:10D1B0008DF8233006A92846FEF735FE0C4A0D4BA4
:10D1C00006A9CDE906232846FF2309228DF8203041
:10D1D000FEF729FE2846FEF720FE0EB0BDE8F081DE
:10D1E0001C9D01000101060063825363549B0100F2
:10D1F00037060103060F3A3B2DE9F04391B005468F
:10D200008846164603F02EFD05F1480407462046E1
:10D21000FEF770FE00280BDC03F024FDC01B404528
:10D2200000F2D280F9F704FF012003F04FFDEEE792
:10D23000242207A92046FEF71AFE9DF81C30022B77
:10D2400040F0BD80B5F86430432B40F0B880089FB3
:10D250003FBA3760062205F108010EA806F042F831
:10D26000064628B92B689F4202D36B689F4207D9B4
:10D270002046FEF768FD0026304611B0BDE8F08379
:10D280000B9B2B610146CC222046FEF7F0FD05F1F9
:10D2900024072046FEF74AFD002840F391802046EF
:10D2A000FEF7CEFD33287DD015DC012844D006DC06
:10D2B0000028EED02046FEF7C3FDC2B253E003289B
:10D2C00044D00628F6D12046FEF7BAFD0422804657
:10D2D00005F1200141E03A284AD020DC352823D04E
:10D2E0003628E7D12046FEF7ABFD05F11C08414684
:10D2F000814601A802F084FE002103A802F07AFE14
:10D30000029A049B9A4230D0414605A802F078FE6A
:10D310002A6E069B9A4228D05FFA89F223E03B28C6
:10D3200033D0FF28B5D0C5E72046FEF789FD20465B
:10D33000FEF786FDC6B2ACE72046FEF781FD04226B
:10D3400005F114012046FEF792FDA2E72046FEF704
:10D3500077FD0422804605F118012046FEF787FD7F
:10D360005FFA88F2043A0021ECE704224146E9E73B
:10D370002046FEF765FD042205F128012046FEF750
:10D3800076FDAB6A1BBAAB6283E72046FEF758FD19
:10D39000042205F12C012046FEF769FDEB6A1BBA59
:10D3A000EB6276E72046FEF74BFD04223946204625
:10D3B000FEF75DFD6B6A1BBA6B622B6369E70026A3
:10D3C0002046FEF7C0FC57E7FF2655E72DE9F34757
:10D3D00004464FF4FA61012003F0C5FA2746606065
:10D3E00047F8480B3846FEF7AFFC44213846FEF7B5
:10D3F000B7FC002800F0908003F034FC4FF00009E7
:10D40000804600254FF0030A94F84430032B1CD0CB
:10D4100043BB63680133636003F024FC4FF47A720A
:10D42000A0EB08000121B0FBF2F2204692B2FFF718
:10D4300017FE012384F84430002DE5D103F012FCDF
:10D44000A36BA0EB08009842DBD93846FEF77CFCC2
:10D4500063680133636003F005FC2064284602B072
:10D46000BDE8F087042B11D163680133636003F0DA
:10D47000F9FB4FF47A72A0EB08000321B0FBF2F243
:10D48000204692B2FFF7ECFD0223D3E7012B19D11E
:10D4900001AAE16B2046FFF7AFFE0228064638D10D
:10D4A000019B636003F0DEFB4FF47A72A0EB08008F
:10D4B0000321B0FBF2F2204692B2FFF7D1FD84F8CF
:10D4C0004460B9E7022BB7D101AAE16B2046FFF710
:10D4D00093FE0528064617D1636A84F844A013B961
:10D4E0004FF461736362A36A13B9636A5B08A36252
:10D4F000E36A1BB9636AA3EBD303E362A36A236302
:10D50000E36A636301257FE7062802D184F844902B
:10D5100092E7FF2EFAD08FE705469FE7F8B5002582
:10D520000F460446C0E90955C562C0E90E2385606F
:10D530008581FFF755FD3B68A360BB88A38184F814
:10D5400044502046BDE8F840FFF740BF10B5044600
:10D5500003F088FB236CC31AB3F57A7F14D34FF41E
:10D560007A71B3FBF1F201FB1233C01A236B206412
:10D5700051008B4234BF00239B1A2363636B994293
:10D580008CBF00239B1A6363206BE0B994F844308E
:10D59000032B06D1042384F844302046FFF716FFFE
:10D5A0000130636B73B994F84430032B00D04BB94E
:10D5B000002384F844302046FFF712FD2046FFF791
:10D5C00005FF033010BD0020EBE74B6843600023EC
:10D5D0000381704770B500240139234611F8010F0B
:10D5E000B8B1A0F13005EEB2092E08D803EB8303E1
:10D5F00005EB43039BB2FF2BF0D900200DE02E2852
:10D60000FBD1032CF9D0601C14442371C4B2002355
:10D61000E4E7032C01D1D371012070BD07B50023CD
:10D6200000931A461946034802F0D8FC03B05DF88F
:10D6300004FB00BF480700202DE9F74305460E46CE
:10D6400003F010FB05F10C04288105F1080102220A
:10D6500002AD2046FEF7E7FB012325F8023D02223A
:10D6600029462046FEF7DFFB4FF48073022229464D
:10D670002046ADF80630FEF7D6FB002302222946ED
:10D680002046ADF80630FEF7CEFB022229462046A2
:10D69000FEF7C9FB022229462046FEF7C4FB3746A7
:10D6A0003378E3B13E46B04618F8013B0BB12E2B60
:10D6B00013D1A6EB0709B9F1000F0CDD01220DF122
:10D6C000050120468DF80590FEF7ADFB4A46394628
:10D6D0002046FEF7A8FB4746E2E74646E3E702A9F5
:10D6E000012201F8033D2046FEF79DFB4FF48076B2
:10D6F000294602222046ADF80660FEF794FB02227E
:10D7000029462046ADF80660FEF78DFB012003B0E8
:10D71000BDE8F0832DE9F04387B006460F469046FA
:10D7200003F0A0FA06F10C0405462046FEF7E2FBE2
:10D73000002808DC03F096FA401BB84200F2C480CF
:10D74000F9F776FCF1E7726A73689A4240F0BF809D
:10D75000338D352B40F0BB802046FEF7E7FA0B28CF
:10D7600040F3B8800C220DEB02012046FEF77FFB50
:10D77000BDF80E203189130A43EA0223BDF80C20BC
:10D780001BB29DB29142ADF8065001D1002B07DBD0
:10D790002046FEF7D8FA4FF6FC7007B0BDE8F083DC
:10D7A00040F20F231D4005D02046FEF7CCFA4FF67D
:10D7B000FB70F2E7BDF812301F0A47EA0327BFB239
:10D7C0002FB92046FEF7BFFA4FF6FA70E5E7BDF82D
:10D7D00010305BBAAAB29BB29A4216DA01220DF15E
:10D7E0000A012046FEF743FB9DF80A201AB10021EA
:10D7F0002046FEF73CFB9DF80A100029EED10422DA
:10D800002046FEF734FB0135E1E70026B146012250
:10D810000DF105012046FEF72AFB9DF8052012F0C8
:10D82000C00134D112B12046FEF721FB9DF805500E
:10D83000002DECD1022202A92046FEF718FB02229D
:10D840000DF10A012046FEF712FB0422294620466C
:10D85000FEF70DFB02220DF106012046FEF707FB45
:10D86000BDF80830BDF80620B3F5807F52BA92B2F9
:10D870001CD1BDF80A0040BA85B2012D16D1042A88
:10D880000DD02046FEF75FFA4FF6F77085E70122CC
:10D8900000212046FEF7EBFA8DF80590C6E708F167
:10D8A00004012046FEF7E3FA284676E70136002118
:10D8B0002046B6B2FEF7DBFAB742A8D12046FEF703
:10D8C00042FA4FF6F67068E74FF6FF7065E74FF6DD
:10D8D000FE7062E74FF6FD705FE700002DE9F34749
:10D8E00005468A4691469846FFF774FE0446B8BB43
:10D8F0001E4B6A685B689A4234D003F0B3F905F1B5
:10D900000C0600F00F0101F580613046FEF728FAA1
:10D910000128074620D1164B009335226B680193EE
:10D9200069463046FEF770FA98B151462846FFF72F
:10D9300083FE70B13046FEF770FA50B14A46414658
:10D940002846FFF7E7FE0446F9F772FB384603F076
:10D95000BDF93046FEF7F8F9204602B0BDE8F08781
:10D960000124F9E76FF00104F6E700BF4807002043
:10D970001C9D010007B5002300931A461946034871
:10D9800002F02CFB03B05DF804FB00BF5007002041
:10D99000006903681B691847006903685B691847D9
:10D9A00013B5006949680368034C01919B690094B1
:10D9B0006946984702B010BD1C9D010000690368CC
:10D9C000DB691847006903689B6A184700690030E3
:10D9D00018BF01207047006C70470164704710B594
:10D9E00090F83830044633B920690368DB689847FB
:10D9F000002808DA10BD03689B6898470028F3D117
:10DA00004FF0FF30F6E794F82220A2F10803022B32
:10DA1000F0D8A36A002BC2BFE36A0133E3620A2A8B
:10DA2000E8D1E36B013BE363002BE3D1092384F8E6
:10DA30002230DFE710B50446006903681B6A984787
:10DA400094F82230083B022B07D8A36A002B04DD90
:10DA50000028A2BFE36A1B18E36210BD73B590F8FB
:10DA60002230092B04460ED10026206903689B68EA
:10DA7000984740B120690368DB689847C5B20A2D12
:10DA80001CD184F8225094F822300A2B04D1E36B85
:10DA900013B9092384F8223094F82230092B22D0BC
:10DAA000206903689B68984794F822300A2B03D1B9
:10DAB000E36B9842A8BF184602B070BD0D2DD4D0BC
:10DAC000284605F0B8FB0028CFD0E06BADF8046025
:10DAD00010228DF804500021050101A807F046FB33
:10DAE0002844E063C1E70020E6E7000000234FF090
:10DAF000FF32C0E90A23084A80F822301268026324
:10DB0000064A4362126880F83830C36347F23053E4
:10DB100042630364704700BF10000020140000201F
:10DB200038B504461D4600204FF47A73C4E901035A
:10DB30000B4B2360C4E9041204F1180002F046FA0A
:10DB40000123258484F8443084F84530054904F1E4
:10DB5000480002F061FF2046FFF7C8FF38BD00BF54
:10DB6000BC9B0100729C010010B50446006903686B
:10DB70005B6A98472046BDE81040FFF7B7BF012316
:10DB800080F822307047000038B504460069154619
:10DB900002F075FA0449206902F071FA29462069F9
:10DBA000BDE8384002F082BA017E010038B5044673
:10DBB0000D460069114602F062FA1D49206902F023
:10DBC0005EFA2946206902F05AFA1A49206902F0E1
:10DBD0006DFA94F84530F3B16369B3B11649206921
:10DBE00002F04DFAD4E9040102F049FA238C502BDB
:10DBF00008D01249206902F042FA0A22218C2069D9
:10DC000002F09DFA206902F041FA0D4B0D491A68A5
:10DC10002046FFF7B9FF94F8443023B10A4A0B4974
:10DC20002046FFF7B1FF012384F82230002038BDE1
:10DC3000247F0100819B01008B9B01008A800100F1
:10DC40000C000020929B01009D9B0100A39B010002
:10DC500038B504460069154602F011FA05492069F5
:10DC600002F00DFA294620690A22BDE8384002F088
:10DC700068BA00BF017E010010B50446006902F0D9
:10DC800005FA022384F8223010BD70B590F82230D6
:10DC9000012B04460D46164601D8FFF7EDFF20691B
:10DCA0000368324629465B68BDE87040184770B586
:10DCB00090F82230012B04460D4601D8FFF7DCFF17
:10DCC0002069036829461B68BDE87040184710B5F5
:10DCD0000446206903689B68984720B1206903685F
:10DCE000DB689847F5E710BD2DE9F347994690F8B2
:10DCF0002230083B022B04460E469246DDE90A78A4
:10DD000004D8FFF7E4FF2046FFF7F0FE94F8225016
:10DD1000012D45D894F844305BB1D4E90401228C3C
:10DD20000368B9B921490091E16901919B6969468C
:10DD300011E0206903689B6A98470028EDD03146BE
:10DD400052462046FFF732FF064650B1304602B039
:10DD5000BDE8F087DB6998470028F0DC4FF0FF361C
:10DD6000F4E7B9F1000F04D04A4611492046FFF705
:10DD70000BFF002F17DD3A460E492046FFF768FFDC
:10DD8000B8F1000F0FD001252046FFF775FF002DD9
:10DD9000DCD023683A465B68414620469847D5E781
:10DDA0006FF00106D2E7002DD0D1EDE71C9D0100F8
:10DDB0005B9B0100689B010090F82230012B01D889
:10DDC000FFF75ABF7047FFF7F7BF000007B5002302
:10DDD0004FF0FF32CDE90023024AFFF785FF03B081
:10DDE0005DF804FBAE9B01002DE9F04790F822306E
:10DDF000012B044651D9DFF8D880002503270023E2
:10DE00006362022384F8223002F02CFF46468246E9
:10DE10004FF00A090A2D46D002F024FF236CA0EB34
:10DE20000A00984245D2236820469B68984748B329
:10DE300023682046DB689847431C0546ECD094F8DD
:10DE40002230022B05D0032B0FD002F00BFF8246AD
:10DE5000E0E733782A2B01D083421AD17278731C01
:10DE60000AB984F822701E46EFE7A0F13002092AB1
:10DE700095BF636A042309FB032384F8223098BF0B
:10DE80006362E2E74FF47A7002F020FFC2E70A2DE6
:10DE900006D16FF00300BDE8F0876FF00100FAE7EC
:10DEA0006FF00200F7E7636AC72B02DC652B18BF2F
:10DEB000002594F82230042BE9D1606AC72801DCE0
:10DEC00065289CD10A2D18BF6FF00200E3E700BF60
:10DED000779B010038B501F1480504463A212846F0
:10DEE00002F07AFE421C034605D10649204602F0A4
:10DEF00093FD204638BD00222946204602F08AFEC6
:10DF0000F7E700BF729C0100F8B501F1480605462D
:10DF10000F4630463A2102F05FFE441C013005D125
:10DF20000C49284602F078FD2846F8BD3B6DA34217
:10DF300009DD2146304602F033FE007805F072F923
:10DF400008B10134F2E73B6D22463146284602F023
:10DF500061FEE9E7729C010010B503680446DB68C6
:10DF6000984794F82230A3F10802022AC0B232D9AD
:10DF7000052B31D0072B39D0042B54D1226B1378C9
:10DF800083420BD1531C2363537823B9C4E90A336A
:10DF9000052284F822200A281DD136E0636B197807
:10DFA00081420BD15A1C62635B78002BF3D10123B1
:10DFB00084F83830062384F82230ECE71B490968DE
:10DFC0008A42F7D11A4A12689342F3D10D28F1D14F
:10DFD000072384F8223010BDA0F13002092AE9D8C5
:10DFE000A36A0A2101FB0323A362D4E70A28F2D122
:10DFF00094F838309BB1092384F822300023E3637E
:10E0000094F82230083B022BE5D9042384F822300F
:10E01000064B1B682363064B1B686363DBE708231F
:10E0200084F82230ECE70A28D5D1E9E71000002077
:10E030001400002038B5044602F014FE054694F89A
:10E040002230083B022B13D902F00CFE236C401B3C
:10E0500098420DD2236820469B68984718B1204605
:10E06000FFF77AFFE8E74FF47A7002F02FFEE6E759
:10E0700094F82230083B022B94BF00206FF002007E
:10E0800038BD10B590F82230083B022B044601D968
:10E09000FFF7D0FFA06A10BD38B590F82230083BDA
:10E0A000022B054601D9002038BDFFF7EAFF0130F9
:10E0B000F9D02846EC6AFFF7E4FF8442B4BF0020A1
:10E0C0000120F1E7FFF7E8BFFFF7E6BF38B500F141
:10E0D000480504460E49284602F0FBFC94F822301D
:10E0E000083B022B09D92046FFF736FF0D2801D047
:10E0F0000A2807D1236D002BF0D0206D003018BF07
:10E10000012038BDC1B2284602F004FDE6E700BF99
:10E11000729C010007B5002300931A461946034874
:10E1200001F05CFF03B05DF804FB00BF680700204E
:10E1300080687047C1607047036810B59B690C46E2
:10E140009847036821461B68BDE8104018472DE931
:10E15000F84380460D46174601EB02090C46A145DF
:10E16000A4EB050609D0D8F800304046DB68984794
:10E17000431C03D004F8010BF1E73E463046BDE8EE
:10E18000F883C368013310B5044612D123682046D2
:10E190009B69984703689B68984758B12368204655
:10E1A000DB6898472028F1DD2368C1B25B6920460F
:10E1B0009847012010BD70B50446C068431C18D1B3
:10E1C00002F050FD00F5FA75236820469B699847D8
:10E1D00003689B68984718B902F044FD8542F3D85C
:10E1E000236820469B6998470368BDE87040DB6858
:10E1F00018474FF0FF33E36070BD10B5182005F0ED
:10E200004FF8044618B11822002105F09EF8204668
:10E2100010BD70B506460C46D4B1237C65681B075B
:10E2200004D4E16811B13046FFF7F3FF237C03F01B
:10E230000F03042B03D1606908B100F005FD2068CD
:10E2400008B100F001FD204605F032F82C46E3E766
:10E2500070BD00002DE9F04F036885B0DB6805460E
:10E260000E469847421C044604D14FF0FF3005B0DB
:10E27000BDE8F08F2D282FD12B682846DB68984702
:10E28000431C0446F1D04FF0FF330093A4F1300358
:10E29000092B4FF000070DD84FF00A082B682846CD
:10E2A000DB689847A0F13003303C092B08FB074797
:10E2B0000446F3D92E2C11D024F02003452B0DD089
:10E2C000009B7B437361022333742B6828465B6990
:10E2D000E1B298470020CAE70123D6E7384604F0A8
:10E2E000DBF92E2C8046894639D12B68DFF814B132
:10E2F000DB6828469847002704464FF0000A52463C
:10E300005B464046494604F031FA80468946A4F10E
:10E31000300004F0C1F942464B4604F071F82B6816
:10E320008046DB68284689469847A0F13003092BD0
:10E3300007F1FF370446E2D924F02003452B2AD108
:10E340002B682846DB6898472B28044609D12B68A0
:10E350002846DB68984704464FF0010A0AE0002788
:10E36000EAE72D28F8D12B682846DB6898474FF05C
:10E37000FF0A04464FF0000B0A22A4F13003092BD8
:10E380000DD802FB0B3B2B680392DB6828469847AD
:10E39000039A0446F1E74FF0010A4FF0000B009892
:10E3A00004F07AF942464B4604F0E0F9CDE9000169
:10E3B000584604F071F980465046894604F05CF9ED
:10E3C00002460B464046494604F0D0F9804638469E
:10E3D000894604F061F902460B464046494604F07E
:10E3E0000FF802460B460020064902F029FF0B46B3
:10E3F0000246DDE9000104F0B9F904F0AFFC0323A3
:10E40000706161E70000244019B10A22496901F0F6
:10E4100074BE084670470000F8B504462DED028B27
:10E4200000295AD091ED058A18EE100A04F046F939
:10E43000B5EEC08AF1EE10FA06460F4606D52C4915
:10E44000204601F01CFE07F100431F4639463046C6
:10E4500004F064FC0A2205460146204601F07BFEDA
:10E460002449204601F00BFE284604F005F9024637
:10E470000B463046394603F0C1FF1BA3D3E9002306
:10E4800003F0BEFF1C4B002204F070F90F46064655
:10E4900004F044FC0A2201460546204601F06AFECB
:10E4A000284604F0E9F802460B463046394603F0A8
:10E4B000A5FF0022002306460F4604F0BFFB60B90B
:10E4C00000220D4B3046394604F050F904F026FC8A
:10E4D0000A220146204601F04DFEBDEC028B0020D1
:10E4E000F8BD00BFAFF300807B14AE47E17A743F04
:10E4F000B3A101006192010000002440F8B5036857
:10E50000DB6806460F469847222803D04FF0FF34B9
:10E510002046F8BD04233B7400F006FB05460028A6
:10E52000F4D033683046DB689847431C044611D06A
:10E53000222C36D01F2C34DD5C2C04D02946E0B2CE
:10E5400000F008FBEDE733683046DB689847421C73
:10E55000044603D1284600F009FBD9E7622817D00A
:10E5600007DC2F2803D05C2801D02228D9D12946E6
:10E57000E6E76E280FD004DC6628D2D129460C20AD
:10E58000DEE772280AD07428CBD129460920D7E7C4
:10E5900029460820D4E729460A20D1E729460D203C
:10E5A000CEE7284600F024FB00247861B0E70000A5
:10E5B00038B50D461D49044601F061FD7DB3013DAE
:10E5C00015F8011F59B31F2907D9222905D05C2945
:10E5D00003D0204601F057FDF2E75C21204601F010
:10E5E00052FD29780C2914D007D8092915D00A29F9
:10E5F00011D00829E4D16221EBE72229E9D003D820
:10E600000D29DDD17221E4E72F29E2D05C29E0D089
:10E61000D6E76621DDE76E21DBE77421D9E7222109
:10E62000204601F030FD002038BD00BF047E01000F
:10E630004969FFF7BDBF38B50368DB6804469847F2
:10E640004FF48075411C0FD020280EDC013D6A1C60
:10E65000236803D0DB6820469847F3E72368C1B2FC
:10E660005B6920469847002038BD002DF6D14FF059
:10E67000FF30F9E703682DE9F047DB680446884678
:10E68000914698477B2803D04FF0FF30BDE8F087D4
:10E69000062388F810302046FFF7CDFF2368204678
:10E6A000DB6898477D2843D02368C1B25B69204668
:10E6B0009847FF264FF0000AFFF79FFD0546002808
:10E6C000E2D096B3C8F80C002046FFF7B4FF294605
:10E6D0002046FFF713FF0130D6D02046FFF7ABFFEF
:10E6E0006B692B602368C5F814A0DB682046984747
:10E6F0003A28C9D12046FFF79EFF4A4629462046C0
:10E7000000F018F80130BFD02046FFF794FF2368CF
:10E710002046DB6898472C282F464FF00006CBD0C8
:10E720007D3818BF4FF0FF30B0E778608760CBE7E7
:10E730000020ABE7F7B504460E461746FFF77BFF10
:10E74000013002D14FF0FF3011E023682046DB6832
:10E750009847431C0546F5D02368C1B25B69204643
:10E760009847222D05D131462046FFF7C7FE03B05A
:10E77000F0BD2D2D03D0A5F13003092B04D831466F
:10E780002046FFF767FDF2E75B2D05D13A4631469B
:10E79000204600F078F8EAE77B2D05D13A4631466D
:10E7A0002046FFF767FFE2E76E2D15D102AD00238B
:10E7B00045F8083D236804221B69294620469847EE
:10E7C00004280246BED11D49284605F080FD0028D8
:10E7D000B8D100233374CAE7662D16D10023009305
:10E7E0008DF80430236805221B6969462046984746
:10E7F0000528A7D105221249684605F068FD0028C2
:10E80000A0D1012333743075B1E7742D9AD102ADD4
:10E81000002345F8083D236804221B692946204649
:10E820009847042802468DD10649284605F04FFD39
:10E83000002887D101233374337598E7369C010093
:10E840003B9C0100419C0100F8B5064617460D4669
:10E8500011B900242046F8BDFFF7CFFC044600287C
:10E86000F7D02846FFF7E7FE3A4621462846FFF74D
:10E8700061FF0130EED121463046FFF7CAFCE8E7E0
:10E880000022FFF7E1BF2DE9F8430368DB68044687
:10E890008846914698475B2803D04FF0FF30BDE88B
:10E8A000F883052388F810302046FFF7C4FE23685C
:10E8B0002046DB6898475D282AD02368C1B25B698F
:10E8C00020469847FF26FFF798FC05460028E4D02D
:10E8D000DEB1C8F80C002046FFF7ADFE4A462946D7
:10E8E0002046FFF727FF06460028D6D12046FFF72F
:10E8F000A2FE23682046DB6898472C282F46E2D0EA
:10E900005D3818BF4FF0FF30C9E778608760E2E7F5
:10E910000020C4E770B505461646002935D0CC68FE
:10E920007B2101F0B0FB013002D14FF0FF3070BD10
:10E9300034B1216876B90B78402B0BD16468E4B907
:10E940007D21284601F09FFB01304FF0FF3018BFBA
:10E950000020ECE72846FFF72BFE0130E5D03A21F6
:10E96000284601F090FB0130DFD032462146284690
:10E9700000F00EF80130E1D1D7E71EB923681B780B
:10E98000402BD5D02C212846CBE70846CFE7000006
:10E99000E9B10B7C03F00F03062B18D8DFE803F076
:10E9A00004070D0F111315000A4901F068BB0B7D18
:10E9B0000BB10949F9E70949F7E7FFF725BDFFF76B
:10E9C0002BBDFFF735BE00F00FB8FFF7A3BF002047
:10E9D000704700BF369C0100419C01003B9C010038
:10E9E00010461A46FFF7D4BF70B505461646F9B172
:10E9F000CC685B2101F047FB013002D14FF0FF30C2
:10EA000070BD5CB1324621462846FFF7C1FF013098
:10EA1000F4D0646814B12C212846EBE75D21284628
:10EA200001F031FB01304FF0FF3018BF0020E7E765
:10EA30000846E5E731B1CB680022D0B2013213B10C
:10EA40005B68FAE70846704731B1C96821B11AB16D
:10EA5000013AD2B24968F9E70846704738B5154619
:10EA60000C4641B1CC6834B12946206805F0ABFBB7
:10EA700008B16468F7E7204638BD51B14AB1CB68A8
:10EA800013B9CA6070470B4659680029FBD15A6018
:10EA900093607047F8B505460E4617461C4673B19D
:10EAA000186808B100F0D0F8384600F077F8224630
:10EAB000206031462846BDE8F840FFF7DEBFF8BDCC
:10EAC00008B5FFF79AFB18B1037C6FF303030374D7
:10EAD000037C6FF30713037408BD10B50C46FFF7F2
:10EAE0008CFB10B102230374446110BD70B50D4658
:10EAF000194604461646FFF7F0FF324603462946FC
:10EB00002046BDE87040FFF7C5BF000007B50023F1
:10EB100000931A461946034801F060FA03B05DF805
:10EB200004FB00BF7007002038B50C2004F0B8FBD0
:10EB3000044650B1064820604FF480752A460021F3
:10EB400004F003FC00236560A360204638BD00BFCD
:10EB500084080020D1E90132013B9A4204D20B68BB
:10EB600098548B6801338B600020704708B104F023
:10EB70009FBB704738B5054658B1074C216819B19D
:10EB8000284605F05AFB10B1A468002CF6D12046A7
:10EB900038BD0446FBE700BF7C070020F8B50746F8
:10EBA000FFF7E8FF20B10379013303710068F8BD76
:10EBB0000E4D2B6843B9384605F052FB01232860FF
:10EBC0002B71F4E73546F4E7AE68002EFAD10C203D
:10EBD00004F066FB04460028E9D0A860384605F03A
:10EBE0003FFB012320602371A660E0E77C07002043
:10EBF000826838B5044622B10368134413F8013C17
:10EC00001BB121460020FFF7A5FF0548FFF7C6FF0F
:10EC1000054610B1204604F04BFB284638BD00BF26
:10EC20008408002010B5074CA06800B910BD026828
:10EC3000836822B9A36004F03BFBA3682046044626
:10EC40001846F2E77C07002038B5FFF793FF05462A
:10EC500060B10479013CE4B204713CB9006804F08D
:10EC600027FB2C60BDE83840FFF7DCBF38BD000053
:10EC700008B5064B1B7843B9054801F007FA05496A
:10EC80000348BDE8084001F0F1B908BDCD070020F8
:10EC9000E00700206C9C0100F0B504789FB00546A9
:10ECA0004CB31C4B1C4F1B68986804F0A9F928460C
:10ECB000194906F079F91EAD012445F8780D394659
:10ECC000002006F071F91E2C264645F8240002D0DB
:10ECD00001340028F3D1114B009F1C6884B12168D6
:10ECE000384605F0AAFA48B963682946304698477D
:10ECF0000446FFF7BDFF20461FB0F0BDA468EDE756
:10ED0000074B1B78002BF6D10649074801F0C4F9E0
:10ED1000EFE700BF38000020247F0100C807002073
:10ED2000CD070020739C0100E0070020F8B50546E0
:10ED30000C200F4604F0B4FA0C4B04461860284629
:10ED400005F0A9FA013004F0ABFA2946064605F0B1
:10ED50007EFA284605F09FFA00233354044B1A68C4
:10ED6000A260C4E900671C60F8BD00BFC8070020AE
:10ED700088070020184B1B7870B5FBB91748184D51
:10ED800001F0D2FCC4B20A2C0CD00D2C0AD0082CF5
:10ED900015D12146114801F076F92B7873B1013B6A
:10EDA0002B700BE02B780F4E0F490C480024F454C5
:10EDB00001F065F93046FFF76FFF2C7070BD2146FA
:10EDC000064801F060F92B783A2B9FBF5A1C2A7035
:10EDD000044AD454F2E700BFCD070020E00700202A
:10EDE000CC0700208C070020709C0100064B1B788C
:10EDF00010B53BB9054C204601F090FC10B1FFF76F
:10EE0000B9FFF8E710BD00BFCD070020E0070020E4
:10EE1000054A00231370054A0146136010B10448E7
:10EE200001F03CBC704700BFCC07002088070020E1
:10EE3000E007002070B504460D4601F013FFA06105
:10EE4000A068036829461B68BDE87040184770B584
:10EE500004460D46164601F005FFA061A068036850
:10EE6000324629465B68BDE87040184710B5044635
:10EE7000C06804F01DFA204610BD2DE9F04105469A
:10EE80000E4601F0EFFE4FF47A778046A8680368DB
:10EE90009B689847044658B901F03AFF01F0E2FE3A
:10EEA000AB8AA0EB08007B439842EFD3204605E0F5
:10EEB000A8680368DB68984730700120BDE8F081DE
:10EEC00038B5148821441546FFF7D7FF08B101343F
:10EED0002C8038BD2DE9F74F02AD002625F8026DD4
:10EEE0008A462A46C1680446FFF7EAFF18B900209F
:10EEF00003B0BDE8F08FE3680DF1080993F80080D6
:10EF000009F8036D0127BDF80630052B07D14FF036
:10EF1000FF33A068E36303685B6A9847E7E7494605
:10EF20002046FFF7AAFF0028E1D0BDF80630E268CE
:10EF3000591CADF806109DF80510D1549DF8053008
:10EF400003F07F0207FB02661A064FEAC717DAD4FE
:10EF50009DF8063008F0F008013BB8F1300F8AF850
:10EF600000301DD12A46E1682046FFF7A9FF00289E
:10EF7000BDD02A46E1682046FFF7A2FF0028B6D0A0
:10EF8000E2689AF80030134459789D78137805EBBD
:10EF900001259B07ADB201D50235ADB2022701E0D4
:10EFA00000273D46BDF806B0A7EB0B0707EB0B02A9
:10EFB00096422AD949462046FFF75FFF002896D09F
:10EFC000A06B88B1B8F1300F0ED19AF80020C2F1D1
:10EFD000FF2202F57F02FE325A44AA4204D9026897
:10EFE0009DF8051012689047BDF80620218A9142CD
:10EFF00008D9E1689DF805008854BDF80620013263
:10F00000ADF806200BF1010BD0E7A26B22B9218AE3
:10F01000594538BFADF80620BDF8060068E7012065
:10F02000704773B50025DC1103F07F06A3B20CB165
:10F0300046F080060DF1080C681C6544C0B205F866
:10F04000046C0546002CEED1C0F10405515501AD0C
:10F05000A04205DD231A1344615D59710134F7E7BD
:10F06000013002B070BDF8B5064617461C46FFF7E2
:10F07000D8FFB368C0B21A680444C0F105015568EE
:10F08000394422461846A847054601F0EBFDB06119
:10F09000A8B2031B58425841F8BD10B5C368E0221E
:10F0A0001A70C36800225A7004468068E1680368D9
:10F0B00002225B689847A0684FF0FF33E363036860
:10F0C0005B699847A06803685B6A984701F0CAFDCE
:10F0D000C4E9060010BD023330B598B20C46631A7D
:10F0E00014F8015B9BB21DB1431C155498B2F6E7AE
:10F0F000C11A0A44191202F8021C02F8013C30BD80
:10F1000038B50546806808B9002038BD03689B6A99
:10F110009847EC6B68B9002CF6D1A8686FF0020331
:10F12000EB6303685B699847A86803685B6A984764
:10F13000EAE7B4FA84F04009E7E700002DE9FF4769
:10F140000C9D9DF840A00446894617461E46FFF7D1
:10F15000D7FF8046002840F0DF80A06803689B6AE4
:10F160009847002840D00123E3826E4B029345F27A
:10F170005443ADF80C3004238DF80E30052302A95A
:10F180001944E26811F8051CD15401330C2BF6D157
:10F19000002D3DD09DF838309DF834205B0143F0C0
:10F1A000040343EAC203DBB2BAF1000F01D043F01B
:10F1B00002031FB1002E2DD143F08003E2681373C8
:10F1C000638AE2681B125373E368628A9A73218A26
:10F1D000484605F0A3F8238A113098421DD9A0684B
:10F1E00003685B6A984797E0A068216B0368A28E6A
:10F1F00039B1DB6998470128B5D06FF00103E363AB
:10F200008AE049499B690291E16A039102A9F1E709
:10F210002B46C9E743F0C003D0E749460F23E26815
:10F220002046FFF758FF814605B3218A284605F09E
:10F2300075F809F102031844238A9842CFD84B4647
:10F240002946E2682046FFF746FF218A05460F98C7
:10F2500005F064F8238A023028449842BFD82B4630
:10F26000E2680F992046FFF736FF814617B3218ADF
:10F27000384605F053F809F102031844238A9842EE
:10F28000ADD84B46E26839462046FFF724FF814659
:10F2900086B1218A304605F041F809F1020318448D
:10F2A000238A98429BD84B46E26831462046FFF7B6
:10F2B00012FF8146A9F105039BB2E26810212046A6
:10F2C000FFF7D1FE01F0CEFCC4E906004FF47A75D9
:10F2D000A06803689B68984758B901F0C3FCE369CC
:10F2E000C01AA38A6B439842F2D36FF00303E3631F
:10F2F00075E70DF107012046FFF7ECFD04287FF4C8
:10F300006EAFE368DD785DB901F0ACFC4FF0010849
:10F31000E06184F82050E563404604B0BDE8F08722
:10F32000E5635CE700044D511C9D010010B586B0FB
:10F33000012404940B9C03949DF8284002949DF8AA
:10F3400024400194089C0094FFF7F8FE06B010BD1D
:10F350002DE9F3470446FFF7D3FE8046D0B101F014
:10F3600081FC628A4FF47A735343E269821A9A42AB
:10F37000074603D8A269821A93421FD294F820301C
:10F3800063B16FF00303A068E36303685B6A9847A7
:10F390004FF00008404602B0BDE8F087E268C021A7
:10F3A0001170E2685370A068E168036802225B682C
:10F3B0009847C4E90677012384F82030A0680368E1
:10F3C0009B6898470028E5D00DF107012046FFF71C
:10F3D00081FD83B20646002B73D0E368E7611A789B
:10F3E00002F0F002302A57D1626A002AD2D09DF88A
:10F3F00007209918901C49781D5C05EB0125ADB2DA
:10F40000D11C19442A46184403F086FFE3689DF88E
:10F4100007202B44134400229A70E1689DF807C02E
:10F4200091F8009009F00609B2B20CF10200B9F1AE
:10F43000020F0844666A0CF10303A2EB0C0225D10B
:10F440002B440CF1050C11F803E00B44521B93F80C
:10F4500001A06544053A29440AEB0E2AB047E36847
:10F4600040221A70E36883F80190E3681FFA8AFA71
:10F470004FEA2A229A70E36883F803A0A068E16843
:10F48000036804225B689847A76183E72B44033A2B
:10F49000521B1944B0477DE7C02A0BD1D0221A7005
:10F4A000E36800225A70A068E168036802225B6882
:10F4B00098476FE7D02A7FF46DAF002384F820309F
:10F4C00068E72046FFF71CFE002808BF4FF0000841
:10F4D00060E770B590B005460E46FFF711FEE0B14B
:10F4E000304604F0D8FE3123C4B28DF80030A31C9E
:10F4F0008DF801303B220023314601A88DF80230FF
:10F500008DF8034004F0F5FE2B68221D5B68694608
:10F5100028469847003018BF012010B070BD2DE973
:10F52000F0470446884617461D469DF82060FFF7C1
:10F53000E7FD50B3B4F810904046494604F0EEFEA3
:10F54000EB1D1844814520D341460523E26820463F
:10F55000FFF7C1FD00211FFA81FC4318AC459BB2A7
:10F56000E26801F1010104D217F80CC002F803C0EF
:10F57000F1E7002EA3F1050320469BB214BF312111
:10F580003021BDE8F047FFF76EBD0020BDE8F087F1
:10F5900073B505460E4614466AB1018A104604F05A
:10F5A000BDFE034600220092314622462846FFF760
:10F5B000B6FF02B070BD1346F4E7F7B505460E4638
:10F5C0001F46144662B1018A104604F0A7FE0346A6
:10F5D0000097224631462846FFF7A1FF03B0F0BD51
:10F5E0001046F4E72DE9F0470446884692461E4649
:10F5F000FFF786FD002843D0218A404604F08EFEA6
:10F600009DF82030002BE3680CBF3022312287B2F6
:10F610001A70B21C3A44012002F07F01E568D20959
:10F6200018BF41F08001431C29545FFA80F9D2B918
:10F6300041469BB2E2682046FFF74DFDA368E168B2
:10F640001A68D2F8048002461846C04755468046DC
:10F65000B244AA4509D0A06815F8011B03681B68CD
:10F6600098478044F5E71846D6E701F0FBFAA06119
:10F6700009F1030038443044A0EB080358425841D4
:10F68000BDE8F087F7B505460E461F46144662B141
:10F69000018A104604F042FE034600972246314696
:10F6A0002846FFF79FFF03B0F0BD1046F4E7F8B51A
:10F6B00005460E4614461F46FFF722FD28B3314685
:10F6C0000523EA682846FFF706FD631F002F034461
:10F6D0000CBF3021312106469BB2EA682846FFF76D
:10F6E000A0FC0146A868EC680368053E0E44C1F121
:10F6F00005015B68214432469847044601F0B2FA9E
:10F70000A861A0B2831B58425841F8BD70B50D46A0
:10F710000446018A2846164604F000FE45B3012E31
:10F7200026D8238A0930834222D32046FFF7E8FCFB
:10F73000F0B1E38A01339BB2C3B1E382E38AE268AA
:10F740001B125371E368E28A9A71E2682946072323
:10F750002046FFF7C0FCE3681E54031FE268204602
:10F760009BB28221BDE87040FFF77DBC0123E4E736
:10F77000002070BD0022FFF7C9BF70B50D460446DA
:10F78000018A284604F0CAFD25B3238A0930834242
:10F7900020D32046FFF7B4FCE0B1E38A01339BB2EB
:10F7A000B3B1E382E38AE2681B125371E368E28A31
:10F7B0009A71E268294607232046FFF78CFC431F15
:10F7C000E26820469BB2A221BDE87040FFF74BBC27
:10F7D0000123E6E7002070BD016382867047416225
:10F7E0007047C06B704738B504460D4609B9002014
:10F7F00038BD038A4BB9084603F052FDE060E0686B
:10F800002582003018BF0120F2E7C06804F020FC18
:10F810000028F3D1EBE7000070B50C4B002504463F
:10F82000456040F8283B0E4600F0D0FB4FF0FF3318
:10F83000E363A660A56325824FF480712046FFF73D
:10F84000D2FF0F236382A382204670BD8C9C0100EF
:10F8500007B5002300931A461946034800F0BEFB83
:10F8600003B05DF804FB00BFD00700208271054A99
:10F87000417112680449B2FBF1F14FF47A724A43C4
:10F88000C26070471800002040420F0038B504469F
:10F890000D464079022101F0D3FB01F0E3F9A0F518
:10F8A000FA60A060657438BD70B505460E46002448
:10F8B000687901F0FFFBB042A3B206D1EA689A4230
:10F8C00004F10104F4D84FF0FF33184670BD30B591
:10F8D0000D46D1B0044601F0C5F93DB9A368C31A7D
:10F8E000B3F5FA6F02D2207C51B030BD0025022161
:10F8F000A06025606079257101F0A2FB012001F074
:10F90000E5F90121607901F09BFB2946607901F05E
:10F91000BFFBA379153B012B00F28C8040F24C40D9
:10F92000013800BF00BF00BF00BF00BF00BF00BF65
:10F9300000BF00BF00BF00BF00BF00BF00BF00BFCF
:10F9400000BF00BF00BF00BF00BF00BF00BF00BFBF
:10F9500000BF00BF00BF00BF00BF00BF00BF00BFAF
:10F9600000BF00BF00BF00BF00BF00BF00BF00BF9F
:10F9700000BF00BF00BF00BF00BF00BF00BF00BF8F
:10F9800000BF00BF00BF00BF00BF00BF00BF00BF7F
:10F9900000BF00BF00BFC3D16079022101F050FB5E
:10F9A000607C00283BD0013800BF00BF00BF00BF13
:10F9B00000BF00BF00BF00BF00BF00BF00BF00BF4F
:10F9C00000BF00BF00BF00BF00BF00BF00BF00BF3F
:10F9D00000BF00BF00BF00BF00BF00BF00BF00BF2F
:10F9E00000BF00BF00BF00BF00BF00BF00BF00BF1F
:10F9F00000BF00BF00BF00BF00BF00BF00BF00BF0F
:10FA000000BF00BF00BF00BF00BF00BF00BF00BFFE
:10FA100000BF00BF00BF00BF00BF00BFC3D172B6B0
:10FA200000212046FFF740FF013007D1002020745D
:10FA300062B659E7142001F049F9ADE701212046EB
:10FA4000FFF732FF0130F1D0002500212046FFF7FB
:10FA50002BFF01214DF805002046FFF725FF0DEB98
:10FA600005030835B5F5A07F5860EED162B60022D7
:10FA70005DF832500DEBC203691C586801D0431C7D
:10FA800002D1002020742FE7D1108542635C4FEA39
:10FA90004303DBB202F1010238BF43F00103282A1D
:10FAA0006354E5D16178237822790B44A1780B4423
:10FAB000E1780B44DBB29A42E3D10120E2E7000097
:10FAC0002DE9F8430D462DED028B11460446FFF754
:10FAD000FEFE00287ED0A3790B3B0B2B7AD8DFE803
:10FAE00003F0063F79797979797979796565A37831
:10FAF000E07808EE103A0106B8EE488A48BFFFEEFB
:10FB0000007A00F00F0048BF37EEC88A02F0C4FD4B
:10FB100031A3D3E9002302F029FE064618EE100AAD
:10FB20000F4602F0CBFD0B4602463946304602F046
:10FB300067FC03F013F903466DB102F0BFFD2AA381
:10FB4000D3E9002302F012FE254B002202F058FCFC
:10FB500003F004F90346BDEC028B1846BDE8F883B8
:10FB6000E078A67800F00F0002F096FD1AA3D3E922
:10FB7000002302F0FBFD07EE906AF8EE677A8046FC
:10FB800017EE900A894602F099FD02460B46404660
:10FB9000494602F035FC03F0E1F83206034648BF5F
:10FBA00080F00043002DD6D01846C6E7A678E3784B
:10FBB000300200F4FE40184307EE900AF8EEE77AB0
:10FBC00017EE900A02F07AFD03A3D3E9002302F0B6
:10FBD000CDFDE0E7034BBEE79A9999999999B93F12
:10FBE000000040400000C07FCDCCCCCCCCCCFC3F52
:10FBF000D0B50446FFF76BFE90B3A3790B3B0B2BFC
:10FC00002ED8DFE803F006062D2D2D2D2D2D2D2DC0
:10FC10001C1C607802F040FD14A3D3E9002302F01D
:10FC2000A5FD064620780F4602F036FD02460B463B
:10FC30003046394602F0E4FB03F090F8D0BD20884E
:10FC400040BA80B207EE900AF8EEE77A17EE900A13
:10FC500002F034FD05A3D3E9002302F087FDEBE7B2
:10FC60000148EBE7AFF300800000C07F9A999999B3
:10FC70009999B93F00B55DF804FB0020704700B5C5
:10FC800001205DF804FB10B50446C06803F010FBCA
:10FC9000B4F90600002802DB002101F0D1F920466A
:10FCA00010BD70B50546C0680E4603F001FBEC7C44
:10FCB0002A7C94420CBF0324042414FB06F4A4B24F
:10FCC000AC80204603F0ECFAE86028B1224600211F
:10FCD00003F03BFB6E8070BDA8806880FBE7F0B44A
:10FCE000FF29C1F38107C1F38112C1F301154774E4
:10FCF00001F003078CBF002101210170C168C47CA1
:10FD0000067CC2740574877461B1A41B6142A2EBC6
:10FD1000050561416A426A41914203D04188F0BCC5
:10FD2000FFF7BFBFF0BC704738B5437804460D46B7
:10FD300033B1B0F90600002802DB002101F080F9A0
:10FD40006378E5804BB12846012101F079F9284616
:10FD50000021BDE8384001F09BB938BD70B50E46B2
:10FD60000021044641700172C16041611946154687
:10FD7000FFF7B5FF31462046FFF793FF204629469F
:10FD8000FFF7D2FF204670BD70B540F2FA5404FB75
:10FD900000F303F500431B14B3F5FF7F98B222DA9A
:10FDA000FE2BD8B242DDC0F1FE00C5B20023FF2019
:10FDB0004E1CC943C9B27043013201EB20205043AD
:10FDC00000F47F4406FB03F006FB05F301EB202063
:10FDD00001EB232150434A43120244EA102002F46B
:10FDE0007F02104370BDB3F57F7F0DDAB0F53F7F22
:10FDF000DBB28BBFC3F1FC030233D8B2DBB294BFDA
:10FE0000FF20FF230025D3E7A04211D040F2FA449F
:10FE1000A042DBB204D80433DDB20020FF23C7E7E1
:10FE2000C3F1FA03DBB20020FF25C1E70023FBE7A3
:10FE300000231846F8E7000070B504460830154660
:10FE40000E4600F0C3F8FF23064A84F82230002350
:10FE5000266025712361A382C4E9062223842046FB
:10FE600070BD00BFB3A10100016182827047000034
:10FE7000024B002908BF194681617047B3A10100F8
:10FE8000024B002908BF1946C1617047B3A10100A8
:10FE90000184704773B50D4601690446164639B9A9
:10FEA0002B4BC2685B689A4202D1002002B070BD41
:10FEB000A28A002AF9D094F8223005F00700034105
:10FEC000DB0738D515F47E7F08BF238C206804BF7C
:10FED00003F47E731D43036800292ED05B6A9847A4
:10FEE0000128E2D13C21206800F0CDF80A22294601
:10FEF000206800F024F9237933BB1649206800F00C
:10FF0000B5F8A169206800F0BAF82021206800F057
:10FF1000BAF8E169206800F0B2F82379B3B90E4964
:10FF2000206800F0A3F83146206800F0A8F82068A7
:10FF300003689B6A98470120B8E708490091E16887
:10FF400001911B6A6946CAE70549D7E70549E7E712
:10FF5000D8070020949C01009A9C01001C9D010080
:10FF60008F7E0100A59C010008B5FFF793FF08BD37
:10FF700007B5002300931A461946034800F02EF8EF
:10FF800003B05DF804FB00BFD80700202DE9F8435B
:10FF900006460D46071D00F10709002417F8011B4E
:10FFA0000A22284600F0E4F82E218046284600F078
:10FFB0006AF84F4540440444F0D10A22F1792846BA
:10FFC00000F0D6F82044BDE8F8830000024A026041
:10FFD00000224260704700BF1C9D010030B5837154
:10FFE000034D9DF80C30056001714271C37130BD45
:10FFF0001C9D0100014AC0E9002170471C9D0100C1
:020000021000EC
:10000000024A02600A684260704700BF1C9D0100FE
:100010000B6843607047416070472DE9F041064628
:100020000D4601EB02080C464445A4EB050707D03A
:10003000336814F8011B1B68304698470028F3D139
:100040003846BDE8F08170B5044608460D4604F018
:1000500022F923680246294620465B68BDE87040C5
:10006000184709B1FFF7EFBF0846704708B5FFF71B
:10007000F8FF08BD03688A685B680968184708B517
:10008000FFF7EFFF08BD03681B6818470149FFF73A
:10009000DABF00BF709C010038B50546FFF7E1FFED
:1000A00004462846FFF7F2FF204438BD38B5054620
:1000B000FFF7D7FF04462846FFF7E8FF204438BD86
:1000C00070B58AB00D460AA9002301F8043D012A43
:1000D00098BF0A22B5FBF2F402FB1456F3B2092EC4
:1000E00094BF30333733DBB2254601F8013D002C95
:1000F000F0D1FFF7B6FF0AB070BD2DE9F041074619
:100100000E4615462AB90368C9B21B68BDE8F0411E
:1001100018470A2A05D1002905DBBDE8F041FFF7A1
:10012000CFBFD2B2F9E72D21FFF7ADFF2A46044633
:1001300071423846FFF7C4FF2044BDE8F081FFF765
:10014000DCBF38B50546FFF7D8FF04462846FFF761
:100150009DFF204438BD10B42AB903685DF8044BF4
:100160001B68C9B21847D2B25DF8044BFFF7A8BFAD
:10017000FFF7F1BFFFF7EFBF2DE9F84F194606462D
:10018000104614461D469DF8287002F089FD28B1DE
:100190004C493046BDE8F84FFFF755BF25F0004900
:1001A0004FF0FF32484B2046494602F079FD48B9EE
:1001B0004FF0FF32444B2046494602F053FD08B948
:1001C0004249E6E74FF06042414B2046294602F0A3
:1001D0005DFD08B13F49DCE74FF060423E4B2046F1
:1001E000294602F035FD0028F4D1002200232046E4
:1001F000294602F02DFDD0B12D213046FFF743FFF7
:1002000005F1004382461D463449DFF8D8904FF08F
:10021000000B00204FF000085FFA8BF39F4208D9D3
:1002200042464B4602F0CCFB0BF1010BF4E7824651
:10023000EAE722462B4602F0E3F80D46044602F0B8
:100240006DFD0A22014680463046FFF739FF8244A1
:10025000A7B3404602F010FA02460B462046294654
:1002600002F0CCF804460D4630461D49DFF8749084
:10027000FFF7E9FE4FF000088244013FFFB2FF2F75
:100280001CD04B4642462046294602F06FFA0D46E6
:10029000044602F01BFD0A22014683463046FFF762
:1002A0002CFF8244584602F0F7F902460B462046DE
:1002B000294602F0A3F804460D46DEE75046BDE8A5
:1002C000F88F00BF209D0100FFFFEF7F249D0100FC
:1002D000FFFFEF41289D0100FFFFEFC10000E03F5D
:1002E00061920100000024409DF800100091FFF78A
:1002F00043BF08B54022002103F027F80022C0E9DF
:10030000102208BD026C10B5531C446C03F03F036F
:100310009C421CBF8154036410BD0023C0E910330C
:100320007047D0E9102393421FBFC25C013303F032
:100330003F03436414BF10464FF0FF307047D0E9CD
:100340001030181A48BF40307047D0E9102393424C
:1003500014BFC05C4FF0FF307047036C406C01333A
:1003600003F03F031B1A5842584170470649074A99
:10037000074B9B1A03DD043BC858D050FBDC00F050
:1003800037F8EFF75DFF0000C4A101000000002076
:10039000A0020020FEE7FEE7FEE7FEE7FEE7FEE73D
:1003A000FEE7FEE7FEE7FEE7044B1868421C04BFC9
:1003B000034B1878831F5842584170473001001092
:1003C000E00F00F0074B1B78062B09D1064B1B688A
:1003D000C3F30313033B032B02D8044AD05C7047DA
:1003E00000207047E00F00F0E80F00F0309D0100A2
:1003F00008B5FFF7D9FF28B1654B664A1B68C3F300
:1004000004231360FFF7DEFF10B1634B634A1A60E9
:10041000FFF7CAFF28B1624B624A1B68C3F342333D
:100420001360FFF7CFFF20B15F4AD36823F08073DA
:10043000D360FFF7B9FF40B14FF080430022C3F80B
:100440000C21C3F81021C3F83825FFF7BBFF10B10A
:10045000564B03221A60FFF7B5FF40B1544B0522FB
:100460001A6001229A6700229A603F225A60514B1B
:100470001A68511C0BBF504B504B1A781B6802BFB7
:1004800008331B68C3F30313062A4DD1033B032B28
:1004900003D84B4AD35C002B46D04FF08052494BD7
:1004A000D2F80414C3F82015D2F80814C3F82415A0
:1004B000D2F80C14C3F82815D2F81014C3F82C1570
:1004C000D2F81414C3F83015D2F81814C3F8341540
:1004D000D2F81C14C3F84015D2F82014C3F8441500
:1004E000D2F82414C3F84815D2F82814C3F84C15D0
:1004F000D2F82C14C3F85015D2F83014C3F85415A0
:10050000D2F83414C3F86015D2F83814C3F864155F
:10051000D2F83C14C3F86815D2F84014C3F86C152F
:10052000D2F84424C3F87025FFF73EFF28B1264BCC
:10053000264A1B6803F04F031360FFF735FF48B1ED
:100540004FF08043D3F80024D20744BF6FF001027C
:10055000C3F80024174B1B68062B09D1174B1B68E7
:10056000033B022B81BF1A4A136843F48063136074
:10057000184AD2F8883043F47003C2F88830BFF3C9
:100580004F8FBFF36F8F144B144A1A6008BD00BF22
:10059000240300104035014074C007400DF0ADBA8F
:1005A000440200103C050040F0ED00E0A0050040D2
:1005B0001056004030010010E00F00F03401001030
:1005C0002C9D010000C0004058020010E40E0040C5
:1005D0003C17004000ED00E0180000200090D00320
:1005E00010B5044600F03EFBE06023682046DB685F
:1005F0009847002808DA00F035FBE368C01AA368C2
:100600009842F2D34FF0FF3010BD2DE9F041804603
:100610000D468F180C46BC42A4EB050607D0404699
:10062000FFF7DEFF002802DB04F8010BF3E730469A
:10063000BDE8F0812DE9F8438046894616461C4600
:100640007BB1D7181546BD42A5EB060409D040463C
:10065000FFF7C6FF002804DB814502D005F8010B37
:10066000F1E72046BDE8F88370B50D460949044618
:10067000164600F0D1F92846FFF7B2FF002806DB46
:10068000864204D0C1B2204600F044FAF3E7204687
:1006900070BD00BF729C01000120704703681322E7
:1006A000DB69184770470369C3F81C150369D3F861
:1006B0001C21002AFBD00022C3F81C210120704716
:1006C00010B490F95C30144C59090122203103F028
:1006D0001F0302FA03F344F8213003695DF8044B69
:1006E0000421C3F8081303695A600369DA600369D7
:1006F0000022C3F8002502694FF0FF33C2F80C3521
:100700000269C2F814350269C2F80835026914306A
:10071000C2F81035FFF701BE00E100E01430FFF72A
:100720000EBE1430FFF711BE1430FFF7FABD000003
:10073000036990F85E2010B5C3F80C25036990F8A2
:100740005D20C3F8142590F861200369012A01BFD8
:1007500090F85F40C3F81045036990F8604006BF09
:10076000C3F8084503690022B1F5966FC3F86C25FC
:1007700069D9B1F5166F69D9B1F5965F69D9B1F547
:10078000165F68D9B1F5615F67D9B1F5964F66D943
:10079000B1F5E14F65D9B1F5164F64D9B1F5614FA7
:1007A00064D9B1F5963F64D9B1F5E13F63D9B1F5AC
:1007B000613F63D9364B994263D9B1F5E12F63D9D3
:1007C000B1F5612F94BF4FF070634FF08053026911
:1007D000C2F8243503690422C3F800250169002307
:1007E000C1F808310169C1F81C31016901230B60AE
:1007F00001698B600169C1F8042390F95C205109FB
:1008000002F01F0293406031224A42F8213090F9F1
:100810005C30002BBDBF03F00F0302F6FC32D21890
:100820009B18B5BF60236022137683F8002390F9EC
:100830005C300122590903F01F0302FA03F3154A41
:1008400042F8213010BD4FF49E23C0E74FF41D2322
:10085000BDE7114BBBE7114BB9E7114BB7E7114BA4
:10086000B5E7114BB3E74FF41D03B0E74FF46B034B
:10087000ADE70E4BABE74FF0EB73A8E74FF06C73AF
:10088000A5E74FF08063A2E74FF0E8639FE700BF62
:1008900090D0030000E100E000B0130000502700FA
:1008A00000F03A0000A04E0000C0750000903A0130
:1008B0002DE9F0411E4600254FF47A73C0E901533B
:1008C0000D4B044640F8143B17468846FFF711FDD0
:1008D0000A4AC4F8108084F85C7052F8263084F814
:1008E0005D309DF8183052F8233084F85E3084F87B
:1008F00061502046BDE8F0813C9D0100AC9C0100A8
:1009000010B50369D3F8082104464AB1D3F8181585
:100910001430C9B2FFF7F6FC23690022C3F808219E
:1009200010BD00000148FFF7EBBF00BFE00700204B
:1009300007B5192300930222182303490348FFF740
:10094000B7FF03B05DF804FB00200040E007002083
:1009500010B5044628B103F047FB90FBF4F303FB0A
:100960001404204610BD884210B5044603DA081A64
:10097000FFF7EEFF0444204610BD10B5029C401A5C
:10098000E41A6043521A90FBF2F0184410BD10B5FF
:100990000446006802F08CFC204610BD10B50446E9
:1009A000006808B102F084FC00232360C4E901332D
:1009B00010BD38B504460D460068013103F048FB10
:1009C00010B1C4E90005012038BD036810B5044624
:1009D00023B143688B4201D3012010BD2046FFF7AD
:1009E000E8FF0028F9D0A368002BF5D12268137026
:1009F000F2E770B50E46114604461546FFF7E5FFCF
:100A000020B92046FFF7CAFF204670BDA5603146D9
:100A1000206803F01CFCF7E738B500230446C0E962
:100A2000003383600D4639B1084603F034FC294693
:100A300002462046FFF7DDFF204638BD38B50546A3
:100A400008460C4603F027FC214602462846BDE82E
:100A50003840FFF7CEBF38B5054600680C4668B190
:100A60006A688B689A4207D3096803F0F0FBA368B1
:100A7000AB600023A36038BD02F01AFC23682B6032
:100A800063686B60A368AB600023C4E90033F1E7DF
:100A9000884210B50B46044604D0096821B19A6813
:100AA000FFF7A7FF204610BDFFF778FFFAE710B564
:100AB00000230446C0E900338360FFF7E9FF2046C6
:100AC00010BD884210B5044601D0FFF7C4FF204690
:100AD00010BD10B5044619B1FFF7B0FF204610BD98
:100AE000FFF75CFFFAE770B505460E4609B900202E
:100AF00070BD6AB1846814442146FFF766FF002880
:100B0000F5D02868AB683146184403F0A0FBAC6010
:100B10000120EDE707B500238DF80410012201A99B
:100B20008DF80530FFF7DFFF03B05DF804FB10B56B
:100B30008A6809680446FFF7D6FF10B92046FFF718
:100B40002DFF204610BD826808B53AB921B108785A
:100B5000B0FA80F0400900E0012008BD006809B942
:100B60000078F5E703F069FBF2E7884270B515D02D
:100B700083688A6893420FD183B104680D68013C91
:100B800014F8010F50B104F09BFB064615F8010B59
:100B900004F096FB8642F3D0002070BD0120FCE7F4
:100BA00083688B4201D9006818B903480023037099
:100BB00070470844704700BF440800208368934290
:100BC00010B506D90468A01803F02AFB08B1001B71
:100BD00010BD4FF0FF30FBE70022FFF7EFBFF8B585
:100BE00083689342054602D84FF0FF30F8BD036892
:100BF000541C00221F5D1A550668304603F09AFB0C
:100C000037550028F0D02B68C01AEFE78268013A08
:100C1000FFF7E5BF2DE9F0419A420E461F460F4906
:100C200088BF13461546804684BF3D461F46FFF7E2
:100C3000F3FEB468AC420DD9BC4228BF3C463368D1
:100C400000221F5D1A55316840462944FFF741FFD5
:100C500033681F554046BDE8F08100BF729C01001B
:100C6000FEE700000A4B19680A4B30B5D3F80405BB
:100C70000C060D0A44EA00024FF47A712B46A2FBDF
:100C8000014501FB0355E00B40EA454030BD00BF84
:100C90004808002000100140094B1968094B30B585
:100CA000D3F804050D0A0C06074944EA00022B4656
:100CB000A2FB014501FB0355E00B40EA454030BD76
:100CC000480800200010014040420F0038B504469B
:100CD00048B1FFF7C7FF054600F01AF8FFF7C2FF5B
:100CE000401BA042F8D338BD074B0022C3F80421B3
:100CF00082B0D3F80431054A0193019B1368013394
:100D0000DBB2136002B070470010014048080020B9
:100D1000704770B58AB061B1931E222B20D801AB09
:100D20001D4648B9AB4207D00A46AB4213D8002350
:100D3000137008460AB070BDB0FBF2F402FB140653
:100D4000092E204603F10103F4B294BF3034573426
:100D500003F8014CE5E713F8010D02F8010BE4E795
:100D60000021E6E77047000008B500F015F8FFF72E
:100D7000F9FF0120FFF7AAFFF4F70EFE034CF4F78A
:100D80000DFE002CFBD0AFF30080F8E70000000060
:100D900002F086BA02F08CBA2A4BE02283F81123C3
:100DA0004FF40032C3F880211A604FF080430122D3
:100DB000C3F818259A6003F588330021C3F8081595
:100DC0000221C3F80413C3F844131A604FF0102330
:100DD000D3F80022002A03DBD3F80432002B2FDAE9
:100DE000194B0122C3F80425D3F80024002AFBD0B4
:100DF0004FF010221521C2F80012D3F80024002A67
:100E0000FBD04FF010231522C3F804220E4B1A46D4
:100E1000D3F800140029FBD00021C3F80415D2F840
:100E20000034002BFBD0BFF34F8F0849084BCA6832
:100E300002F4E0621343CB60BFF34F8F00BFFDE7C6
:100E4000704700BF00E100E000E0014000ED00E07D
:100E50000400FA05192837B50CD84B4B53F820304D
:100E6000052B00F0828007D8032B12D07BD8022BF1
:100E700000F08180002074E01D2B78D003D81C2B5B
:100E8000F8D1052206E01E2B73D01F2BF2D10822C9
:100E900000E002223D4B196808296EDD0A296FDD4A
:100EA0000D29B5BF0C240E24022303233848C0F8B3
:100EB000F0350123C0F8003500200546030103F199
:100EC000804303F5E04301300828C3F81455C3F804
:100ED0001055F3D12F4B18682F4B1B6800021B03D2
:100EE00003F4805300F4E0601843294BC3F818055D
:100EF000C3F81425C3F810250DF10602C3F82C26FB
:100F00000122C3F830261A60D3F80021002AFBD052
:100F10000022C3F8002101225A601D4B1A46D3F863
:100F200004010028FBD00020C3F8040101209860D0
:100F3000D2F81431002BFBD00023C2F81431BDF9D4
:100F400006209A42124AB8BFADF80630A142C2F854
:100F50000035BDF9060004D035BF611A091BC84031
:100F6000884003B030BD032294E7042292E70622B2
:100F700090E707228EE701228CE70824002395E7FB
:100F80000A24012392E700BFAC9C01002800002046
:100F9000007000402C00002054080020192830B5B3
:100FA0003CD8224B53F82000214B00221D4653F819
:100FB0002240B4F1FF3F32D11E4C45F822006FEAC7
:100FC00041411D4D1D4B246853F822306FEA5141B9
:100FD00025F81210012101FA04F4C3F86005013C60
:100FE000C3F8640505EB4202C3F86805C3F86C0555
:100FF0000020C3F80015C3F80C05C3F80405C3F8B6
:101000000845C3F81405C3F81005C3F82025C3F834
:101010002415C3F82815C3F82C05996030BD844207
:10102000CAD00132032AC2D1F8E700BFAC9C01004C
:101030001C000020300000204C080020649D0100AE
:1010400019280FD8114B53F8203003290AD8DFE8AC
:1010500001F002160A1003F5E0734FF0A0420021E0
:1010600042F82310704703F5E0734FF0A0420C21C3
:10107000F6E703F5E0734FF0A0420421F0E703F533
:10108000E0734FF0A0420321EAE700BFAC9C0100EF
:1010900019280CD8064B53F82020012393404FF019
:1010A000A04211B9C2F80C357047C2F80835704734
:1010B000AC9C010019289FBF4FF0A043054AD3F80C
:1010C000103552F820009ABF23FA00F000F001001A
:1010D00000207047AC9C010038B50025057329B984
:1010E0000B4B0C4A0C48252101F088FE01600B498E
:1010F00051F82220027151F8233083719DF810308D
:1011000051F8233043710223C371856038BD00BF9D
:10111000709D0100D39D01007E9D0100AC9C0100EB
:10112000037B23B943738373036101230373704704
:1011300084B00DF1100C0CE90E009DF80810026847
:1011400000230129C2F80035039B12D00BD30329D9
:101150000CD0C2F85435019BC2F824350123C2F8E3
:10116000003504B0704743F00203F2E743F0040394
:10117000EFE743F00603ECE710B5FFF7D1FF036894
:101180008279C3F808254279C3F80C250279C3F89F
:101190001025034BBDE810400ECBFFF7C9BF00BFC1
:1011A0006C08002010B485B001AC84E80E0094E80F
:1011B0000E0005B05DF8044BFFF7BABF7047036837
:1011C000C3F81C15D3F80821002AFBD0D3F8180562
:1011D0000022C3F80821C0B27047000007B5094BD0
:1011E00009490A484FF080421A6000229A600222A0
:1011F0001A710B2300930C220D23FFF76DFF03B030
:101200005DF804FB6C080020003002405808002004
:101210000B460146184601F01BBE0000C0F3C75341
:101220007F3B162B024605DC002B04DB03481841EC
:1012300022EA0000704700F000407047FFFF7F0087
:101240002DE9F04FDFF82C938DB006460F4614467B
:101250001D4600F095F999F90080B8F1FF3FCDE9FE
:10126000000136D022462B462046294601F018FDC3
:10127000834670BB32463B463046394601F010FD8E
:101280008246002840F0A2803046394600220023E2
:1012900001F0D4FC10B3002200232046294601F0BF
:1012A000CDFC8346002867D09FEDA77B0122AC4B85
:1012B000CDF828A00292CDE90467CDE906458DED71
:1012C000087B0393B8F1000F41D09FEDA17B8DED1A
:1012D000007BDDE900010DB0BDE8F08FDDE9000124
:1012E00000F066FF8046002800F08D804FF0000A75
:1012F0004FF0000BDDE9000152465B4601F09EFC19
:101300000028E6D03046394600F052FF0028E0D0F1
:101310002046294600F04CFF0028DAD099F9003029
:101320008F4A039204210022022BCDE90467CDE904
:101330000645CDE908AB02910A9203D002A800F05D
:101340003DFF50B901F092FD2223036005E002A8A1
:1013500000F034FF002800F09B800A9B1BB101F0D5
:1013600085FD0A9B03609DED087B8DED007BDDE92B
:1013700000010DB0BDE8F08F2046294600F018FFAF
:101380000028A6D0002200232046294601F060FC58
:1013900000289ED0724A99F90030CDF828B001217A
:1013A000CDE90467CDE90645CDE90212002B74D0E2
:1013B0006C490020022BCDE9080172D101F056FDE5
:1013C000212303600A9B002BCDD0C8E70022002315
:1013D0002046294601F032FC00283FF47AAF624BE8
:1013E0005F49CDF828B000220120B8F1020FCDE905
:1013F00004670290CDE90645CDE908230391A6D103
:10140000CDE9002365E73046394600F0D1FE0028DB
:101410003FF46CAF2046294600F0CAFE00283FF496
:1014200065AFDDE900231046194601F039FC99F952
:1014300000A000286BD10323DFF824C10A902946BD
:10144000204602930022494BCDF80CC0CDE9064559
:10145000CDE9046701F08AF904460D46BAF1000FA0
:1014600025D1DFF814B14FF0604A00220023304646
:101470003946CDE908AB01F0EBFB38BB02A800F020
:101480009DFE00289ED101F0F1FC2223036099E724
:1014900001F0ECFC212303605FE79FED2B7B8DEDDA
:1014A000087B02A800F08AFE00288BD186E79FED1A
:1014B0002A7B00220023304639468DED087B01F05F
:1014C000C7FBA0B9BAF1020FDDD0D7E72046294605
:1014D00000F07CFE22462B4601F0B0FBA0B9244B65
:1014E00099F900A04FF06042CDE90823EAE72046D1
:1014F000294600F06BFE22462B4601F09FFB18B9EF
:10150000184B0022CDE9082399F900A0DAE701225F
:10151000134BCDF828800292CDE90467CDE906454A
:101520000393BAF1000FB8D00022002310461946E9
:1015300001F046FABAF1020FCDE908013FF43EAFDF
:10154000AFE700BFAFF30080000000000000000024
:10155000000000000000F03F000000000000F07FED
:10156000109E01000000F0FF0000F03F0000E03F8F
:10157000FFFFEFC734000020FFFFEF47000000002F
:101580002DE9F04F23F0004555EA020493B00DD049
:101590006B4E21F00044B4420F4682460BDD04F14D
:1015A000404404F5801454EA0A0350D165490020F0
:1015B00013B0BDE8F08F9B46944647D0B542EEDCB1
:1015C0005F4EB5425DD0002F80468946CDE90023AD
:1015D0005BDB0026BCF1000F0ED1594B9D423FD082
:1015E000584B9D4200F08880BBF1804F00F09C80FA
:1015F000554B9B4500F0B8834046494600F0D4FD6A
:10160000BAF1000F06D1002C59D04E4B27F04042C2
:101610009A4254D0FF0F013F56EA070373D04B4B59
:101620009D4240F39B8003F104739D4240F33E844E
:10163000474B9C4272DDBBF1000F72DD3EA3D3E944
:1016400000231046194601F091F8B1E728B141484E
:1016500013B0BDE8F04F00F0B3BDA542F7DCAFE733
:1016600004F1404303F5801353EA0A039ED0384B3C
:101670009C4240F38383BBF1000F52DBDDE90001A4
:1016800096E7BCF1000F9ED089E7334B9D4231DCD9
:10169000A3F154739D429CDD2B15A3F2FF33142B51
:1016A00040F3A583C3F134032CFA03F202FA03F3E7
:1016B00063458ED102F00102C2F102068AE7BBF156
:1016C000000F05DA02460B4600201E4901F078F9AA
:1016D000002FBFF66DAF04F1404404F5801454EAC6
:1016E000060300F03F84012E7FF462AF01F1004356
:1016F00019465DE702266DE7BBF1000FC0F2488393
:101700004046494654E742464B461046194600F0CB
:1017100075FE02460B4601F053F949E7BBF1000F95
:101720008CDB0020002143E742464B4640464946B9
:1017300001F01CF83CE700BF9C7500883CE4377E54
:101740000000F07F0000F03F0000E03F0000E041BB
:10175000FFFFEF3F149E0100FFFF3F43B4F5801FE2
:1017600080F261830022D24B01F000F86FF0340C5C
:101770000C462315CF4DC4F31302A3F2FF3342F0FE
:101780007F546344AA420B9344F4401440F33F83D4
:10179000C94B9A4240F304849FEDAF7B8DED087BEB
:1017A0008DED107B9FEDAE7B0B9B8DED067B0133AA
:1017B0000B93A4F580140025DDE90623214682461B
:1017C00000F01CFEA346DDE906238046894650460C
:1017D0002146CDE90CAB00F013FE02460B4600207B
:1017E000B64901F0EDF80A460146CDE90E1213465E
:1017F00049460246404600F0B9FF631043F00053EB
:1018000082468B4603F500238C46CDE904AB59197B
:10181000D3460023CDE902BC0293DDE902AB0020F0
:1018200004460D4602460B465046594600F09EFFC0
:1018300002460B464046494600F0E0FDDDE906233E
:10184000804689462046294600F0D8FD02460B46D0
:10185000DDE90C0100F0D2FD52465B4600F086FF48
:1018600002460B464046494600F0C8FDDDE90E231E
:1018700000F07CFFDDE90445CDE9060122462B4658
:101880002046294600F072FF77A3D3E900230446DF
:101890000D4600F06BFF76A3D3E9002300F0B0FD06
:1018A00022462B4600F062FF73A3D3E9002300F029
:1018B000A7FD22462B4600F059FF71A3D3E9002370
:1018C00000F09EFD22462B4600F050FF6EA3D3E9A8
:1018D000002300F095FD22462B4600F047FF6CA345
:1018E000D3E9002300F08CFD2246804689462B4632
:1018F0002046294600F03AFF02460B46404649463C
:1019000000F034FF524604460D465B46DDE9040113
:1019100000F076FDDDE9062300F028FF22462B4685
:1019200000F06EFD5246804689465B465046594659
:1019300000F01CFF0022624BCDE90C0100F060FDBD
:1019400042464B4600F05CFD02980D460446224696
:101950002B465046594600F009FF002282468B462E
:10196000574B2046294600F049FDDDE90C2300F0E5
:1019700045FD02460B464046494600F03FFDDDE985
:10198000042300F0F3FE2246804689462B46DDE91B
:10199000060100F0EBFE02460B464046494600F0C9
:1019A0002FFD8046894602460B465046594600F0B8
:1019B00027FD029838A3D3E9002304460D4600F022
:1019C000D5FE5246CDE904015B462046294600F08B
:1019D00015FD02460B464046494600F00FFD30A378
:1019E000D3E9002300F0C2FE2FA3D3E900238046F1
:1019F00089462046294600F0B9FE02460B4640467D
:101A0000494600F0FDFCDDE9102300F0F9FC8046BA
:101A10000B98894600F040FE424682468B464B4674
:101A2000DDE9040100F0ECFCDDE9082300F0E8FC4E
:101A300052465B4600F0E4FC029852465B46044680
:101A40000D4600F0DBFCDDE9082300F0D7FCDDE902
:101A5000042337E0AFF30080000000000000000026
:101A6000000000000000F03FEF4E454A287ECA3FCC
:101A700065DBC9934A86CD3F01411DA96074D13F02
:101A80004D268F515555D53FFFAB6FDBB66DDB3F14
:101A9000033333333333E33F000000E009C7EE3F45
:101AA000FD033ADC09C7EE3FF5015B14E02F3EBEB3
:101AB000000040438E98030079B60B000000F03F11
:101AC0000000084000F09AFC0B460246494640469A
:101AD00000F094FC013E56EA070382468B4600F074
:101AE0005E819FEDD37B8DED047BDDE90012002349
:101AF0000E461746CDE902670293DDE90267084604
:101B00003B461146324600F079FC22462B4600F057
:101B10002DFEDDE90023804689465046594600F0F7
:101B200025FE02460B464046494600F069FC324617
:101B3000804689463B4620462946CDE9008900F08B
:101B400015FE0B46024606460F464046494600F043
:101B500057FCD14B994204460D468A4640F32481F6
:101B600001F13F4303F5E003034340F0FF81B2A3DB
:101B7000D3E90023DDE9000100F042FC3246804653
:101B800089463B462046294600F038FC02460B4673
:101B90004046494601F07AF8002840F0E781A8461F
:101BA0004FEA2853A3F2FE324FF4801313415344FB
:101BB000C3F30A52B94DA2F2FF321541C3F3130425
:101BC00023EA05010020C2F1140B44F48014BAF199
:101BD000000F02460B4644FA0BFB30463946B8BFAD
:101BE000CBF1000B00F00AFC06460F463246DDE959
:101BF00000013B4600F004FC4FEA0B5A0D4600245E
:101C00008FA3D3E900232046294600F0AFFD3246DA
